:020000021000EC
:10F000000000012039F5010061F5010063F5010000
:10F0100065F5010067F5010069F5010000000000D9
:10F020000000000000000000000000006BF501007F
:10F030006DF50100000000006FF5010019220400C9
:10F040004D4F020073F5010089520200AD4F0200DE
:10F05000015002009D620200F553020073F50100A9
:10F0600073F501005D22040073F5010073F50100E2
:10F0700073F501005D5D020073F5010073F5010099
:10F0800059220400152B020073F5010073F50100ED
:10F090001D2C02005DDB0300111C020073F5010052
:10F0A00073F5010073F5010073F50100FD640200C2
:10F0B00073F5010073F5010000000000000000007E
:10F0C00073F5010073F5010073F5010073F501009C
:10F0D00073F50100295F020073F5010000000000D4
:10F0E0000000000000000000000000000000000020
:10F0F0000000000000000000000000000000000010
:10F1000000000000000000000000000000000000FF
:10F1100000000000000000000000000000000000EF
:10F4000010B5054C237833B9044B13B10448AFF35E
:10F4100000800123237010BD602D0020000000003B
:10F4200028C4060008B5034B1BB103490348AFF3DA
:10F43000008008BD00000000642D002028C40600E4
:10F44000154B002B08BF134B9D46A3F5803A0021B6
:10F450008B460F461348144A121A00F063F80F4BFC
:10F46000002B00D098470E4B002B00D0984700206F
:10F47000002104000D000D48002802D00C48AFF315
:10F48000008000F02BF82000290026F06FFA00F031
:10F4900011F800BF0000080000000120000000007B
:10F4A00000000000602D0020E0E3002000000000CC
:10F4B0000000000008B5074B044613B10021AFF36C
:10F4C0000080054B1868836A03B19847204600F016
:10F4D00031F800BF000000005800060070B50D4D67
:10F4E0000D4C641BA4100026A64209D10B4D0C4CF8
:10F4F00040F0A6FD641BA4100026A64205D170BDF5
:10F5000055F8043B98470136EEE755F8043B984719
:10F510000136F2E7482D0020482D0020482D00201C
:10F520004C2D002002440346934200D1704703F85B
:10F53000011BF9E7FEE700BF0649074A074B9B1A84
:10F5400003DD043BC858D050FBDC06F0DBFDFFF7C1
:10F5500077FF000034C40600402C0020602D0020FE
:10F56000FEE7FEE7FEE7FEE7FEE7FEE7FEE7FEE773
:10F57000FEE7FEE72DE9F04F00250646A84628469F
:10F580004FF480744FF6FF7C2E270B78B8F1000FF4
:10F5900000D1013003F0C00EBEF1C00F11D0013117
:10F5A0009BB283B3013CE41A24B2002C33DBB8F1E4
:10F5B000000F00D1184401F1FF3A02F1FF399E46D5
:10F5C00012E0B8F1000F00D1013049781B0203F4BA
:10F5D0007C530B44F1180131F35C4FF00108E0E774
:10F5E0001AF801BF09F801BF0EF1FF3E1FFA8EFEA7
:10F5F000E645F5D102EB030E194401331A448EF8A7
:10F6000000700135C1E715B92E2302F8013B002334
:10F610001370BDE8F08F4FF0FF30FAE71FB50123FC
:10F620008DF80030054B8DF8080001916846D3E94C
:10F630000012904705B05DF804FB00BF9CCA002093
:10F6400061DF704748DF704710B50388012B11D880
:10F65000094A02EB031243885189CC1A032C09D4BE
:10F66000C3F57F43FD330B44538100230380438064
:10F67000184610BD0420FCE7A0CF002010B5124AA8
:10F680000B6802EB0010426873B15888033003EB3B
:10F69000800302F580524FF6FF749A4202D918682F
:10F6A000013004D1002009E002F10803F1E7988855
:10F6B000A04204D0188810B10B60012010BD5888FA
:10F6C000033003EB8003E8E7A0CF002073B5436865
:10F6D00004460D4613B31E4A11688B421ED352686E
:10F6E00093421BD813F0030018D11A4A21891289BA
:10F6F000914213D121689A6891420FD1164A5268FB
:10F70000934201D80A2004E002F580529342F9D2D4
:10F710002880B0FA80F0400902B070BD00232B8031
:10F720001E46019601A92888FFF7A8FF30B92B884B
:10F7300001339BB22B80002BF3D0EDE7019B2268B5
:10F7400099689142EED16360024B1B892381E3E704
:10F75000502D002060CC0020A0CF0020033083B2C9
:10F7600040F2FD32934230B50ED909200BE02289D8
:10F7700065892A441A4492B2B2F5806F08D2088093
:10F7800062891344638130BD024C20780028EED09A
:10F790000720F8E7A0CF002010B50A494A788C78F6
:10F7A000531CDBB29C4208BF00230C789C421FBF55
:10F7B0000370486802EB420200EBC20008BF002061
:10F7C00010BD00BF1CCF0020AADF7047A9DF704723
:10F7D000A7DF704785DF70477FDF70477EDF7047A8
:10F7E000084A30B500230C2404FB03F18D5A8542EE
:10F7F00002D10A44508830BD0133082BF4D14FF6B2
:10F80000FF70F8E7CACB00206EDF704758B1CB0815
:10F8100001F00701C25C012303FA01F10A4214BF9F
:10F8200018460020704701207047000070B50A4E4E
:10F830003468054654B1706860B1FF2D08D0294680
:10F84000FFF7E4FF30B1F36803FB0544204670BDC9
:10F850000024FBE70446F9E724D10020012804D066
:10F86000043804288CBF0020012070478378013BB6
:10F87000072B07D8DFE803F007060606060704098A
:10F880001423038070470123FBE743689B880933F7
:10F890009B08F6E770B5054D0646002455F8043B75
:10F8A000304601349847052CF8D170BD5802060047
:10F8B000114BF0B5002214261D4606FB02F4E75A50
:10F8C000874212D12344142600249A788A420AD00F
:10F8D00001342246072A0BD806FB02F3EF5A87426F
:10F8E00008D1EB18F1D11846F0BD0132082AE4D155
:10F8F0000023F8E70132EDE734D1002030B50721CD
:10F9000085B0FFF7D5FF044600283AD04568002DA2
:10F9100039D1007CFFF78AFF0721CDE902558DF828
:10F920000A1040B3E368039003EB83031B019BB20F
:10F930009B0802A8ADF80830FFF798FF9DF80A0071
:10F94000FFF78CFFD8B1114B1B789B0715D5BDF87D
:10F9500008500DF106012846FFF700FF48B9BDF831
:10F960000630A380E5800A4B185C092803D005B057
:10F9700030BD0928F7D90320F9E70220F3E708464C
:10F98000F5E70520F3E70020F1E700BF5DCC00209C
:10F990007400060038B54FF6FF73984218BF013067
:10F9A0000D4614BF84B20024FF2C03D94FF6FF7418
:10F9B000204638BD21462846FFF728FF0028F7D10A
:10F9C0000134A4B2F0E70000F8B5074D074E074632
:10F9D00000243378A34200DCF8BD55F8043B3846D8
:10F9E00098470134F5E700BF3CCC0020EDCD002066
:10F9F0007DDF704779DF70476DDF704738B5074CA2
:10FA0000051E04F1080318BF1C4623682BB11A68B1
:10FA100022605B6828469847F7E738BD74CB002022
:10FA200040DF70473FDF704737B5D0F818350A7DA3
:10FA3000DBB28DF807300B7F9A4282BF0A699DF8CE
:10FA40000740D4540B7F0D7B0133DBB25A1C954227
:10FA50000B7705D98B689B5CC0F81C3501200AE048
:10FA60000C7D944201D9CB7EF6E7AB42F6D3A3429C
:10FA70002CBF0020012003B030BD0023435082B0D2
:10FA800043580193019B02B070472DE9F0470D7870
:10FA90009DF820609DF824A004460F469946002D4D
:10FAA00060D1D0F8243192F800809BB14FF492716C
:10FAB000FFF7E3FF012363613B70B04550D1D4F8F9
:10FAC0000431002B4CD04FF482712046FFF7D5FF54
:10FAD00000251DE0D0F81C31FBB14FF48E71FFF70B
:10FAE000CCFFD0F824311BB14FF492712046DFE7F0
:10FAF00013789E4207D919F80330C0F81C351378E3
:10FB000001331370D9E70123BAF1000F03D0C361A9
:10FB10002846BDE8F0874361CFE7D0F80831002BD5
:10FB2000CBD04FF48471FFF7A8FFD0F82431002B1D
:10FB3000DAD113789E42C0D9D0F8181509F803100D
:10FB400013780133DBB21370721E934205D1022386
:10FB5000C0F8003201232362AFE79E42FAD1ACE73E
:10FB60000125D5E74FF49271FFF787FF4FF48E71AF
:10FB7000FFF783FF4FF48471FFF77FFF9FE72DE9C5
:10FB8000F3470C4605464FF4827120461F469046C7
:10FB9000FFF773FF4FF49271FFF76FFF4FF48E7111
:10FBA000FFF76BFF4FF48471FFF767FF0023012F0E
:10FBB00085F8263085F8233008BF02224FF0010374
:10FBC0000CBFC4F80022C4F80032236223602E6800
:10FBD00046BB05F1260A05F12309CDE90076434627
:10FBE000524649462046FFF750FF0028F5D195F8C8
:10FBF0002330EBB1D4F8C434C4F8C434C3B113F027
:10FC0000010F14BF4FF40240032048F2012213F009
:10FC1000020F18BF104613F0040F48F2022318BF5A
:10FC2000184606E040F28623AB60AB68C4F80433A4
:10FC3000002002B0BDE8F0872DE9F3470C460546E9
:10FC40004FF4827120461F4616469DF82880FFF724
:10FC500014FF4FF49271FFF710FF4FF48E71FFF70E
:10FC60000CFF4FF48471FFF708FF0023C4F8003243
:10FC700085F8263085F8233001232362A36095F8A8
:10FC80002620974232D9B35CC4F81C3595F826304B
:10FC9000013385F826302B687BBB05F1260A05F178
:10FCA0002309CDE900783346524649462046FFF7FE
:10FCB000ECFE0028F5D195F8233023B3D4F8C434F2
:10FCC000C4F8C434FBB113F0010F14BF4FF4024069
:10FCD000032048F2012213F0020F18BF104613F060
:10FCE000040F48F2022318BF18460DE0B8F1000FC8
:10FCF00001D0E361CFE76361CDE740F28623AB60DB
:10FD0000AB68C4F80433002002B0BDE8F0872DE9E9
:10FD1000F04793F9005090B00024013D6E46AD00CD
:10FD20002746A446A0465FF0000E03E05FEA080EF7
:10FD3000BEEB050EB8EB0E0952F809A051F80E9073
:10FD4000A9FB0A9A14EB090457EB0A075CF1000CB3
:10FD50001EF1040EAE4501DCC645EBDD46F8084059
:10FD60003C4667465FF0000C18F10408A845DADD50
:10FD7000B8EB450FDADD46F80840D3F8B03031462D
:10FD8000984710B0BDE8F08713460A46FFF7BFBF9B
:10FD9000F0B5154689B01C4607460E461A46294658
:10FDA0006846FFF7F1FF23466A4639463846FFF7B3
:10FDB000AEFF23462A4669466846FFF7A8FF23465A
:10FDC0006A4631463046FFF7A2FF09B0F0BD00EBAE
:10FDD00081010023884200D3704751F8042D43EA83
:10FDE00052030B60D307F5E710B5013A52B2130680
:10FDF00001D5002010BD50F8224051F822309C421D
:10FE000005D802F1FF32F2D24FF0FF30F2E70120C5
:10FE1000F0E710B500235CB2A24200DC10BD51F83F
:10FE2000234040F823400133F5E7013910B549B2CA
:10FE3000041D0A06CBB204D4013954F82120002A4B
:10FE4000F7D001335BB273B103F18042013A50F84D
:10FE50002220002022B9013B00EB431318B210BD51
:10FE600052080130F6E71846F9E7002310B51C46A2
:10FE70005AB2914200DC10BD40F823400133F7E74D
:10FE8000C3F10803DB0070B50133002403A500BFF4
:10FE90005B1920C940CAAD1B20C0184720C940CA01
:10FEA000B54120C020C940CAB54120C020C940CAC0
:10FEB000B54120C020C940CAB54120C020C940CAB0
:10FEC000B54120C020C940CAB54120C020C940CAA0
:10FED000B54120C06441B4FA84F0400970BD00BF50
:10FEE000C3F10803DB0070B50133002403A500BF94
:10FEF0005B1920C940CAAD1920C0184720C940CAA3
:10FF0000754120C020C940CA754120C020C940CADF
:10FF1000754120C020C940CA754120C020C940CACF
:10FF2000754120C020C940CA754120C020C940CABF
:10FF3000754120C06441204670BD00BFF0B5082265
:10FF400089B00C460646FFF764FFCB6A03930B6B40
:10FF500004934B6B05938B6B0693CB6B0793002736
:10FF600008236A4669466846CDE901770097FFF79E
:10FF7000B7FF082305466A4631463046FFF7B0FF13
:10FF8000236B0393636B0493A36B0593E36B0544AB
:10FF9000CDE906376A46082369466846FFF7A0FFA1
:10FFA000082305446A4631463046FFF799FF236A25
:10FFB0000093636A0193A36A0293A36B0693E36BB6
:10FFC0000793054408236A4631463046CDE9047755
:10FFD0000397FFF785FF636A0093A36AA26B0193FF
:10FFE000E36A02930492636BE26B0393CDE905230A
:10FFF000236A0793054408236A4631463046FFF7D3
:020000022000DC
:100000006FFFE36A0093236B0193636B0293236A90
:100010000693A36A0793054408236A46314630468F
:10002000CDE904770397FFF72BFF236B0093636BF6
:100030000193A36B0293E36B0393636A0693E36AF2
:1000400007932D1A08236A4631463046CDE90477D6
:10005000FFF716FF636B0093A36B0193E36B0293AF
:10006000236A0393636A0493A36ACDE90537236B7C
:1000700007932D1A08236A4631463046FFF700FFE2
:10008000A36B0093E36BCDE90137636A0393A36A23
:100090000493E36ACDE90537636B07932D1A0823B0
:1000A0006A4631463046FFF7EBFE2D1A0D4C0FD451
:1000B00035B9082231462046FFF796FE01280FD0B9
:1000C0000823224631463046FFF7DAFE2D1AEFE7C5
:1000D0000823224631463046FFF702FF2D18F7D499
:1000E00009B0F0BD900006002DE9F04391B00F4635
:1000F0001C220021804609A8FFF714FA01251C22C2
:10010000002101A80895FFF70DFA394608AA11F950
:10011000046B009533461046FFF7E2FE314608A80F
:10012000FFF783FE013804B2012C07DC3246694632
:100130004046FFF76EFE11B0BDE8F0833A466846D0
:100140006946FFF721FE10AB601103EB80001FFA38
:1001500084F909F01F0350F8202C05FA03F3134229
:1001600005D03B46424669466846FFF7D0FD09F197
:10017000FF3424B2D8E770B5036813F001050646D2
:10018000144605D013460A460146FFF7A9FE054668
:1001900021463046FFF71BFE45B104F18042013A8B
:1001A00056F8223043F0004346F8223070BD70B557
:1001B0009DF910401E4623460546FFF761FE38B103
:1001C0002346324629462846BDE87040FFF788BEE0
:1001D00070BD2DE9F0438BB01446129D15F9046BE8
:1001E00000961F46804689462B460246214602A8B5
:1001F000FFF7DDFF02A9129A0846FFF7C5FD129B23
:1002000002AA41464046FFF782FD129B02AA214600
:100210002046FFF77CFD2B464A4639463846009675
:10022000FFF7C5FF129A394602A8FFF7ADFD02A9F4
:100230002B46424608460096FFF7B9FF02A92B4617
:10024000224608460096FFF7B2FF2B46424621465B
:1002500020460096FFF7ABFF129B224649464846D0
:10026000FFF755FD2B4602AA414620460096FFF7B0
:100270009EFF129B224639463846FFF748FD2B4623
:100280004A46394638460096FFF791FF324602A9A2
:100290002046FFF7BEFD0BB0BDE8F08370B59DF9B9
:1002A00010401E4623460546FFF71AFE30B9224687
:1002B00029463046FFF798FD012807D023463246ED
:1002C00029462846BDE87040FFF7DABD70BD2DE92C
:1002D000F0439BB01646229C14F9045B00959846A7
:1002E0000746894623460246314612A8FFF75FFFBC
:1002F00012A9229A0846FFF747FD229B12AA394607
:100300003846FFF704FD229B12AA31463046FFF71C
:10031000FEFC23464A46414612A80095FFF7BEFF61
:1003200023464A46414640460095FFF740FF234694
:100330003A4631460AA80095FFF739FF229B0AAAE0
:1003400049464846FFF7E3FC2346324639460AA8A9
:100350000095FFF7A3FF229A41463046FFF714FDB0
:1003600023460AAA314630460095FFF720FF234670
:100370003246394602A80095FFF719FF229B02AAD0
:1003800041464046FFF7C3FC23464A4641464046A5
:100390000095FFF70CFF229A12A902A8FFF7F4FCC0
:1003A00002A923460AAA08460095FFF700FF234644
:1003B0003A4602A90AA80095FFF7F9FE0AA9229B6E
:1003C00012AA0846FFF7A3FC23464A460AA9484654
:1003D0000095FFF7ECFE2A4602A93846FFF719FD03
:1003E0001BB0BDE8F0832DE9F04115468AB0044604
:1003F00088461C22002103A8FFF794F82E1D95F9CA
:10040000007003232A46414620460293FFF7BCFCB6
:10041000334602AA214620460097FFF7C8FE2B4626
:10042000424621462046FFF772FC0097334605F10D
:10043000840221462046FFF731FF0AB0BDE8F08173
:100440000C4B1B78062B10D10B4B1B681A070CD1D9
:100450000A4B186800F0F003302B08D000F0E000E1
:10046000A0F14003584258417047002070470120D6
:10047000704700BFE00F00F0E40F00F0E80F00F05D
:10048000094B1B78062B0CD1084B1B681A0708D1A7
:10049000074B186800F0F000A0F1300358425841B3
:1004A00070470020704700BFE00F00F0E40F00F03D
:1004B000E80F00F010B9024B01221A60704700BF2C
:1004C0000050004010B50C494A6E042A044611D071
:1004D0000B6E1344032B02F101024A6688BF043BF2
:1004E000182202FB031318460021FFF71BF82060B7
:1004F000012010BD0020FCE740D0002010B50446CC
:1005000086B01422002101A8FFF70CF86088ADF82E
:100510000800FFF765F92378ADF80600092B0CD821
:10052000DFE803F005051014161B1D0E1F2107231D
:100530008DF8043008238DF80C3001A8FFF744FA39
:1005400006B010BD0D238DF80430F6E70E23FAE750
:1005500007238DF804300523EDE70F23F3E710237D
:10056000F1E70523EFE706238DF80430A368039332
:10057000A388ADF80630E0E708B5134644F201025F
:10058000904203BF5A681988986800221BF0FCFE4D
:1005900030B50B4B1B68012293F8641021338A425B
:1005A00004DB405CB0FA80F0400930BD13F8014B29
:1005B000855CA54201D10132F1E70020F5E700BFDB
:1005C000F0C9002070B5244B0022C3F80025234A4F
:1005D000516831B12249C3F8081322490420C1F8F7
:1005E0008000D3F80C55D3F81445D3F80815D3F888
:1005F00010054FF0FF36B542C3F8146518BF05F576
:10060000E075C3F80C65C3F80865C3F810651EBF34
:100610004FF0A043022643F82560651C1FBF4FF032
:10062000A04304F5E074022543F82450441C1FBF86
:1006300000F5E0704FF0A043022443F820404B1C2B
:100640001FBF4FF0A04301F5E071022043F82100E5
:100650000023D376536070BD002000409CCA002068
:100660008402020000E100E02DE9F04F85B08A46E7
:100670000390039C2578284633F0AAFA0746D8B998
:100680002D2D1CD10134012303940193DDF80CB00E
:10069000BAF1000F01D0CAF800B00022114603A839
:1006A00033F03EFA8046002835D1614D00242046C3
:1006B000294605B0BDE8F08F01340394D9E72B2D0E
:1006C00004BF013403940190E0E71846029333F02D
:1006D00012FAB0F10009029B20DBC8451EDD40463E
:1006E0003EF0DAFE22462B463EF040FF04460D4621
:1006F00048463EF0D1FE22462B463EF081FD0136B3
:1007000004460D460396039E3378002BDDD1B8F1E5
:100710000A0F37D113E000240025F4E7B8F10A0FDF
:1007200030D12E2B0BD10FF20019D9E900890136F7
:100730000396039E30783038C3B2092B39D9039B16
:100740001A7802F0DF02452A1CD15A1C03925A780B
:100750002D2A01D02B2A05D12D3A574203F102034D
:10076000574103934FF000080A20039A1378303B57
:10077000D9B2092936D9002F39D12E4F0026B8F128
:10078000000F46D1039BBAF1000F01D0CAF8003028
:100790009B458AD09BF800202E2A03D10BF1010B38
:1007A0005B4582D0019B002B81D005F100431D46A3
:1007B0007DE73EF071FE42464B463EF0D7FE0246D4
:1007C0000B46204629463EF01BFD002204460D46FE
:1007D00040464946174B3EF0F3FF013680468946B6
:1007E0000396A6E7013200FB08380392BDE7114FDC
:1007F000C8F100080026B8F1000FC3D020462946F2
:1008000032463B463EF0DCFF08F1010804460D4647
:10081000F1E72046294632463B463EF0A7FE08F166
:10082000FF3804460D46AAE79A9999999999B93FD4
:100830000000F87F0000244070B58AB00C460146E5
:1008400068461D4633F0A6FE0022214605A833F077
:10085000A1FE684633F0E7FD044605A833F0E3FD4A
:100860008442064621D0039850B1C389A3F5007392
:100870009BB2C381C38903F4F0530BB938F01AFC5F
:10088000089850B1C389A3F500739BB2C381C38993
:1008900003F4F0530BB938F00DFC002C01DB002EF3
:1008A00000DAF5B9A01B0AB070BD002C1BDA039862
:1008B00050B1C389A3F500739BB2C381C38903F40C
:1008C000F0530BB938F0F6FB089850B1C389A3F583
:1008D00000739BB2C381C48914F4F05401D138F081
:1008E000E9FB0020DFE7684633F02EFB05A833F074
:1008F0002BFBAEE7044A138A9BB223F0410343F07B
:1009000040031382704700BF8C2D002030B587B0A4
:100910000A46014601A833F03DFE0025DDE901321B
:10092000934205F1010401D2013514D1049850B16C
:10093000C389A3F500739BB2C381C38903F4F05349
:100940000BB938F0B7FB20202DF042FA14F1FF3438
:100950000DD207B030BD059810B1C05C0A28E5D0B3
:100960002DF036FA01A8254633F0EEFAD6E7082036
:10097000EAE730B587B00D46019009B100230B605E
:100980000021102202A8FEF7CDFD02A901983BF03C
:100990000BF8E0B10024029B039A23F07F4303335A
:1009A00023F00303013203F110030AD11C44002297
:1009B00002A901A83BF032F80028ECD1204607B08C
:1009C00030BD002DF3D02A6813442B60EFE70446B6
:1009D000F4E730B587B04FF4DA240021102202A8E2
:1009E0000194FEF79FFD02A920463AF0DDFF70B1A9
:1009F000002202A901A8DDE901543BF00FF800280C
:100A0000F6D124F07F4413352C4424F00304C4F5BC
:100A1000EC2007B030BD2DE9F04F89B0D51C019313
:100A200025F00305002382468B46174610350393B5
:100A3000984604AC039E86B330463AF0B9FF804630
:100A400003983AF0DBFF064678B1039BC21A954241
:100A50000BD9FB1A0344984507D9B5F5007F04D29A
:100A600021463AF0A1FF00B90396019B039947EA9A
:100A7000036710224FF0FF33204605930497CDE91A
:100A800006AB20F065FD129B23B194E80F00129C89
:100A900084E80F00039E103638E04FF4DA23039306
:100AA000B146214603983AF07FFF78B1059B0133A8
:100AB00006D1DDE906235B4504BF5245DDF80C9005
:100AC0000122214603A83AF0A9FFEEE703983AF085
:100AD0006FFF85421ED903983AF090FF01230390DF
:100AE0000398C8B9B9F1000F0BD0214648463AF037
:100AF0005BFF0422002309EB020105A8059320F007
:100B000027FD039878B9B8F1000F11D0304609B02D
:100B1000BDE8F08F0023E3E7002BC2D13AF048FF95
:100B20008542BED8DEE73AF043FF8742EBD881E743
:100B30003BF09AF880460028E8D00023039379E739
:100B40002DE9F04F8DB002AFB3F10009C7E9020102
:100B500092463E6D4FF0000519DBAE4217DB07F100
:100B6000100110463D6138F091FE804600BB5046B2
:100B700035F0E2FB0446386132F066FE04F580731E
:100B8000834209D95A49012033F0E8FF002528465D
:100B90002C37BD46BDE8F08FE31D23F00703ADEB16
:100BA000030D0DF1080822464146504635F0B4FBCE
:100BB00006B93E6907F1180B5A46D7E902013AF027
:100BC00058FF044620B9B9F1000F2FD04949DAE7A0
:100BD000B9F1000F35D1BB691A0E05D1B34203D16B
:100BE00031463AF09FFF60BBBD6925F07F439E42CE
:100BF0001CD12D0E1AD1D7F810A0564516D1331F8F
:100C000010E062597A619D428CBFAAEB0502042272
:100C100008EB050107F114007B603FF0ADF928B93E
:100C20007B680435AA45ECD80125B0E7CDF800B0C3
:100C300000233246D7E90201FFF7EDFE0446002803
:100C4000C4D03969BB6909EB010223F07F439A42A2
:100C500001D9294997E74C4420463AF063FF0546FD
:100C600020B92649012033F079FF90E714F0030002
:100C70001FD0A4EB0009C0F10406D9F800307B6155
:100C80003B699E4228BF1E4607F1140318443246B2
:100C900041463FF07FF90422494607F1140020F055
:100CA00057FC3B69B3427FF672AFB04434449E1B9D
:100CB0003E613A6902F00306921B3A611AB121467D
:100CC000404620F045FC002E3FF461AF39690C44EA
:100CD000324623687B61414407F114003FF05AF922
:100CE0000422214607F1140020F032FC4FE700BF38
:100CF0004D0106007401060092010600AE010600D7
:100D00000C4A002330B41146184640F6C41401EBD7
:100D100003151032E8819D1C0133A34222F80C5CBC
:100D2000F5D149F634430122C852034B1A8030BC36
:100D300038F06AB8AC2D0020AA2D002070B586B01E
:100D400015460C460022014601A833F023FC2E462E
:100D5000DDE901239A4210D3049850B1C389A3F569
:100D600000739BB2C381C38903F4F0530BB938F00D
:100D7000A1F900232370AD1B0DE07EB9049850B19A
:100D8000C389A3F500739BB2C381C38903F4F053F5
:100D90000BB938F08FF9284606B070BD059B03B13A
:100DA0009B5C04F8013B01A833F0CEF8013ECFE78D
:100DB00037B50123009300231A460A49044638F048
:100DC00033FA05465CB1E389A3F500739BB2E38176
:100DD000E38903F4F05313B9204638F06BF9284641
:100DE00003B030BD4F020600F8B5858907460C46B2
:100DF00095B31A4B013D03EB05152846EB8903F526
:100E000000739BB2EB8139F0A5FAEB89A3F500736F
:100E10009BB2EB81EB8903F4F053461C13B92846CF
:100E200038F048F9304637F02DFD214638F08CFE79
:100E3000044680B10146384639F002FBE389A3F548
:100E400000739BB2E381E38903F4F05313B92046A6
:100E500038F030F9701CF8BD0126E3E7AC2D002016
:100E600038B5074C25780023EDB2024619462370A9
:100E700037F08AFA25700348BDE838402CF096BF59
:100E8000A82D002025B6060070B5044638F0F6F807
:100E90000546B0B120460022184939F025FC044629
:100EA00037F033FF78B900255CB1E389A3F500730F
:100EB0009BB2E381E38903F4F05313B9204638F081
:100EC000F9F8284670BD00220D49204639F00CFC87
:100ED00006460028E7D00B492EF020FDF389A3F544
:100EE00000739BB2F381F38903F4F0530546002BA2
:100EF000DAD1304638F0DEF8D6E700BF3E02060011
:100F00000244060048020600002370B50B60054647
:100F10000E4637F03FFD044610B90025284670BD47
:100F2000294638F0EDFC054668B9E389A3F500735E
:100F30009BB2E381E38903F4F053002BEDD120460B
:100F400038F0B8F8EAE7204637F029FF3060E38947
:100F5000A3F500739BB2E381E38903F4F053002B04
:100F6000DCD1ECE7F0B54FF080530220D3F85014F9
:100F7000D3F85424284BC3F804032848C3F80403C7
:100F8000274B93F800E093F801C09F78DE781D7935
:100F90005C7998794EEA0C033B4333432B4323435C
:100FA0000343204B2AD083F800E083F801C09F70F0
:100FB0001E715D719C71D8711D789C785A785E792C
:100FC000586885EA0401514081F08801D970197987
:100FD00071409E797140DE797140197212020321CD
:100FE000597242EA05420C4B2243C3F8942500BAD9
:100FF0004422C3F89005C3F8A025F0BD080A197073
:10100000090C9970110A1A715971110C120E58704D
:101010009971DA71D0E700BF0050004080000800ED
:1010200014CF0020FFCE00202DE9F0471546804662
:1010300015F8014B894644F480740F2601F1510ADA
:101040004F46574504D10136312EF9D1BDE8F0871E
:10105000220606D5D8F80C3032463946404627F0ED
:1010600015FC6400E30348BF15F8014B07F10107C5
:1010700048BF44F48074E4E738B50022054639F0EF
:1010800033FB044698B100231A460146284630F047
:101090000BF9E389A3F500739BB2E381E38903F4C1
:1010A000F05323B92046BDE8384038F003B838BDC6
:1010B00070B5EFF3108672B60D4A94680123A4B997
:1010C00093600C4B0C4DD3F8801029401160C3F88D
:1010D0008050D3F8841051604FF0FF32C3F8842061
:1010E000047006B962B6002070BD0370F9E700BF56
:1010F000DCD1002000E100E0FC06FFBC10B588B0A8
:1011000012788DF80C20CDE90001FF220021029118
:101110008DF80D2001214FF6FF72104C8DF81C1038
:10112000ADF80E208DF810302BF018FA70B132F0B7
:1011300067FB58B914F1FF34F6D20949042033F0A3
:101140000DFD68462BF01AFA08B010BD002CF4D043
:1011500032F056FB0028F0D1F3E700BF80841E0078
:10116000250206002DE9F341314C637E0546002B34
:101170005BD123680BB10123637695E80F002D4EF8
:1011800086E80F00A27E637F2B4E23F00303FF2A25
:1011900063771EBF012393404FF0A0424FF0000140
:1011A00018BFC2F80C35254B21770422C3F8082359
:1011B0003160316800910099297939B32A68127831
:1011C000C3F81C252A79012A22D92A685278C3F843
:1011D0001C2525680DBB194FDFF85480D7F808315E
:1011E000002BFBD035603368019341463846019BA4
:1011F000FEF71AFC0028F1D1A27EFF2A12D00123AB
:1012000093404FF0A042C2F808350BE0E27ED7E7EA
:101210002A7B012ADDD9E27ED9E7084B0422C3F8F4
:101220000423002002B0BDE8F0811120FAE700BFDE
:10123000E0CA0020E8CA0020083100400030004029
:1012400037B50B015BB249B2044643EA01008DF8A1
:1012500004001A4D50B20343120152B28DF805300A
:101260002B78114302438DF806108DF8072013B335
:1012700002AB03EB941302AA13F8040CC4F301139A
:10128000134413F8043C43EA002020F0D3F82B78F1
:101290008BB102AAC4F3810304F003041344144481
:1012A00013F8040C14F8043C43EA002003B0BDE832
:1012B000304020F0BFB803B030BD00BFEAD10020FD
:1012C000C30914BF13020B0270B510F0400F0D4696
:1012D0000CBF29461146194306461320144620F038
:1012E00033FAB1064CBF23022B0216F0100F14BFC5
:1012F000214629461943132020F026FA32074CBF15
:1013000023022B0216F0040F14BF2146294619436D
:10131000132020F019FAB3074CBF2102290216F05E
:10132000010F08BF2C4621431320BDE8704020F078
:101330000BBA00002DE9F047FF2705463C4604267E
:101340004FF6FF78296911B9002E61D051E0286865
:1013500029F0ADFB064600284BD168690378002BC5
:101360005ED0C27AE52B02F03F0247D022F0200186
:10137000082943D00F2A46D159063DD503F0BF04B2
:10138000EB88477B2B84437BBB4237D10378EE69E4
:10139000DFF890E003F03F03013B0D2253434FF091
:1013A000010C00211EF8019B00EB090292F801A03C
:1013B00010F8092042EA0A22BCF1000F20D03E2B8F
:1013C0001CD826F813209446013301310D29E9D1A8
:1013D0000278520604D53E2B10D8002226F813209E
:1013E000013CE4B20021284629F016FD06460028FB
:1013F000A8D000232B610CE0A342C4D0FF24F1E766
:101400004245E2D0FAE73CB927F070FFB84203D179
:1014100000263046BDE8F0874FF6FF732B84F8E7CF
:101420000426E6E77E0006002DE9F047ADF5127DC3
:1014300080460CA80D4622F00FFF32F0E9F9C0F308
:101440000E02002302F5FA620221404622F048FE15
:101450004045F2D1AA4A1388013312AC9BB21380E3
:101460005BBA238001234FF480722946638052A81F
:101470000023C4E901233EF0CFFD52A83EF0C4FD95
:1014800015AB1FFA80FA0DF5A4791D4649460A7876
:101490000F4601312AB12E2AF9D1A7EB0906B6B2BF
:1014A00001E05646174603F8016B5EB11846324616
:1014B00049463EF0B1FD03463344002F40F093808F
:1014C00003F8017B01225A70DA7000211A1D19708D
:1014D0009970121B3523009392B20DF142032146FD
:1014E000404622F049FA20F01FFB10F580130293CA
:1014F00041F100030393404622F0F4F80646002829
:1015000000F0EF80B0F5807F28BF4FF480760DF1BA
:101510001603B2B221460093404606AB22F03CFBD4
:10152000404622F0FFFA0023ADF81E30227863789F
:10153000E07894F8058003EB0223ADF81C30A37823
:1015400000EB032080B2020444BF01238DF81E305B
:10155000C0F3C3238DF81F30430544BF01238DF82A
:101560002030870544BF01238DF82130C60544BFD4
:1015700001238DF82230010644BF01238DF823306A
:101580002379E779227A08EB0328A37907EB03276D
:10159000637A03EB0223ADF82A30A27AE37A00F0F3
:1015A0000F061FFA88F8BFB203EB02238DF8246000
:1015B000ADF82680ADF82870ADF82C304FF000095A
:1015C0001FFA89F3434515D3DFF838814FF000093E
:1015D0001FFA89F39F421AD8B6FA86F040090DF532
:1015E000127DBDE8F087721CF643B24491441FFAA5
:1015F0008AFA4BE7294652AA2046FDF7BBFF421C58
:101600001ABF2D180435002509F10109D8E752AA9F
:1016100029462046FDF7AEFF431C03D1002509F102
:101620000109D5E729182A5C4B7803EB02239BB20A
:10163000013B01F10A050E2BF1D801A252F823F06B
:101640007D160200AF1602001F1602001F160200D0
:10165000AF160200BF160200AF160200AF1602005E
:10166000AF1602001F1602001F160200AF1602007E
:101670009B1602001F160200AB1602008B7A88F838
:101680000030CB7A88F801300B7B88F802304B7B36
:1016900088F8033001F10E05C1E701F10B028B7AE6
:1016A000D05CD51801300544B9E701F10C05294695
:1016B00052AA2046FDF75EFF411CF4D1AEE752AAC4
:1016C00029462046FDF756FF421CA7D0054452AAE2
:1016D00029462046FDF74EFF431C9FD00544143594
:1016E0009DE74FF47A7018F0DBFF20F01DFADDE97A
:1016F000022382428B41BFF6FEAE30466FE700BF49
:10170000A42C00207C2D002010B5074A002332F8BD
:10171000024B8C4203D1184100F0010010BD01338F
:10172000082BF4D10020F9E7F8C90020F0B5224BCE
:101730009F7C1C4600221D46D6B2B7420ED895F8B3
:1017400078701D4C0022D6B2B74216D895F8DE50FC
:101750000022D4B2A54220D800200DE0B4F814C075
:10176000844502F1010204F10A04E5D142F64D2359
:1017700001200B808870CE70F0BDB4F87AC060454F
:1017800002F1010204F10A04DDD142F64D230B807F
:1017900002238B70CE700120EEE7B3F8E060B04218
:1017A00002F1010203F10A03D3D142F64D230B806B
:1017B00003238B70CC70EEE76CCC002010B50C4C82
:1017C000226886B0034682B104208DF804000868C0
:1017D000D989ADF80C10123333F8021C0290ADF821
:1017E0000E10049301A92046904706B010BD00BF1B
:1017F0006CCC00207FB54B89022B0FD1094A1368AE
:1018000063B1097B0068029011F0010F14BF02213F
:1018100003218DF80410104601A9984707B05DF820
:1018200004FB00BF6CCC002070B50D4D002435F8D2
:10183000026B964210D10122A240D2B2D543EDB242
:10184000014410F8014B2BB11443884200F8014CBD
:10185000F7D170BD2C40F8E70134082CE7D1F8E748
:10186000F8C9002070B50023084C1A4641FA02F569
:10187000ED0706D504EB420600EB4305B688AE80C3
:1018800001330132082AF1D1036070BDF4C9002090
:1018900010B586B004460022684616F017FF2046B1
:1018A000009916F0CDFC204606B010BD38B50123D6
:1018B0000B7004460D4637F028FA88B100220B4918
:1018C000204638F011FF10B139F095FB2870204602
:1018D0000022074938F008FFBDE8384039F076BAF1
:1018E0002046BDE8384038F035BD00BF4001060055
:1018F00045010600084B5A6E013A5A6622B907495B
:101900000A7822F002020A701A6E0132042A08BF15
:1019100000221A66704700BF40D000205ECC002035
:1019200030B5044685B00D46102200216846FDF70B
:10193000F9FD237A012B0AD0022B0ED063680193A4
:10194000236829469B686846984705B030BD2369DF
:101950000293A38AADF80C30F0E70123A2898DF839
:101960000030E389ADF80A20D31AADF80830E5E776
:1019700028DF704729DF704738B51C4B5A6E19466F
:101980005AB31C6E182202FB04331A7A012A07D0BC
:10199000022A23D018460921BDE83840FFF7C0BF0E
:1019A0001825D88A9A8A05FB0414D4E90314121A5C
:1019B000B2F5806F4FEA80000144B4BF92B24FF499
:1019C00080622044FFF7D6FF11280BD1084A137814
:1019D00023F0020343F00403137038BD9889FFF726
:1019E000C7FFF1E70028F8D0D4E700BF40D00020BF
:1019F0005ECC0020054A137813F0060F04D143F0A3
:101A000002031370FFF7B8BF704700BF5ECC002021
:101A10002DE9F3411F4B1B781746DA070646884627
:101A20002BD51D4D1D4B9D4229D31D4B9D4226D2CA
:101A300039B330B341EA00039B0724D12B689842A5
:101A400023D36A6800EB87039A421ED3FFB101A833
:101A5000FEF738FD78B1019B0024C3E90054019BD7
:101A600001221A72C3E903869F82FFF7C3FF204653
:101A700002B0BDE8F0810720FAE70120F8E7022074
:101A8000F6E70320F4E70620F2E70520F0E704205C
:101A9000EEE700BF5ECC0020502D0020502D00202E
:101AA000602D002038B5074B074A596894881068A4
:101AB0004A880332032592B200EB84001D70FFF7C1
:101AC000A7FF38BD60CC0020E4D0002010B5012273
:101AD0000C460649FFF79CFF28B9054901EB0411A4
:101AE00001238B7310BD0E20FCE700BF6C020600C3
:101AF000A0CF002008B502220149FFF789FF08BDE9
:101B00007002060008B5034B034918680222FFF76C
:101B10007FFF08BDE4D000207802060073B51B4BA0
:101B20001B78DB0705462BD5194E1A4B9E4229D34D
:101B3000194B9E4226D238B3C0F30B04D4B9336894
:101B4000984219D3726800F580539A4214D301A8C1
:101B5000FEF7B8FC90B1019BC3E90064019B02222F
:101B60001A722D0B01229D811A82FFF743FF204636
:101B700002B070BD0620FBE70520F9E70720F7E774
:101B80000120F5E70220F3E70320F1E75ECC002017
:101B9000502D0020502D0020602D002010B50B4C42
:101BA0000B4B628803EB02139A892AB95868FFF736
:101BB000B5FF0423237010BD05232370054B0222BB
:101BC00018689A80FFF7AAFFF5E700BF60CC0020F5
:101BD000A0CF0020E4D0002008B5074B191D58887D
:101BE000FDF74CFD18B1BDE80840FFF75BBFBDE84D
:101BF0000840FFF7D3BF00BF60CC002060DF704714
:101C000010DF7047002208B511461AF0BDFB000036
:101C10002DE9F347254B1B681BB1984730B3FFF7FD
:101C2000F1FF234B1B7803F0FF07FBB1214D224E40
:101C30002C68DFF88C90B4FA84F46409B0463378E9
:101C4000A3B901A8FDF7FEFC052812D00028E6D1B3
:101C5000019B0BB9FDF7D2FE184B1B680BB1019825
:101C600098474CB10124EAE7002CFBD002B0BDE854
:101C7000F087002CFAD13C46DFF848A098F80030F5
:101C8000002BF3D1B9F80030ADF80430DAF80030A9
:101C900001A91846FDF7D4FC0528E5D00028BED1DF
:101CA0002A6818469047002CE8D1C8E74CCC0020A1
:101CB000E1D000202CCA0020E2D00020ECD000208F
:101CC00028CA0020D4D1002010B5084B9A685AB118
:101CD00050B9EFF3108172B6054A1C6814605C6855
:101CE0005460986001B962B6002010BDDCD10020BC
:101CF00000E100E02DE9F3411D4F7B6806460D46EB
:101D00009BB304292FD943697BB3437C0024012B67
:101D10000DF107000CBF8846A0468DF80740FFF77D
:101D2000C7F90DF10600FDF737FDD0B101230370AF
:101D3000104B4660D3F80435C0E90484C0E902358D
:101D40009DF806307B709DF80700FFF7BDFF24B9B2
:101D5000094B4FF48012C3F80021204602B0BDE8C1
:101D6000F0810424EFE70724F7E70824F5E700BF34
:101D70001CCF00200010014000E100E02DE9F341FC
:101D8000CE0801F007044FF0010808FA04F4855D5D
:101D9000E4B22540074613D10DF107008DF8075036
:101DA000FFF786F9BB5D9DF807001C4202BF1C438C
:101DB000BC554546FFF788FF284602B0BDE8F081D4
:101DC0000025F9E72DE9F3478146002701261FFA90
:101DD00087F84FEAD80A08F0070406FA04F419F85D
:101DE0000A50E4B2254008D00137B7F5807FEED124
:101DF000B846404602B0BDE8F0870DF107008DF807
:101E00000750FFF755F919F80A309DF807001C42F2
:101E100002BF1C4309F80A400125FFF755FF002DBA
:101E2000E2D0E6E773B50546B8B1C1F3C70401F0E7
:101E3000070301269E40035D33420ED000230DF1BF
:101E400007008DF80730FFF733F92B5D9DF8070089
:101E500023EA06062E55FFF737FF02B070BD0000DB
:101E600038B50A4B1A687AB15D686DB1FF280BD09E
:101E700084B221462846FDF7C9FC28B121462846F0
:101E8000BDE83840FFF7CEBF38BD00BF24D10020E9
:101E90002DE9F74F9846531E072B81460F461546EE
:101EA00000F2BB80FF2800F2B88001465E48FDF7D3
:101EB000ADFC0646002800F0B08039464846FDF7E4
:101EC000F7FC044600283ED0C3689D4247D805D29F
:101ED0005FFA85F9E368207C994543D394F8109024
:101EE000B9F1FF0F40F09780504B1A689B46002ACB
:101EF00041D14FF6FF732380A3700023C4E901335F
:101F0000E360238A03F4784343F0FF032382112024
:101F100084E0237C1844C0B2FFF7A2FFE3685FFAB5
:101F20008AF083420AF1010AF3D84FF6FF73238047
:101F3000A3700023C4E90133E360238A03F47843E8
:101F400043F0FF032382FF214FF6FF70FDF7B0FC43
:101F500004460028DBD0A0F800908770BEE74FF061
:101F6000000ADBE74844C0B209F10109FFF778FF36
:101F70005FFA89F9AEE75B68002BBAD00023DBF883
:101F800008205FFA83FA924502D34FF0FF0912E06E
:101F9000DBF8040060B351460193FFF7EFFE019BAD
:101FA00030B3B9F1FF0F08BFD146AAEB090A0AF115
:101FB000010AAA4521D1B9F1FF0F84F8109098D0F9
:101FC000E560207CFDF732FC58B305EB85052D015B
:101FD000ADB2AD0888F80270C8F80400A8F8005047
:101FE00026B1082F02D1AD00063D8580002015E006
:101FF000B9F1FF0F0CD14FF0FF090133BFE748469D
:10200000019309F10109FFF72BFF019B5FFA89F9A1
:10201000D145F4D3EFE70026D2E7072003B0BDE8AF
:10202000F08F0320FAE700BFF8CF002024D1002072
:1020300038B504460025E368AB420ED84FF6FF736F
:102040002380A3700023C4E90133E360238A03F4EF
:10205000784343F0FF03238238BD207C2844C0B27C
:10206000FFF7FEFE0135E6E737B5FDF721FC054633
:10207000A0B144682CB10A4B01941B789B0706D48D
:1020800003242846FFF7D4FF204603B030BD01A843
:10209000FDF7DAFA04460028F3D0F1E70524F3E768
:1020A0005DCC0020FF2810B5044609D8014605483C
:1020B000FFF7B8FE21460448BDE81040FFF7B2BE66
:1020C00010BD00BFF8CF002018D0002013B50DF1CF
:1020D00006010446FDF7FAFA70B1BDF80620084B78
:1020E00003EB02139A894AB1A17A39B1013A00206F
:1020F0009A81A07202B010BD0A20FBE70620F9E722
:10210000A0CF002037B50D460DF106010446FDF7BE
:10211000DDFA88B1BDF80620084B616803EB0213B5
:1021200000209A8901329A81296063680C336B60C0
:102130000123A37203B030BD0A20FBE7A0CF00202B
:102140002DE9F043DFF88480D8F874E0BEF1030F86
:102150000F46944635D81C4E756CC1F108039D425C
:102160002FD8D8F8704074441C2304F0030481462F
:1021700003FB0484B9E80F000FC499E807000EF1CF
:10218000010384E80700C8F87430C7B1336C2B44EE
:1021900003F0070306EBC303002206F138040CEB3F
:1021A000C20103C9A34202F1010283E8030014BF84
:1021B0000833054B9742F2D1736C1F4477640120BA
:1021C00000E00020BDE8F08324CB002024CF0020D5
:1021D0002DE9F0411C46184B1B789B0706460F461D
:1021E000154627D5DFF85880A3880BB10A201FE0D9
:1021F00098F800302BB92146A088FDF73FFA20B9A6
:102200002060A3880133A380EEE723681EB199887C
:1022100032889142EFD11FB119883A889142EAD1B0
:102220009B682B6023686B60044B1B892B8100200B
:10223000BDE8F0810220FBE75DCC002060CC0020EF
:10224000A0CF002030B587B04CF2070305460C46FE
:10225000ADF8043003AA0F4B01A90020FFF7B8FF27
:1022600010B1002007B030BD01A903A8FFF74AFF55
:102270000028F6D10723A370019B5A882280029A76
:1022800062609B8803F580432B8003A8FFF71EFF45
:102290000120E7E750CC00201FB50023A0F58040C7
:1022A000A1F58041CDE90233ADF80400ADF8061088
:1022B00002AB0DF1060101A8FFF78AFF002818BF45
:1022C000052005B05DF804FB2DE9F04102230B80E9
:1022D000164B00251C6800F5805E2F4608304FF62F
:1022E000FF7870450AD305B11C6002B11770BDE8D4
:1022F000F08101270EE0344601250BE00668013627
:10230000F1D086884645F4D00688002EF1D0866844
:10231000A642F0D8468806F1030C00EB8C00B1F819
:1023200000C00CF1030C66440E80DAE7E8CD002013
:1023300070B5064D0646002455F8043B0BB13046F7
:1023400098470134082CF7D170BD00BF00CB0020A6
:102350002DE9F047AA4C266F1C2707FB06F586B02F
:10236000635D013B8046052B00F22A81DFE813F014
:102370000600640064001D011D017E0130B1A14A08
:10238000137823F00103137001201FE025442B79FB
:10239000032B15D8DFE803F002072C34FFF7B2FB5C
:1023A00001232B7109E0984D2B78022B40F03C82E1
:1023B0006868FFF79FFB00232B70002800F0F08077
:1023C000904A137823F0010313700E201C237343EB
:1023D000E218E35C0290023B012B00F232818B4B4E
:1023E000907D196C5A6C0144121A19645A6428E1E0
:1023F000874F3868FFF792FB0223BB800023D0E7AA
:10240000834FDFF804823868FFF774FB814BD7F8FD
:1024100000E05B88B7F804C01B0108EB03025168B9
:10242000A2F808C0C2F804E00222BA800022396093
:1024300008F803202A71C0E707FB0647724BB7F87C
:1024400012A04FEA0A1A03EB0A029946118960B1F9
:10245000FB8803F103088844C3F57F435189A2F840
:102460000880FD330B4453818EE7536803EB8108EA
:102470003B7C062B00F29780DFE803F02D733C4D88
:102480001F84040041F61D501C2303FB0643D14466
:10249000DB88B9F80810DA1C0A44A9F80820C3F54B
:1024A0007F43B9F80A20FD331344A9F80A3041F6F6
:1024B0001D53984200F0C38088E7574857490023CE
:1024C00043601C2303FB06439B690360FDF7FEF892
:1024D000002800F04C81291D012221444046FFF7CD
:1024E00097FA1C2303FB064302221A74002857D0D4
:1024F0000E20C9E705F10C010122214408F1080072
:10250000FFF786FA1C2303FB06439A7D002A14BFBB
:1025100003220122E9E73D4B5A6C002A00F08C812E
:10252000196C1C2505FB0645481C00F0070003EB51
:10253000C1071864A88A53F83110013A5A6408EBAD
:102540008000BA88FFF764FAAB8ABA881344AB827A
:10255000AB7D013BDBB2AB75002BC7D101232B74E4
:10256000C4E705F108010122214408F10400FFF746
:102570004FFA1C237343E25C032A0CBF0522062298
:102580002344B2E7254B1988234B5868FFF79EFA7E
:102590001C2303FB064306221A7400287FF474AF41
:1025A00006B0BDE8F0870F206EE700287FF4ECAEA0
:1025B00007FB06473B79012B32D01BB1022B3ED0E3
:1025C0000F2003E7CDE90200FB6801930DF1020142
:1025D00001A8FDF77BF880B10298BDF8021083884E
:1025E000FB8003883B81FFF771FA1C2303FB064342
:1025F00002221A710028D3D059E70A20F5E700BF5C
:1026000024CF00205DCC0020A0CF002024CB0020D0
:10261000E4D0002060CC0020802D0020E8D10020F4
:10262000864FA81D3B4601AA41462044FFF7D0FD36
:10263000B8B9B9880298FFF749FA0A28DAD1002315
:1026400002931C2303FB06F2A25C013A052A00F266
:10265000B580DFE812F08E009200A000CB00D5001C
:10266000E1000A28C7E90088E9D020E700287FF4C4
:102670008BAE734BDA7AAAB1D8721A78013A062A6D
:102680009ED801A151F822F0392702003327020019
:10269000492702004F270200C125020055270200EA
:1026A000652702001A78072AE7D801A151F822F01D
:1026B000D12602007B2602007B260200ED260200C6
:1026C000012702001F2702001F270200E92602003F
:1026D0001A8901321A8100225A80DA72594A127814
:1026E000B2FA82F252099A72012207E056495868FA
:1026F0008A884088033202448A8002221A70BCE72A
:102700005D88504A504902EB0512086855685060D0
:102710008888108102228A800D600622EEE7072257
:10272000ECE7484900229A728A8942B9897B31B123
:102730005A80FFF751FA5DE79A7A002AF1D1002218
:102740001A705A805A607AE7FFF7ACF952E7FFF740
:1027500025FA4FE75A883B4B03EB02135868FFF703
:10276000C9F947E700225A60FFF7CCF942E70A208F
:102770002CE600238DF8043020E003FB0643012201
:102780008DF804201A89ADF810209A88ADF812202F
:10279000DB68039312E003FB064302228DF804205A
:1027A0001A89ADF810209A88ADF81220DA681B7CDF
:1027B00003929A1F534253418DF8143001A8FFF73A
:1027C000B7FD206F1C22002102FB0040FCF7AAFE8F
:1027D000636F1BB3226F013202F00302013B2267D9
:1027E0006367DBB10020FFF7B3FDD9E603FB0643C7
:1027F00003228DF80420DA88ADF810201A89C5E785
:1028000003FB06430422DB88ADF8103000238DF86B
:102810000420ADF81230D1E70523ABE70B4A13785B
:1028200023F004031370BBE6084A137843F0020355
:1028300023F00103137002E71368FFDEF0D10020DC
:1028400060CC0020A0CF0020E4D000205DCC002090
:102850000846FFF77DBD0000054A137813F0040019
:1028600004D143F004031370FFF772BD704700BF3B
:102870005DCC0020F0B51C463D4B1B789E0789B00F
:1028800007460D466FD509884FF6FF7399426CD005
:102890006B88002B69D06968B5F808C000239C4597
:1028A00003D8BAB9164604310AE051F8330080075C
:1028B00057D10133F3E731F83200304486B20132A8
:1028C0009445F8D80DF102013046FCF747FF28B1D6
:1028D00009B0F0BD13885688ADF8023000238DF89A
:1028E0001430BDF80230ADF816300323ADF81830BF
:1028F000204B8DF804401A6829898DF81A1001328E
:102900001A602B88ADF80C30032C6B88ADF80830BA
:1029100004BF04238DF81430049208BF3B686A6832
:1029200008BF0793002401A8ADF80A60ADF80E4077
:10293000FFF706FC50B9BDF802200F4B03EB021362
:1029400058890338801B58810820C1E7049B3B60ED
:102950000A4B7C601B89BC723B81FFF77DFF2046E0
:10296000B6E70320B4E70220B2E70420B0E700BFD7
:102970005DCC0020E8CD0020A0CF002060CC00205E
:1029800030B58BB0FF28044601921D4645D88B78A0
:102990001846FCF763FF00283FD04A6802920A8875
:1029A000ADF80C20A4F58042ADF81C20A3F58042C0
:1029B000ADF81E2002AA08920122ADF82420194683
:1029C00004AA2046FFF768FC0528019A0ED10223CD
:1029D00052B907A904A8FFF74DFF07281FD010D848
:1029E000B0B103200BB030BD01AAF2E732B10E4BFB
:1029F0001B789B0702D501A8FCF726FE03230022C3
:102A0000E7E708280DD00E280CBF11200320E9E7C6
:102A1000002DE7D0049B2B60E4E70720E2E7862047
:102A2000E0E71120DEE700BF5DCC00201F4B204A0D
:102A30001B6800BF00BF00BF00BF00BF00BF00BFDA
:102A400000BF93422FD000BF00BF00BF00BF00BF38
:102A500000BF00BF00BF00BF00BF00BF00BF00BF7E
:102A600000BF00BF00BF00BF00BF00BF00BF00BF6E
:102A700000BF00BF00BF00BF00BF00BF00BF00BF5E
:102A800000BF00BF00BF00BF00BF00BF00BF00BF4E
:102A900000BF00BF00BF00BF00BF00BF00BF00BF3E
:102AA00000BF00BF00BF0138C3D17047A82C002071
:102AB0000024F40073B5154E736805461BB34369D3
:102AC0000BB3002404740DF107008DF80740FEF7E6
:102AD000EFFA0DF10600FCF75FFE90B102230370E0
:102AE0009DF80630456073709DF80700FFF7ECF81D
:102AF00024B9074B4FF48012C3F80021204602B0DE
:102B000070BD0424F0E70824F8E700BF1CCF0020C4
:102B100000E100E02DE9F8432649274B0025C1F8E4
:102B20004051C1F84451C1F84851C1F84C51C1F865
:102B30000051C1F804511B68002B39D0D1F804456D
:102B40001E49DFF88C800968641A24F07F442F4600
:102B50001A68A24217D8A41A15441A7CDE6982B1F9
:102B6000D8F800901F74D3E90521B9F1000F06D001
:102B70001046C84728B1FFF745F83346E8E708464E
:102B80009047002EF9D10E4A0E4B11781B788B42DC
:102B900005D10133DBB2022B08BF0023137012787A
:102BA000094B43F82250094B4FF48012C3F800211F
:102BB000BDE8F88300100140D8D10020FCD00020EF
:102BC000F9D00020F8D00020F0D0002000E100E093
:102BD00048CC00200D4B0E494FF4003210B5C3F81D
:102BE000802001244FF48033C1F848332F20C1F8EE
:102BF00008334C60FFF71AFF064B8C602F20002132
:102C00001960FFF713FF044B197010BD00E100E0DD
:102C100000100140FCD00020D9D000202DE9F04F59
:102C2000B64AB74913780978B64D85B09942D5F8B8
:102C30000080019500F095800133DBB2022B08BFC4
:102C4000002313701278B04B53F82260019A08EBFE
:102C5000060323F07F4313600127AC4BAC4A18688E
:102C60000290AC48117890F800904FF0000CE246CA
:102C70005078884278D1BCF1000F02D0A54981F884
:102C80000090002F40F0BB801F6802997F1A18BF88
:102C900001270020196802919E49039191F800E0F4
:102CA00000244FF00108002840F0AD8092F8019018
:102CB000D2F804C092F802A01178494540F0C180D2
:102CC0001B68029A9A4201D1002F44D0002B00F0D9
:102CD0001281D3F80090904C019BD4F804651968D8
:102CE0008E4F751A3B7825F07F450335A3B94FF415
:102CF0008033C4F84433C4F80433894B4FF40032B2
:102D00004FF00108C3F880212F201A60C4F800801A
:102D1000FFF78CFE87F80080A9452CBF494449196C
:102D200021F07F41C4F84015D4F804359B1B23F0F3
:102D30007F43891B033321F07F418B420BD9D4F8A9
:102D40000435C4F840352F20FFF770FE744B4FF464
:102D50000032C3F80021039A0023137005B0BDE8C8
:102D6000F08F0026374678E701EB4104506892F86F
:102D700002B000EBC40E013110F834401868C9B23B
:102D80008B4508BF0021022C04D0032C7FF470AFC8
:102D9000002410E0DEF804B004468646002C3FF420
:102DA00067AFA34500F0C080A646E469F6E780F867
:102DB00010A0C06901240028F9D1002C3FF458AFBD
:102DC000186055E7D4F80C90C4F800E0761A8C44EB
:102DD000E1691960B9F1000F07D008EB0C0121F08F
:102DE0007F41C4E90119E06120461C68002C3FF4D2
:102DF00051AF2168B142E5D98E1B26604AE7002019
:102E000084468646F1E70146C069019DD1F804A0D9
:102E10002E68444DD1F80890AAEB060C2CF07F4C9C
:102E2000AC4535D80CEB09060E60D3F800C081F82C
:102E30001080C1E90144CC61BCF1000F33D11960AD
:102E400031E701EB410B0131C9B2514514BF11709B
:102E500014701CF83B1001290CEBCB067FF42CAF4F
:102E6000716891F810B0BBF1000F7FF425AFD6F870
:102E700008C0C1F804C0F5688D603569CD60766919
:102E80008E61BEF1000F0CBF66465E464E60BCE729
:102E9000A6EB0A0626F07F464E4502D2A9EB0606AF
:102EA000C2E70C60C1E7D1F80090DCF80060B145E2
:102EB0001FD8A6EB0906CCF80060C1F81CC0BEE71D
:102EC000A9EB0A09D6F81CA0B446BAF1000F0AD043
:102ED0005646D6F800A0CA45F2D3AAEB090AC6F8AE
:102EE00000A0B2466646C1F80090C1F81CA0F1618E
:102EF000D9E66646EDE7FFF76DFE2CE7F8D0002037
:102F0000F9D00020FCD00020F0D00020D8D1002043
:102F10001CCF0020D8D0002000100140D9D00020C4
:102F200000E100E0FEFF7F0074450FD1D0F81CB037
:102F3000C3F800B0BBF1000F08D10A4D0120A86012
:102F400001984FF0010CC0F800B0E1462068E46938
:102F5000CEF81C40002C3FF48BAE2568284420603E
:102F600086E600BF0010014037B5074B054693E8E1
:102F700003006C46002384E803001A4621462846D5
:102F8000FFF7FEFC03B030BD5C000600FDF7B6BAEB
:102F900010B54FF6FF7304469C42084609D1FEF770
:102FA00011FFB0F5807F044601D14FF6FF74204633
:102FB00010BDFF2CF9D82146FEF7E0FE0028F6D11F
:102FC000F3E710B5044601F0EFFC2046BDE81040E1
:102FD00000F02EBF1FB5037893B90279072A0FD1ED
:102FE000448803932046CDE901338DF80420FCF793
:102FF000F7FBADF8060001A8ADF80840FFF7E1FFC8
:1030000004B010BD1FB50023CDE901330393ADF823
:103010000600022301A88DF804308DF80810FFF790
:10302000D0FF05B05DF804FB86DF704738B5048833
:103030004CB9821C00F10A0512F8013B1BB99542FC
:10304000FAD100200AE00B88A342FAD1082202310B
:1030500002303CF091FFB0FA80F0400938BD08B56D
:1030600070B171B103780A78534013F0FE0F08D1A4
:103070000622013101303CF07FFFB0FA80F04009B8
:1030800008BD0020FCE710B5044600F0BDFF204657
:10309000BDE8104000F04ABF43DF70476FDF704764
:1030A000024B0022C3E90022704700BF50CC002031
:1030B000F0B5FF2887B004460E4615461F4629D8AE
:1030C0000846FCF7CBFB28B303AA2046FFF7E4F839
:1030D00018B10524204607B0F0BD01A903A8FFF7E9
:1030E00011F804460028F4D1019BAE705A882A805A
:1030F0005FB13B6892009A420AD3029968683CF03B
:1031000049FF03A8FEF7E2FFE4E7029B6B60F8E7E4
:103110000424DFE70724DDE72DE9F041CEB020AE3F
:10312000502380460CADB822002130460193039510
:10313000FCF7F8F90DF1970305930DF1AE03069333
:103140000DF1C503079337AB08930DF1F303099312
:103150000DF585730A931C4F04960DF221130B9302
:103160000024444507D1E2B2002104A8FFF796FFEE
:103170004EB0BDE8F081502200212846FCF7D2F97C
:1031800001AB02AA072137F8020BFFF791FF20F0ED
:1031900002000528ECD06B7C032B12D817230DF10D
:1031A000310203FB04630DF1450152F8040B43F8AF
:1031B000040B8A42F9D11188198092789A700134EF
:1031C000CFE743F20220D3E702D100202DE9F041FE
:1031D00010220546A6B000212D48FCF7A3F935B909
:1031E00029462846FCF710FB26B0BDE8F0816A00AE
:1031F00028492748DFF89C8004AE3CF0CBFE3822FB
:1032000000213046FCF78EF900245023CDE901342B
:1032100012AF0397502200213846FCF783F901AB27
:1032200002AA072138F8020BFFF742FF20F0020044
:103230000528D9D09DF85930032B26D8C4EBC402F9
:10324000B318DDF85910B1500134BDF85D209A80F3
:10325000A5429DF85F209A71DCD10DF117031393FD
:103260000DF11E0314930DF1250315930BAB16936B
:103270000DF1330317930DF13A0318930DF1410348
:1032800012961993E9B23846ACE743F20220ABE755
:1032900012D1002002D100202DE9F043037889B03B
:1032A0000546002B3FD1017907293CD104AA40886B
:1032B000FFF7FEFEB8BBFFF7F3FE02A90DF1060013
:1032C000FEF7C0FF78B36E88BDF80670BE42F4D03A
:1032D000059C631C1846113413F8012B12B9A34244
:1032E000FAD1EAE7DDF80C80102208F101013CF088
:1032F00043FE08F1110181462046FFF7B0FEB9F107
:10330000000F01D00028D8D03046FCF769FA00231E
:10331000ADF81A0006A88DF81830ADF81C60ADF8AD
:103320001E70FFF7B0FE09B0BDE8F083CA1F012A86
:1033300073B5064654D80025CDE900558DF8021026
:10334000FCF7B6FA044600284CD0437CDB074BD48C
:10335000007CFCF76BFA10B9032002B070BDE36883
:10336000019003EB83031B019BB29B086846ADF8F9
:103370000030FCF77BFA626804F1080369463046C6
:10338000FFF7FEFA637C03F00603062B01BF174A22
:10339000136803F1FF33136030B9637C23F0070334
:1033A00043F001036374D8E711280BD10F4A136867
:1033B00001331360637C23F0060343F0040363745A
:1033C0000020CAE7862809D1084A13680133136030
:1033D000637C23F0060343F00203E3E70728BBD135
:1033E0000720BAE70520B8E72846B6E7F0CD002069
:1033F0002DE9FF410546102200216846FCF792F8AE
:1034000068882979ADF802008DF80410FCF750FAAD
:103410002B78454E092B5ED8DFE803F00505684D93
:103420004D6C7173757D00283FD0437CDC073CD523
:10343000FEF7FEFD2B78581E4342434100246846A8
:103440008DF800408DF80830FCF724FA33684BB350
:10345000364E002537464FF0140808FB05735B7C99
:103460005A0703D49B0759D5002C57D0B178308820
:10347000FFF75CFF002851D014235D437B19862899
:103480009B788DF804307A5B16BF029008230923DD
:103490006846ADF802200CBF8DF800308DF8003082
:1034A000FCF7F8F904B0BDE8F08101238DF8003095
:1034B000AB68029316E080B18268AB689A420CD187
:1034C000437CD90709D5326823F00503013243F064
:1034D0000403326043740024B8E702238DF80030FF
:1034E000EB6803936846FCF7D5F9F4E703238DF8FE
:1034F0000030F7E704238DF80030EB68D9E70523A7
:10350000F5E70623F7E7072368468DF80030012426
:10351000FCF7C0F99AE7EB680293DCE70135082D68
:1035200006F1140699D1BDE7F0CD002034D100207A
:1035300070B500238CB02D492C4E4FF6FF70CDE9AD
:103540000033FCF727FA4FF6FF750446AC420BD068
:10355000A4F58043ADF8143002AA6B46002105A8FB
:10356000FEF736FE0A2822D0214B1A781846E2B917
:103570004FF6FF718C4218D01E4E367801251D7013
:10358000B607A4F580439BB21DD58B422CD00521F4
:103590008DF8141005A811468DF81850ADF81A30A2
:1035A000FEF7CEFD60B1FFF757F90CB070BD2046B5
:1035B000FEF778FD20463146FCF7ECF90446C5E7F6
:1035C0000D4B1D70F1E702230022092102708DF8D6
:1035D000141005A8FF21ADF816408DF81810CDE99C
:1035E0000723FFF705FFE0E70423EDE718D00020ED
:1035F000B1CF00205DCC0020B2CF0020F0B54268F2
:1036000005783D4C85B0B2FA82F149090391691EF3
:103610000346042924D8DFE801F0030330496A0097
:103620009989DE8901F5804189B243F6FE77B94276
:1036300004D906F5804080B2B84211D8012DADF80A
:1036400002108DF8046013D1002A14BF0321002159
:103650008DF8001003929B6802936846FFF7C8FE3E
:1036600023781BB100232370FFF762FF05B0F0BD84
:10367000002A14BF04210121EAE79989DD8901F5B7
:10368000804189B243F6FE76B14204D905F5804007
:1036900080B2B042E4D8002A0CBF02220522ADF865
:1036A00002108DF804508DF80020D4E7988900F5B9
:1036B000804080B243F6FE718842D1D8DB89002B6E
:1036C000CED1FF23ADF802008DF804305AB906239D
:1036D0008DF80030FEF7E6FC084A002323701370D3
:1036E000FFF726FFB9E707238DF80030F4E708233A
:1036F0008DF80030B1E700BFB2CF0020B1CF00207D
:10370000F8B50D490D4DFCF745F94FF6FF76044627
:10371000A5F12007B44201D12046F8BDFF2CFBD80B
:1037200021462846FCF772F80028F5D02046394695
:10373000FCF730F90446EDE7F8CF002018D0002060
:1037400070B504468AB0142200216846FBF7EAFEF1
:103750006588ADF804502846FCF742F82378ADF8A8
:103760000200092B15D8DFE803F005163048525E39
:103770008614A1A507238DF8003023798DF8083031
:103780009DF80A3043F001038DF80A306846FCF7D3
:103790001BF90AB070BD07238DF8003023798DF82E
:1037A00008309DF80A30444AA168039143F00103B0
:1037B0008DF80A301368002BE8D09942E6D1002337
:1037C00013603E4A03931580E0E708238DF800302C
:1037D00023798DF80830E3680493374BA1681A68A1
:1037E0000391002AD2D09142D0D1354900221A60EB
:1037F0000B680392013B0B60C8E707238DF800308C
:1038000023798DF8083001238DF80930BEE70823AD
:103810008DF8003023798DF8083001238DF80930B8
:10382000A3680493B2E7274D09238DF800302B7865
:10383000002BABD04FF6FF70FFF762FF4FF6FF7320
:1038400098420646A2D12049FCF7A4F8B0420446AB
:103850009CD1142200210DEB02002970FBF762FEBF
:103860000B238DF81430ADF81840ADF8164005A8BC
:10387000FCF7AAF88AE70A238DF80030114BA468F8
:103880001A780294002A81D0142200210DEB020044
:103890001970FBF747FE0C238DF814304FF6FF73B9
:1038A000ADF81830ADF816300794E0E705238DF831
:1038B00000306BE70623FAE7F4CF0020E4CD0020C8
:1038C00034CC00203ACC002018D0002073B5104B27
:1038D000104C93E803006D46002385E803001A4668
:1038E00029462088FFF74CF84FF6FF762388B3422D
:1038F00001D0112801D102B070BD1846FFF700FFBA
:1039000000231A4629462080FFF73AF8EEE700BF69
:103910006400060038CC00201FB50378012B044654
:1039200015D10179012912D1002302AA4088FFF79D
:10393000BFFB60B902238DF800306388ADF8023018
:10394000039B68461B788DF8043000F0EFFC054BB4
:103950001A884FF6FF739A4201D0FFF7B7FF04B001
:1039600010BD00BF38CC00202DE9F047474B1B7835
:103970008AB00546002B00F08780454B454F93E801
:1039800003003C7803AE86E80300BCB94FF6FF7035
:10399000FFF7B6FE0123ADF8143001AB0693042304
:1039A000029305AA02AB062180460194ADF81640A9
:1039B000FFF77EFB07284AD101233B70364B1C687A
:1039C0009846002C5AD1354A354F12883B68AA4296
:1039D00041D1002B3FD0142221460DEB0200FBF712
:1039E000A1FD072328468DF81430FBF7F9FE0623C6
:1039F000ADF8160005A8ADF818508DF81C30FBF78F
:103A0000E3FF20460AB0BDE8F087CDF804A0019B93
:103A10004046A34224BFC1461C46FFF771FEBDF8D5
:103A200014309B00029305AA02AB06218046FFF7E3
:103A30003FFB0028EBD00528E7D04FF6FF739845F1
:103A40001CD1164BA3F80090154B1C60B4E74FF641
:103A5000FF79A246EDE701333B6000220E4B314671
:103A60002846FEF78DFF0028CCD00023C8F8003090
:103A70003B68112803F1FF333B6001D11120C1E7FE
:103A8000862818BF0320BDE70820BBE7ECCD002047
:103A90006C000600F3CF0020F4CF0020E4CD00201E
:103AA00034CC002063DF7047A6DF7047A2DF704789
:103AB0002DE9F04391B0984611238DF80430137826
:103AC0008DF805300024164601254FF0000365F3FC
:103AD0004203074689461C22214609A88DF8063074
:103AE000FBF720FDB3788DF80930C3F30302A2423F
:103AF00014BF1A2212228DF8242001AA0E9203ABC1
:103B000072788DF808200493224602AB65F34202D6
:103B1000059308238DF80A20CDE9064404AAADF8E0
:103B20001C3009A9434638888DF80E50ADF80C902A
:103B30000894FFF7BBFF11B0BDE8F083A0DF70472A
:103B4000044A0123116883400B401ABF1218507EAB
:103B500018467047F4C9002070B4094D1346012679
:103B60002A6806FA01F4144207D001F1190402464A
:103B70003146281970BCFDF757BE70BC704700BFB6
:103B8000F4C900201FB50023CDE9013303938DF85C
:103B90000A201A46074BADF8081006241978ADF82C
:103BA00006008DF80440FFF7D7FF01A8FFF709FAD8
:103BB00004B010BDB32C002010B4084A01231468CF
:103BC0008B40234006D00A445DF8044B0146507EEA
:103BD000FDF79ABD18465DF8044B7047F4C9002004
:103BE00010B50A4B19780446FFF7E6FF58B1084BA9
:103BF00000205A88A24201D1C0B210BD013008286D
:103C000003F10C03F5D1FF20F7E700BFC8CB00207C
:103C1000CACB00202DE9F8430546FBF7E1FD234B15
:103C2000074600221420984600FB02F1CC5AAC4211
:103C30002AD10B44002634464FF014095BB1997821
:103C40002846FEF711FA10B1052818BF03240136E3
:103C50003246072A1DD9A4B9FF2D24D81449284675
:103C60004FF6FF75FFF794F9FFF762FCAF4208D0FB
:103C70003846FFF7B5FFFF2803D00C2343430D4A16
:103C8000D5522046BDE8F8830132082ACCD1002362
:103C9000D0E709FB02F338F80310A94201D14344ED
:103CA000CCE70132D5E70724EBE700BF34D1002091
:103CB00018D00020CACB00202DE9F0411F46154B3B
:103CC0009DF818400E46904619780546FFF744FFC8
:103CD000B8F1000F17D0104B3A4619782846FFF775
:103CE0003BFF0E4B224619782846FFF735FF44B1BB
:103CF0002846FFF775FFFF2803D00C234343084AEB
:103D0000D652BDE8F081002CFBD03046BDE8F04132
:103D1000FFF780BFB32C0020B52C0020B42C00206E
:103D2000CACB002008B5FFF75BFFFF281DBF0C239F
:103D30004343034A4FF6FF7018BFD05A08BD00BF77
:103D4000CACB00202DE9F04385B00546FFF7EAFF16
:103D50004FF6FF739842074641D001224FF0030906
:103D600001AB0821384602F10108FEF791F81FFA6D
:103D700088F8064648BB02990A46032342F8049B8A
:103D800006312846FBF720FD044660B90821384675
:103D9000FFF7CCFA0446112C3FD01AD80CB30C2CE8
:103DA0002FD107231EE00C280DD0052800D1344662
:103DB00008213846FEF758F9002818BF0324424668
:103DC000002ECDD1E7E70126F2E70728E9D0044627
:103DD000E1E7862C13D043F202039C4211D100226A
:103DE0001CE0012328468DF80430ADF80850FFF799
:103DF00099FFADF8060001A8FFF7C8F8EFE7082320
:103E0000F0E7092328468DF80430FFF78BFFADF863
:103E10000850ADF806000394EDE70122034B284655
:103E20001978FFF799FE05B0BDE8F0835ACC002061
:103E30000378072B02D14088FFF784BF704700004A
:103E40002DE9F0434FF6FF75A84285B0044668D0CF
:103E5000FFF768FFA84227D100260327B0464FF09E
:103E600001093B46324641462046FBF7AFFC042899
:103E700005464DD0082847D00B282DD117F0020356
:103E80001FD1B8F1000F20D11EBB032320468DF8AF
:103E90000430FFF747FFADF80840ADF8060001A871
:103EA000FFF774F8002237E0002301AA0821FFF78A
:103EB000FFF80028D0D1029B03F106089E881F68F6
:103EC000CDE701274FF00009CBE703271E469846B0
:103ED000F8E703274646F5E7B9F1000FD5D01128DA
:103EE00019D043F202039842DCD008B90223CDE78F
:103EF000092320468DF80430FFF714FFADF8084081
:103F0000ADF806000395CAE7B9F1000FEED1BCE7A2
:103F1000B9F1000FB9D00122034B20461978FFF701
:103F20001BFE05B0BDE8F08359CC002037B50578FD
:103F3000012D044614D14088FFF782FF6088FFF707
:103F4000F1FE00236A462946FFF7B2F840B9019B0B
:103F50001B782BB1034B608819782A46FFF7FCFDCC
:103F600003B030BD5BCC0020F0B587B004460E46F0
:103F70001746FFF7D7FE4FF6FF739842054624D049
:103F80001E4B20461978FFF717FE80B30023CDE9BA
:103F90000033029304238DF80030194BADF8024032
:103FA0001978ADF8046020468DF80670FFF704FE1E
:103FB00068B12846FFF72EFE124B204600221978E2
:103FC000FFF7CAFD6846FEF7FCFF07B0F0BD07210A
:103FD0002846FEF749F80528EED10923049003A8E6
:103FE0008DF80C30ADF80E40FEF7EBFFE4E73A46F3
:103FF00031462046FFF7C6FDE7E700BFB52C00209D
:10400000B42C0020B32C002010B5027886B00446F2
:104010001AB1012A09D006B010BD0E4B1B78002B37
:10402000F9D0C088FFF7F6FDF5E70B4B408819780B
:10403000FFF792FD1422002101A8FBF773FA6088B4
:10404000ADF80600FFF76EFEADF8080001A8FBF71B
:10405000BBFCE0E7ECCD002030CA002070B5044680
:1040600086B01422002101A8FBF75CFA237860884F
:10407000ADF80600013B0B2B00F29080DFE803F067
:104080002106233A4E585C68747A7C8C2679444B1E
:10409000321C19784FF0010518BF01228DF8045029
:1040A000FFF75AFD731B5A425A413E4B60881978FC
:1040B000FFF752FD6088FFF735FEADF80800002DD0
:1040C00042D106B070BD02238DF804302379002B55
:1040D00014BF012302238DF80C30314B01221978D3
:1040E000FFF73AFD2F4B227919786088FFF734FDEE
:1040F0000125DFE703238DF804302A4B1978FFF7F9
:104100005BFD002814BF012302238DF80C30A37936
:104110008DF81030A388ADF80E30E9E7204B197800
:10412000FFF74AFD0028CCD102238DF80430DFE7E9
:1041300003238DF80430EAE70723A2888DF80430C2
:10414000ADF808208DF80C3001A8FBF73DFCB8E76E
:1041500008238DF80430A388ADF8083007238DF8C4
:104160000C30A3680593EFE706238DF804306368ED
:104170000393BDE70523D8E703238DF80430094BEB
:104180001978FFF719FD002814BF012302238DF8C9
:104190000C3041F20113BEE70423C6E7002589E78E
:1041A000B0CF002030CA00201FB50D294FF000030A
:1041B00001930393ADF80600029108D10B2301A8E7
:1041C0008DF80430FFF74AFF05B05DF804FB86293F
:1041D0000CBF0A230923F2E730B508490A68002317
:1041E000012505FA03F42242D8B202D122430A6023
:1041F00030BD0133182BF4D11846F9E7F4C900207B
:1042000010B50378182B044602D1FFF7E5FF2070A4
:1042100010BD000010B5024B197DFDF723FB10BD4A
:10422000F4C900202DE9F04F3D4D89B02878FFF703
:1042300087FC60B103A8FFF7EDFFDFF8E8A0DFF827
:10424000E8B00DF110090027039B9F4202D309B08B
:10425000BDE8F08F39F8024B29782046FFF7ACFC17
:10426000064678B39AF800102046FFF7A5FC804672
:1042700040BBBBF800304FF6FF7219462046FBF7F3
:10428000A7FA43F20302904229D10133ABF8003080
:10429000EFE7052320468DF80030FFF743FDADF82A
:1042A00002006846ADF80440FEF770FEB0463246A4
:1042B00029782046FFF750FC42469AF80010204625
:1042C000FFF74AFC0137BFE72046FFF72BFDFEF75B
:1042D0004BFE0026EBE72046FFF7B2FDE7E7082894
:1042E000F2D012D80028D4D00628EDD009230290AD
:1042F00020468DF80030ADF80440FFF713FDADF80F
:1043000002006846FEF742FED1E743F202039842FC
:10431000CDD043F201439842DDD01128E6D1C6E763
:104320005BCC00205CCC0020ECD100201FB5044603
:1043300040882378ADF80600012B10D05AB21AB18C
:10434000022B15D004B010BD01A88DF80420FEF793
:104350001DFE6088FBF744FAFFF772FDF2E78DF867
:10436000043001A8A388ADF80830FEF70FFEE9E796
:104370002379002BE6D0FBF733FA4FF6FF73984210
:10438000E0D0044B01221978FFF7E6FBFFF74AFF64
:10439000D8E700BF5BCC002038B5074C0146207D34
:1043A000FDF7B2F930B1A07DFDF7AEF9002814BFDA
:1043B0000220012038BD00BFF4C900202DE9F047DC
:1043C0008CB0894616468046FFF7E6FF20228246DB
:1043D000002104A8FBF7A6F8BAF1000F46D0B9F106
:1043E000000F17D099F8005015F001054FF6FF7433
:1043F00015D04046FFF796FCA042074639D1404809
:10440000FDF7E0FCB0F5807F01D0B84275D1002502
:10441000032470E04D4685264FF6FF775FE02E4679
:1044200027465CE04A4631464046FBF7D5F904464C
:10443000B9F1000F5DD000285DD199F8003013F07C
:10444000010F14BF012102214046FEF7DBFDB6F14A
:10445000850218BF012200240095012339464046F9
:10446000FFF72AFC20460CB0BDE8F08743F20204B7
:10447000F8E7002502AB012207213846FDF708FDC9
:104480000446002837D1214650220398FBF74AF80A
:10449000039B83F800A0039C079604F13403049364
:1044A00004F118030893631C09934046154B0B93C2
:1044B000FFF796FBFF280CD0134A0C2101FB0020CC
:1044C00050F8042FC4F811208288A4F815208279AE
:1044D000E2753846FBF712FA044660B90646BAF1AF
:1044E000020F04AB9ED1002231464046FBF774F91F
:1044F0000446002CABD00022AEE707460125B9E701
:10450000F8CF0020B3CF0020CACB0020F0B585B093
:104510000446FFF741FF324F012806463D7831D16E
:104520002046FFF7FFFB4FF6FF7398422AD0204644
:1045300032462946FFF710FB0023CDE901330393F0
:1045400001A80C238DF80430ADF80640FFF786FD76
:10455000244B1B78E3B139782046FFF72DFBB8B91F
:10456000214B22491A682046FFF728FF8628054676
:1045700032D011280FD070B129462046FFF714FE23
:1045800005B0F0BD002229462046FFF7E5FADFE737
:1045900000221146E7E7A5F111035E425E410022C9
:1045A000134B20461978FFF7D7FA124B3246197889
:1045B0002046FFF7D1FA104B002219782046FFF76A
:1045C000CBFA0E4B002219782046FFF7C5FA002DD2
:1045D000D6D0112DD4D0CFE700260122E0E700BFCE
:1045E000B22C0020DFD000209CCF0020DAD00020A9
:1045F000B12C0020B02C0020AF2C0020AE2C0020CD
:10460000F0B587B0074601A8FFF704FE02AD00240D
:10461000019B9C4201D307B0F0BD35F8026B3946CF
:104620003046FFF7C9FA10B13046FFF76FFF01348B
:10463000EEE700002DE9F04F054687B09046994619
:104640000F4639B9A14B1B78F3B90524204607B0B2
:10465000BDE8F08FFFF7A0FE0138C0B2012800F2DC
:104660002D8100212846FBF7B9F80446862C00F07E
:10467000B080112C00F09980002C00F09680B9F1E8
:10468000000F00F0BF80B9E0FFF786FE012800F0C0
:104690009E80022840F012818D490B78284613F045
:1046A00001048B4614BF4FF0010A4FF0020AFFF7D6
:1046B00039FB4FF6FF739842064659463AD03B46BF
:1046C00002AA0721FEF7F4FC0446F0B9039B93F815
:1046D0004420D10740F1C780B8F1000F40F0D680E8
:1046E00003F1340202F112012846FBF773F84FF090
:1046F000000A044600230093BAEB030318BF01230A
:10470000B4FA84F25209314645E00528F2D1BDE001
:1047100004AB012207213046FDF7BAFB044600280E
:1047200040F0C1803046FBF7E9F80446002800F06D
:10473000B280B8E0002C41D06648FDF743FBB0F5ED
:10474000807F834637D0B04236D004AB01220721A8
:10475000FDF79EFB044650B95846FBF7CFF80446D8
:1047600028B95B492846FBF739F8044638B10721D8
:104770005846FDF779FC10B1052818BF03244FF601
:10478000FF73BBEB030318BF0123B4FA84F2009359
:104790005209012359462846FFF78EFA002C7FF470
:1047A00065AF51462846FEF72DFCA4F111035E4289
:1047B0005E4100220FE0B3460324E0E72846FBF702
:1047C0000DF8009704460123B0FA80F29AE74049B9
:1047D00048E700260122404B28461978FFF7BCF92C
:1047E0003E4B324619782846FFF7B6F9B9F1000F6B
:1047F00008D0002C3FF42AAF112C17D021462846B0
:10480000FFF7D2FC0D2C3FF421AF06D8002C3FF46B
:104810001DAF082C18BF032418E7862C14D043F2D0
:1048200002039C423FF412AF112C1AD12C4B3A4692
:1048300019782846FFF790F92A4B424619782846FE
:10484000FFF78AF9002401E7254B3A4619782846F4
:10485000FFF782F9234B424619782846FFF77CF987
:10486000F4E60324F2E6B8F1000F0FD1598D03F1FD
:10487000180200297FF436AF03F12C01343311F80C
:10488000010B00287FF42EAF8B42F8D19BF800304B
:10489000DA073FF53DAF0E492846FAF79FFF044679
:1048A00000283FF427AF07213046FDF7DDFB002845
:1048B0003FF420AF052818BF03241BE743F202048E
:1048C000B9F1000F3FF4C2AE98E700BFDFD000207F
:1048D000DAD00020F8CF0020AF2C0020AE2C002032
:1048E000AD2C0020AC2C00202DE9F04786B0074607
:1048F000FFF726F958B101A8FFF78CFCDFF84880D4
:10490000DFF8489002AE0025019B9D4202D306B01D
:10491000BDE8F08736F8024B39462046FFF74CF9E0
:1049200080B198F800102046FFF746F999F800107A
:1049300082462046FFF740F90123014652462046B1
:10494000FFF778FE0135DFE7AC2C0020AD2C00200E
:1049500010B50378062B0ED9072B1BD10E4B1C78F4
:104960002046FFF7EDF810B12046FFF749FE0B4B4C
:104970001878FFF7B9FF0A4B1C782046FFF7E0F8DC
:1049800010B12046FFF73CFE064BBDE810401878FA
:10499000FFF7AABF10BD00BFB12C0020AF2C002034
:1049A000B02C0020AE2C00201FB503780446092B44
:1049B00009D8DFE803F0050A20202020202020204D
:1049C0004088FFF7A3FD04B010BD144B197819B34C
:1049D000134B00791B7803F00102904206D86179ED
:1049E000C3F34003994294BF002101210123002217
:1049F0006088FFF71FFE23788DF80430043434F804
:104A0000023CADF8063094E8030004AB03E9030070
:104A100001A8FFF723FBD6E70121E7E7DFD000205D
:104A2000DAD0002037B5174B174A5B881188174C2E
:104A3000174D994208D852889A4205D36369FBB949
:104A400000232B7003B030BD2B783BB16369002B82
:104A5000F6D000228DF8042001A80FE00D490E4881
:104A60000978D4E9012300290CBF11461946FDF746
:104A700041F90028E4D0A369002BE1D09847DFE793
:104A80000122E7E72ACC002038D000208CCB002080
:104A900020CB002000D10020A8CB00207BDF704776
:104AA0007ADF704776DF704775DF704737B5164B92
:104AB00018884FF6FF73984210D0144A144D13789B
:104AC000297B0133DBB2994213702C4608D311497C
:104AD000FFF7EAFF10B1AB6903B1984703B030BDEF
:104AE000002313702B7C33B13B21FFF7DBFF10B1A8
:104AF000AB6903B198476369002BEFD000228DF8B2
:104B0000042001A8E9E700BF88CB002000D10020E5
:104B10008CCB002038D0002065DF70472DE9F74F9F
:104B20000C9CBDF834B02788002580468A46914603
:104B30002E46B8F80020B2420BDC35B12288013A8B
:104B4000D21B92B2FF2A39D8DA55002003B0BDE853
:104B5000F08FD8F8042052F82600019000220DF1C1
:104B6000030101A8FFF7D8FF0028EFD19DF803202B
:104B70004A4521D12288002D14BF0020022002EBDB
:104B800009010144594519DC3DB9013292B2228034
:104B900003F802A022880132228022880DF103014D
:104BA0001A4401A8FFF7B8FF0028CFD121889DF84B
:104BB00003200A44228001250136BAE70C20C5E70C
:104BC0002DE9F341089CBDF824501746CDE9004576
:104BD00002220646FFF7A2FF48B9102239463046A6
:104BE000CDE9084502B0BDE8F041FFF797BF02B03C
:104BF000BDE8F0812DE9FF470023138090F82D30A8
:104C000006460D4614463BB302A8FAF7F5FE002807
:104C100040F0FB8013880822CA54238801339BB2DA
:104C20001B222380CA54238801339BB2CA18DDF8A3
:104C300009102380E950BDF80D30938023889DF83A
:104C4000082006339BB212F0FE0218BF0122238017
:104C5000EA54238801332380B378FBB123880433DB
:104C60001F2B21D802A8FAF7C5FE002840F0CD80FE
:104C700023880322EA54238801339BB2192223801C
:104C8000EA542388BDF8082001339BB2E918238039
:104C9000EA54120A4A70238802332380F278AAB1B8
:104CA0002388D91C1F2901D90C20AEE00221E95428
:104CB000238801339BB201212380E95423880B44CC
:104CC0009BB22380EA5423880B4423807268AAB1E4
:104CD0002388D91C1F29E7D8022192F90020E95422
:104CE000238801339BB20A212380E95423880133AE
:104CF0009BB22380EA542388013323803389002B1D
:104D000076D1338A5BB11F23CDE9004307222B46BE
:104D1000032106F11000FFF753FF002875D1338BF4
:104D20005BB11F23CDE9004315222B46142106F168
:104D30001800FFF745FF002867D1326A002A67D1C3
:104D4000776A4FB3BB882188981C8A1C02441F2AAB
:104D5000AAD8FE28A8D803336B54238801339BB20A
:104D6000FF222380EA54238801339BB223803A88B0
:104D7000EA54E918120A4A702088023080B2208072
:104D8000BA884AB1B96800294AD028443BF002F9F0
:104D90002388BA881344238096F82C30002B79D1CD
:104DA000307890B33388012B3AD023889F1C1F2F73
:104DB0003FF67AAF012805D1727802321A441F2AD1
:104DC0003FF672AFC3F11D039BB202A9E819ADF81B
:104DD0000830FAF70DFEC0B93278022A40F0988008
:104DE000BDF808209A4240F2AE80ADF8083098E055
:104DF0001F23CDE9004306222B46022106F10800BD
:104E0000FFF7DEFE00283FF47CAF04B0BDE8F0877A
:104E10002788BB1D1F2B3FF647AF1188052901D8F6
:104E20000720F2E76FF4486C01EB0C039BB24FF2E2
:104E30007D3C6345F4D95388052BF1D96FF4486064
:104E4000181880B26045EBD94FF6FF70814203D04D
:104E5000834201D09942E3D80523EB5523880133DF
:104E60009BB212212380E954238801339BB2238013
:104E70001188E954E818090A4170238802339BB26B
:104E800023805288EA54E918120A4A7023880233B0
:104E9000238055E7B36A002BC2D04FF000084FF0D3
:104EA0000C094FF0160A96F82C305FFA88F29342FC
:104EB0007FF676AFB16A09FB02F28F18BB88981CA7
:104EC000FE283FF6F1AE208803332B5423880133AC
:104ED0009BB2238005F803A0238801339BB2238073
:104EE0008A5AEA54E918120A4A702088023080B2BD
:104EF0002080BA884AB1B968002991D028443BF093
:104F000049F82388BA881344238008F10108CAE7C6
:104F1000012A7FF46AAF72789342FFF466AFADF86E
:104F200008200821BDF80830FE2B3FF6BDAE2288D0
:104F30000133AB542288013292B22280A9542288D4
:104F40001344238061E70921ECE7000007B5144B07
:104F50001A686AB1002018601B6800934FF0804205
:104F6000009B0123C2F808330E4A5370FAF746FD3E
:104F70000D4B1A688AB100221A601B680193019BCD
:104F80004FF080430222C3F80823064B012098709B
:104F900003B05DF804EBFAF731BD03B05DF804FB34
:104FA000000100406CCB00200401004013B5104B01
:104FB000104C114800221A601B6801932146019B86
:104FC000FAF732FD88B9A27E0C48FF2A1FBF0123E1
:104FD00093404FF0A042C2F8083500236376237156
:104FE000236802B0BDE81040184702B010BD00BFF2
:104FF00008310040E0CA002000300040E4CA002030
:1050000070B52D4C86B094F82130019394F820307F
:105010000093E36904F1260204F123014FF04020DC
:10502000FAF733FD2346E0B994F82360A56906BB7F
:10503000217B8A1E012A1CD8E0692269904218D17E
:105040006269E37BE261C5F34015032984F82030EF
:1050500084F8215007D100954FF040212046FAF7FF
:10506000EBFD06B070BD4FF040212046FAF787FDFA
:10507000F7E7124A07CA06AC04E90700C6B14FF0C9
:105080004021D1F8C424C1F8C42490070CD50122D2
:105090008DF80820002283F824206A07E1D4D3E9A0
:1050A000002102A89047DCE75107F3D50222EFE781
:1050B0008DF80860EEE700BFB8CA0020C4CA00201F
:1050C000F7B515464FF0FF32C1F8082390F82420B9
:1050D00004460F4602F0FF0E2AB18368C1F804337C
:1050E000112003B0F0BD012680F82460836100F137
:1050F0000C0C95E807008CE80700AA7884F82020BB
:105100006A68E2616A78C7F888252A78B24212D0C4
:1051100012B91E1C18BF012684F821600096AB78D6
:105120006A6839462046FAF787FD2368002BD8D1F4
:1051300084F82430D5E784F821E0AB786A683946F2
:105140002046FAF71CFDF0E70023435082B0435895
:105150000193019B02B07047064A08B54FF4927163
:105160001046FFF7F1FF4FF48471FFF7EDFF0123C5
:10517000136008BD0020004010B5CB7D0A464FF4F7
:10518000847123B9FFF7E0FFD0F8183510BDFFF7A1
:10519000DBFF537ED168D0F81805C854537E013325
:1051A000DBB25376F2E70000F8B52C4C626822B10E
:1051B0002B4B4FF40171C3F80813E37D4BB1237EF1
:1051C0007BB322B1264B4FF40172C3F804231120A4
:1051D00026E00122E275E0606376A27E237612B9B2
:1051E0000BB9FFF7B9FF636873BB4FF4A2711C489A
:1051F0001B4E1A4FFFF7A8FFD6F82431D6F8082126
:10520000D6F8445182B90DB9002BF5D00022E275D1
:1052100003BB0DBBA17E124B012299B11A60002085
:10522000F8BD20610123D8E7002BEFD1002DEDD18F
:1052300039463046FFF7A0FF637EE27D9A42DBD815
:105240002B46E3E75A60EAE7054B4FF40172C3F8D7
:105250000423E4E70320E3E70F20E1E79CCA0020F2
:10526000002000400A4610B54FF48E71FFF76CFF26
:10527000938A91689BB2C95C938A01339BB29382F3
:10528000C0F81C1510BD000030B54A4AD2F80433EE
:1052900013F4007F85B015464AD0D2F82431002B94
:1052A00046D04FF492711046FFF74EFF4FF4017352
:1052B000C2F80833404B997E09B9012151603D493C
:1052C00002228DF80020D1F88024C1F880240392B6
:1052D000DA7D8DF80820DA6801920022DA751A76F4
:1052E0006846D3E9001290473248D0F81C313BB1F0
:1052F000314A938A917D994247D91146FFF7B2FF0F
:105300002C4AD2F844318BB14FF4A2711046FFF70A
:105310001BFF294B997E09B101211160DA7D2AB169
:105320000022DA75587ED968FAF778F905B030BDF1
:10533000D5F804335B07D7D5D5F80831002BD3D087
:105340001D4C1C482146FFF717FF637EE27D9A4201
:105350002346C9D1227E52B12369E168E36000236C
:10536000607EE27523766376FAF758F9BCE7A27E91
:105370000AB901226A600F4A4FF40171C2F808139A
:105380000022DA75587ED968EEE74FF48E71FFF788
:10539000DBFE917D0029B3D000238DF808109168C1
:1053A0008DF80030019193756846D2E90013984753
:1053B000A6E700BF002000409CCA0020800000F14A
:1053C000A040D0F8003723F44033C0F80037D0F8BD
:1053D000003743EA0141C0F80017704700F18040F0
:1053E00000F5C040002382B0036003680193019B75
:1053F00002B070472DE9F04F85B00024594D01945B
:105400004FF48072012102F1804303F5C04390B252
:105410001B68012B06D1D5F804330B4202D0FFF7ED
:10542000DDFF0C430432B2F5907F4FEA4101EAD12F
:105430004D4B1B68012B0AD14FF4BE70FFF7CEFF16
:105440004FF0A04344F00044D3F81035019314F01A
:10545000FF0F1AD0454F01260025344210D0AB0073
:1054600003F1804303F5C043D3F81005D3F81015BA
:1054700057F8253023B1C1F30141C0F30420984708
:105480000135082D4FEA4606E7D1002C63DA4FF0CC
:10549000FF330022CDE90232344D354E0024A246BE
:1054A00001274FF0A04816F9012B531C46D0D2B269
:1054B00022F0C0094FEAD90104A8084402F007030A
:1054C00010F808CC07FA03F31CEA030F36D005EBFB
:1054D000090C92099CF930C055F82CB0BBF1000FB3
:1054E0000AD1032A2AD10DF10C0E1EF801C04CEA94
:1054F000030C0EF801C001E0032AF4D009F5E071B5
:1055000010F80C0C58F821101842C1F3014105D0D5
:10551000022913D1032A0BD1114604E003290DD12E
:10552000032A05D102214846FFF748FF0134E4B2BF
:10553000BBF1000F02D011464846D8470AF1010AD4
:10554000BAF1040FAFD134B14FF0A043019AD3F8B0
:105550001035934202D105B0BDE8F08F0193039B53
:1055600002939AE7006000407C61004044CA00203A
:1055700094CA00200028C3B2A8BF00F160424FEADD
:10558000501010B5BABF0D4A03F00F0402F5614286
:105590004FEA41114FEA8000C9B200F16040B4BF48
:1055A000115582F8001300F5614003F01F0201233A
:1055B0009340C0F88031036010BD00BF14ED00E0DF
:1055C0002DE9F8430446C279C17A0F2027F0F8F993
:1055D000237B644A0BB3537843F010035370256860
:1055E000EB175906604B41EAD51168064FF0FF32C0
:1055F0008B4208BF82420AD35C4A00233AF0FEFA8B
:1056000000F5006020F47F6626F00F064EB92946AB
:105610005748BDE8F8432FF06FBA537803F0EF0313
:10562000DCE7207929F0B2FA40B9607929F0AEFAC6
:1056300020B95048BDE8F8432FF05EBA4E4F3B7892
:105640001BB100233B70FAF7BDFF25794B4B0022BD
:1056500028461A7029F09AFA20B14FF44071284672
:105660001CF0D0FB6579284629F090FA20B14FF460
:10567000985128461CF0C6FB637A2579002B2846F2
:1056800014BF4FF00E094FF0000929F07FFA0028EF
:105690005AD03B4B05EB45051D4495F801806479D4
:1056A000204629F073FA002851D0354B04EB44040E
:1056B0001C446378334CE27E002A4BD15A1C0AD03A
:1056C0004FF0A04101229A40C1F8082503F5E0728D
:1056D000032041F82200B8F1FF3F2B4D1FBF4FF0D0
:1056E000A04108F5E072002041F82200C5F82465C9
:1056F000C5F86C950026C5F81485C5F80C35234B04
:10570000636028464FF48E712660FFF71DFD4FF44D
:10571000A271FFF719FD1E4BC5F80433022108469C
:10572000FFF728FF0423C5F80035B8F1FF3F4FF419
:105730008073E6822676638310D0FFF70DFD012388
:10574000A3761CF045F809E04FF0FF38A7E74FF0CB
:10575000FF33AFE708210F482FF0AEF901233B706C
:10576000BDE8F883ECC9002047E8010048E80100E3
:10577000D7010600EC010600F9D10020FAD1002083
:10578000800206009CCA0020002000400918040086
:10579000800002000202060010B50D4C002262607B
:1057A000A2602261E2600B4A106810F0010002D191
:1057B0000621FFF7DFFE084B1B7823B94FF080432B
:1057C0000122C3F8182501232370002010BD00BF5B
:1057D0006CCB002000E100E0E1D00020F8B50E46DF
:1057E000D11C48BF911D144641F387010546671E31
:1057F000FAF73BFB00214AB2A24201F1010100DBB2
:10580000F8BDBB1A23F00300B25C03F00303DB0016
:1058100002FA03F32A581A432A50ECE7F0B50025A0
:105820004F1E6CB28C4205F1010500DBF0BD3B1B45
:1058300023F0030603F003039659DB0026FA03F373
:105840000355EEE72DE9F041B3F9024014F11F05CD
:1058500048BF04F13E050F4603F1240645F3471502
:10586000904601462B4632463846FAF739FBB8B91E
:10587000B4EB451F16DA6211012304F01F0403FA8A
:1058800004F457F822301C4214BF012400242B4694
:10589000324639464046FAF723FB2046BDE8F08100
:1058A0000124F4E70446F2E710B500231A465CB27F
:1058B000A14203DCB2FA82F0400910BD50F8234047
:1058C00001332243F3E700002DE9F04F8A46234FCE
:1058D0008BB00646114650461446FAF7A6FA3B68C6
:1058E000FBB10425C0EB441014FB05FB00B205FB23
:1058F00004654FF0FF38043D28FA00F84FF04009E6
:105900003B6859463046984758B12B6803EA08036C
:105910002B6021463046FFF7C7FF20B1B9F10109DE
:10592000EED1002017E023463246514602A8FAF78E
:10593000A7FA2146019002A8FFF7B6FF019B0033AA
:1059400018BF01235B00002814BF5842C3F10100B7
:10595000C0B20128E2D10BB0BDE8F08FA42D002029
:105960002DE9F04FD1B0CDE905015B9D95F90040DF
:1059700048A8914622461F46FAF74BFAA300079320
:10598000069BA20013441946224638A80293FAF750
:1059900040FA95F90060002F00F08C8032463946BD
:1059A00028A8FAF736FA0DF5807A324630AF48A9C2
:1059B0005046FAF72EFA38A93846FAF72AFA2B4653
:1059C00028AA38A948A8FAF7E3F92B4628AA38A943
:1059D00048A8D5F8A460B0472B4628AA39465046B7
:1059E000FAF7D6F9BDF968310497023B1BB2002BD8
:1059F00067DCD9F80030009503F001084FEA481839
:105A000040AADB4302EB080A03F0010330AA9044EA
:105A10005B0140AA1A44039230AAD3184146039A64
:105A20000493504605F10409FAF751FC4B4640AA8D
:105A300048A908A80094FAF7BAFB08A908462B461B
:105A40004246FAF764F908A908462B46069AFAF77F
:105A50005EF9214608A8FFF727FF00285DD008A8B7
:105A6000FAF703FA08A92B46029A0846FAF74FF903
:105A700008A92B4652460846FAF749F9DDE9030121
:105A8000434652460095FAF7A4FB2B4608AA30A9D4
:105A900040A8FAF77DF9224640A90598FAF7B9F926
:105AA000059B079C234430A91846FAF7B2F951B078
:105AB000BDE8F08F314628A8FAF7D7F901232893DB
:105AC00071E71FFA83F85B1108F01F0259F82330C1
:105AD0000095012101FA02F21A42049B13BF20270C
:105AE0000027202600260AEB070B1F440AEB0603BB
:105AF0000393049B039A1E44334639465846FAF7EB
:105B0000E6FB08F1FF383B4600955A4631460398BC
:105B1000FAF75FFB0FFA88F369E710AF224608A98E
:105B200038460DF1600BFAF774F920AE4946584635
:105B3000FAF76FF930462146FAF797F9012328A8BA
:105B40002093FAF792F9224659463846FAF74CF96B
:105B500028B9224620A908A8FAF75BF982E73B6832
:105B6000DA0709D421463846FAF731F92246494680
:105B70003046FAF700FBE6E7189BDB0707D421461F
:105B80005846FAF724F92246494628A8F1E70028A2
:105B900023461CDD5A4639463846FAF771F9214644
:105BA0003846FAF714F9224628A93046FAF71CF9C4
:105BB000002805DA23464A4631463046FAF790F97E
:105BC000234628AA31463046FAF75AF9CEE73A4634
:105BD00059465846FAF754F921465846FAF7F7F865
:105BE0002246314628A8FAF7FFF8002805DA28A946
:105BF00023464A460846FAF773F928A9234632464F
:105C00000846FAF73DF9BEE72DE9F04793F9006041
:105C100092B0044689461046314615469846FFF72D
:105C200043FE002840F09180424649460AA8FAF710
:105C3000ABF843460AAA214602A8FAF768F80AA96F
:105C400008464246FAF7A0F843462A4649464846DF
:105C5000FAF75DF808F10407424629462846FAF7A4
:105C600093F83B462A46214620460096FAF716FB53
:105C70003B462A46294628460096FAF70FFB3B4644
:105C80002A46214628460096FAF791FA43462A46C4
:105C900021462046FAF73BF83B4622462146284655
:105CA0000096FAF7FBFA3B4600962A462146204624
:105CB000FAF7F4FA2368DB074AD533463A46214619
:105CC0002046FAF70DF9314682462046FAF77FF86A
:105CD00006F18043013B54F8230040EACA7044F8BF
:105CE0002300424621462846FAF74EF83B4602AAD0
:105CF000294628460096FAF75AFA3B4602AA294650
:105D000028460096FAF753FA02A908463B462A4667
:105D10000096FAF74CFA434602AA21462046F9F7C4
:105D2000F6FF0AAA3B46104621460096FAF73FFACC
:105D3000324629462046FAF76CF849462846FAF7D3
:105D400068F80AA94846FAF764F812B0BDE8F08787
:105D500031462046FAF73BF8C3E7000073B500234D
:105D60000DF102008DF80230FBF7A2F9264B1B78EB
:105D700003F0FF04002B41D1244B1A68002A3DD0C8
:105D8000234AD2F80813C90738D51C601B68214D77
:105D900001930DF10300019BD2F808658DF80340D3
:105DA000FBF786F96A6829681F2A98BF541CA1422C
:105DB000F6B26C6004D1202C14BF611C0021296054
:105DC00015499DF803008E542A6894423ABFC2F1E7
:105DD00021021319A31AAA689A4238BFAB60FBF7D5
:105DE00073FF6B682A681F2B94BF013300239A420C
:105DF00001BF074A0123C2F8083353609DF802002F
:105E0000FBF762FF02B070BDE1D0002000D100407E
:105E100000D00040CCD00020A8D0002030DF704758
:105E20002DE9F74F3B4F06468846B8F1000F03D1E6
:105E3000012003B0BDE8F08F4546202D28BF202566
:105E40005FFA85FB002400230DF102008DF802307B
:105E5000FBF72EF9304B1B7803F0FF0993BB0DF1D4
:105E600003008DF80390FBF723F9D7E900148C4267
:105E700004D3641AA54207D9052414E02134641A16
:105E8000A542F9D8C1F12104244BA542194431D8C7
:105E90002A4630463AF07EF83B682B44212B28BF37
:105EA00000233B6000249DF80300FBF70DFF1C4B13
:105EB00000221A601B680193019B1A4B0122C3F850
:105EC00004231A609DF80200FBF7FEFEB9F1000FF3
:105ED00008D059463046FFF7A1FF42F20703984227
:105EE0000446ADD0022CAED0002CA9D1A8EB0508F9
:105EF0002E449AE7224630463AF04CF8074BA5EB81
:105F0000040A5246194630193AF044F8C7F800A07E
:105F1000C8E700BFCCD00020E1D00020A8D00020EE
:105F200000D1004000D0004017B4314A314B116815
:105F300089B90021304A106820BB00205A79D40763
:105F400040D408B9002949D01C68DA88234603B038
:105F50005DF8044B1847002111601268D96800925F
:105F6000009A0029E5D0254AD2F84005814204BFB5
:105F7000D88801EB8001C2F840155A7942F004023A
:105F80005A71D7E700201060126898680192019A50
:105F90000028D2D0194AD2F83845A04204BFDC8884
:105FA00000EB8400C2F838055A7942F00202140767
:105FB0005A71C3D512F0010402BF64F3C3025A71CF
:105FC0002046BBE702F00601062907D122F00602AF
:105FD00011075A7106D56FF3C3025A7103B05DF809
:105FE000044B7047054AD2F83805D2F84015ABE7A4
:105FF0001451024034CA00200451024000500240B3
:10600000A5DF7047A4DF7047A3DF70472DE9F04795
:106010000E4690B016F01005814692469846189CA0
:106020000CD011238DF8083023788DF80930012227
:106030004FF0000362F342038DF80A301C22002166
:1060400009A8F9F76FFA8DF8246005B102AD42F6A0
:106050004D23ADF80C3063789DF864108DF8043052
:106060000022A3788DF80530134661F3C303DBB239
:1060700043F00303CDE906220E95012701AD8DF80B
:106080000630089203AE1A9BB9F800008DF80E7026
:1060900004AA09A9CDE90465ADF81CA0FDF706FD29
:1060A00058BB42F60813ADF80C3063788DF8043015
:1060B000A3788DF80530034667F342038DF8063068
:1060C0001A9A98F800308DF8003098F80130CDF821
:1060D0001A00ADF81E008DF8013032F8080B8DF86B
:1060E0000E70022304A9CDE90465ADF81830ADF8AF
:1060F0001C30CDF820D0FFF787FF10B0BDE8F08747
:10610000A1DF704708B5FAF7BBF910B14F4B504A01
:106110001A60FAF795F928B14E4B4F4A1B68C3F342
:1061200042331360FAF7ACF920B14C4AD36823F03C
:106130008073D360FAF784F940B14FF080430022B6
:10614000C3F80C21C3F81021C3F83825FAF798F9E1
:1061500010B1434B03221A60FAF792F940B1414B58
:1061600005221A6001229A6700229A603F225A6033
:106170003D4B1B78062B50D13C4B1B681B074CD169
:106180003B4B1B6803F0F003502B46D14FF080527D
:10619000384BD2F80414C3F82015D2F80814C3F809
:1061A0002415D2F80C14C3F82815D2F81014C3F82B
:1061B0002C15D2F81414C3F83015D2F81814C3F8FB
:1061C0003415D2F81C14C3F84015D2F82014C3F8C3
:1061D0004415D2F82414C3F84815D2F82814C3F88B
:1061E0004C15D2F82C14C3F85015D2F83014C3F85B
:1061F0005415D2F83414C3F86015D2F83814C3F823
:106200006415D2F83C14C3F86815D2F84014C3F8EA
:106210006C15D2F84424C3F87025FAF711F928B1A7
:10622000154B164A1B6803F04F031360144AD2F84B
:10623000883043F47003C2F88830BFF34F8FBFF348
:106240006F8F104B104A1A6008BD00BF74C0074022
:106250000DF0ADBA440200103C050040F0ED00E046
:10626000A005004010560040E00F00F0E40F00F0E1
:10627000E80F00F000C0004058020010E40E00409B
:1062800000ED00E0A82C00200090D003002382B095
:10629000036003680193019B02B070472DE9F3414D
:1062A000844BD3F8042162B3D3F800339F0728D579
:1062B000814D8248FFF7EAFF2B7803F0FF08F3B91E
:1062C0007F4F804E7B783C4603F0FF02002B00F0AE
:1062D000AF8073684046984701A88DF80480FAF7AC
:1062E000E7FE7B689DF8040001337B60FBF7ECFC64
:1062F000754B0122DA601A60744B00221A60012388
:106300002B706C4BD3F81821D2B1D3F8002356066A
:1063100016D5D3F824356E48DB08C3F3080113F40F
:10632000FF7F18BF0239FFF7B1FF624B4FF4805275
:10633000C3F808254A1EFE2A40F2A4800122DA6131
:106340005C4AD2F81031D3B1D2F80033DD0616D54D
:106350006048FFF79BFF1023C2F808335E4BC2F87A
:106360001035FF23C2F814350123D3615B4B1C6841
:106370002CB15B4800231A4603210068A0474D4A10
:10638000D2F84C3133B3D2F800331C0322D5554830
:10639000FFF77CFF4E48FFF779FF5348FFF776FF82
:1063A0004D4BC2F81035FF23C2F814350123D361D9
:1063B0004FF48863C2F804330D23C2F80C34C2F8DA
:1063C0000434464B1C682CB1454800231A46194634
:1063D0000068A047374AD2F828315BB1D2F80033C1
:1063E000580507D54048D2F80C34FFF74FFF0D236E
:1063F000C2F80C342F4AD2F81C31B3B1D2F80033B2
:10640000190612D53948D2F80414FFF73FFFCB071D
:1064100007D5374B197821B10121C2F804140022A5
:106420001A70244B0D22C3F8042402B0BDE8F08199
:106430000DF103008DF80320FAF73AFEBA6813460F
:1064400083B93260A660636833B92A4B1B7803F0C6
:10645000FF025BB1F9F7E6FA63689DF803000133C8
:10646000636043E7B342EED01B68E9E7224B1A6052
:106470001B680193019B4FF080430122C3F8042362
:106480001A60E9E7144A1078502803D1184901220C
:106490000A7054E711480468002C3FF451AF4FF6DE
:1064A000FF70C3F808050E480B4600680221A0479C
:1064B00046E700BF0050004058CC00200451004087
:1064C0006CCB002080CB002000B00140A02D00202C
:1064D000185100401051004000CE00200CCF002089
:1064E00010CF00204C510040285100401C5100406A
:1064F000E0D00020E1D000200001004013B5284B7F
:106500002849D3F83C3413F0030345D10A6801321B
:10651000072A0A602CD9244A012414610DF10700CE
:106520008DF80730FAF7C4FD204B5A68013A5A60DB
:106530005A6822B91E4A127802B3F9F771FA9DF827
:106540000700FBF7C1FBBFF35F8F1A4A00231360FC
:10655000BFF35F8F01211160174A14681CB11748FF
:106560001A460068A047164B00221A70FAF7FAFC88
:106570000D4B0022C3F8402102B010BD114A4FF06C
:1065800080411460D1F80C2402F00112B2F1011F15
:10659000F8D000225A70D2E700230B60E8E700BF72
:1065A00000500040A02D002000B001406CCB002026
:1065B000E1D00020FC5F00400CCF002010CF002075
:1065C00058CC0020040000408DDF704777DF704713
:1065D0002DE9F04F89B00E4600AF0023044607F1C5
:1065E000140130467B6133F051F9054618BB304643
:1065F0002FF0A2FE804678612DF026F908F5807311
:1066000083420CD9A64901202EF0A8FA3246A549AA
:1066100001202EF0A3FA2437BD46BDE8F08F08F123
:10662000070323F00703ADEB030D6D4642462946F1
:1066300030462FF071FE7E6926B99B4901202EF06D
:106640008DFAE8E74FF00308B6FBF8F303EB4303DA
:106650009E4201D09549F1E7204628F097FA08B903
:106660009349EBE7934BC7F808D004EB44041C4470
:106670006178914C2079002840F009818F4A0123EC
:10668000C2F80405FF29C2F82405C2F82005C2F8A3
:106690001C35C2F82805C2F818054FF0C050C2F8E2
:1066A0001405C2F8103518BF01F5E0704FF0A04393
:1066B00008BF4FF0FF31C3F85887C3F8FC8A18BFF2
:1066C00043F820801623C2F86435FF23C2F86835EA
:1066D0004FF0FF33C2F860352520C2F87015C2F8BC
:1066E0006C350221764B2360FEF744FF01232371B2
:1066F0000323B6FBF3F39BB203EB430808F1010855
:1067000028F001029100ADEB010D6846FA606D4A78
:106710003A6041184FF0000C796082F800C0E91C23
:106720004FF0EE09851C4FF0880A4FF08E0B634541
:106730005FDC0C2202FB030300227968994200F21D
:106740009E802679012E40F0A28000F06043B3F1D4
:10675000005F40F0A280FB68C3F34E02574B00215C
:10676000C3F85025C3F83815C3F80815C3F8400519
:10677000C3F80C656579E28025F0090545F0080548
:106780006571C4E90210C3F80065022323710D4648
:10679000002977D04FF6FE7208EA0202F8F7C2FE2F
:1067A000494B00221A601B68FB61FB69474B1A606A
:1067B0001B68BB61BB69414B2222C3F80423012241
:1067C0001A603A681278042AFBD94149002222252E
:1067D0000120C3F808530860C3F80025C3F8085324
:1067E0000860C3F800253B4B2021C3F884102271B8
:1067F00050E011F8026C11F8032C360246EA02460A
:1068000011F8012C05F10C0E164306F44012B2F5F6
:10681000001F1ED0B2F5401F20D0B2F5801F20D13E
:1068200005F802BC06F44002B2F5000F1CD0B2F528
:10683000400F1ED0B2F5800F1ED105F801BC023505
:10684000AE454FEA0616E0D10CF1010C0331754656
:106850006DE76FF0170205F8022CE3E705F8029CDC
:10686000E0E705F802ACDDE76FF0170205F8012C50
:10687000E5E705F8019CE2E705F801ACDFE703F87E
:10688000012B5AE7014623682846984788E70820E5
:10689000FBF7B8F9D7F808D0BDE61020F8E700BF3D
:1068A0004D010600641E0600901E0600B01E060084
:1068B000DB1E06008002060034CA002000500240A1
:1068C000818A030046D40020045102401451024042
:1068D0000450024000E100E010F5A24F0FD006DCAA
:1068E00010F5A34F0ED0414208482EF005B910F51F
:1068F000A14F09D010F1220FF5D1054900E005495B
:106900000548F2E70549FBE70549F9E7351B0600AD
:10691000111B0600261B0600F6370600EB1A0600C0
:10692000FD1A06002DE9F04FADF51B7D00AF1446B2
:1069300005461022884607F1180000219B46F8F70B
:10694000F1FD204632F0E1F90646002859D0002238
:10695000BE49204633F0C8FE064680B1102207F13A
:1069600018012FF0D9FCF389A3F500739BB2F381D2
:10697000F38903F4F05313B9304632F09BFB204601
:106980000022B34933F0B0FE0446002843D0B14999
:1069900032F0D8FC002840F05582AF49204632F052
:1069A000D1FC002840F05182AC49204632F0CAFCAC
:1069B000002840F04D82AA49204632F0C3FC00284E
:1069C00040F04982A749204632F0BCFC0646002828
:1069D00040F044822246A44901202EF0BFF8B1467F
:1069E000E389A3F500739BB2E381E38903F4F053D9
:1069F00013B9204632F05EFBB9F1000F0DD100262D
:106A000003E044B199482EF077F8304607F51B773C
:106A1000BD46BDE8F08F4FF001094FF48C720021A4
:106A200007F13800F8F77EFD002307F1140128462E
:106A30007B6132F02BFF0446D0B928462FF07CFC56
:106A4000064678612CF000FF06F58073834204D976
:106A5000874901202EF082F8D1E7F31D23F00703C8
:106A6000ADEB030D6C463246214628462FF054FC10
:106A7000002307F1100140463B6132F007FF054655
:106A8000A8B940462FF058FC064638612CF0DCFED1
:106A900006F580738342DBD8F31D23F00703ADEBCB
:106AA000030D6D463246294640462FF035FC3E69BF
:106AB000F600BBF1000F3DD14FF48C72594607F53B
:106AC000A870F8F72FFD07F140033246294607F575
:106AD000A870FB631CF040F88046F8B9D7F8501155
:106AE000D7F85401B9630B01C218C3583B6453680B
:106AF0007B649368BB64D368FB645E4E4B1E7B6013
:106B0000103A07F150037968002921DC11681960F7
:106B10005168596091689960D268DA60002340F248
:106B20001912184607F5A87119440133934208D089
:106B30000870F7E73246294607F138001CF00CF8D8
:106B40008046B8F1000F2ED04046FFF7C5FE56E74D
:106B5000A2F1040E03F1100A5EF8040F4649C5B213
:106B600016F805C0050E51F82CC0755D434951F863
:106B7000255043498CEA050CC0F30725C0F30740B4
:106B8000755D305C51F825503E4951F820008CEA83
:106B90000505454043F8045B5345DDD1796801396B
:106BA0007960103AAFE707F10C017869C7F80C80FB
:106BB000FAF7AAF9FD6806461DB933482DF09CFF87
:106BC0001DE709F1FF39B9F1040F00F23381DFE865
:106BD00019F00500AF00E30031012F01D7F814A030
:106BE0001AF00F0F40F02981BBF1000F4ED0013D8C
:106BF0000F3405F10109BAF1000F4FD007F1180168
:106C0000A4F1100328468B4613F801CF11F8012B8D
:106C10009C4282EA0C0200F8012FF5D14A4649460F
:106C200007F138001BF03CFE4A465B4605F1110EA9
:106C3000106851689C46ACE8030008327245634610
:106C4000F6D1AAF1100A10351034D2E7761A0600F0
:106C5000694B0600791A06007D1A0600811A0600A3
:106C6000851A0600891A06008D1A0600A41A060065
:106C70004D0106000F030600100406001010060068
:106C800010080600100C0600CE1A06000F35A244AC
:106C900007F5A8795445A5F10F0222D1002340F24F
:106CA0001912184607F1380119440133934240F094
:106CB000C780B8F1000F3FF4A8AE4046FFF70CFEC6
:106CC000002E3FF49CAEF389A3F500739BB2F381D1
:106CD000F38913F4F0547FF492AE304632F0EAF9BF
:106CE0008DE62346CE4604F1100B18685968F44629
:106CF000ACE8030008335B45E646F6D1214607F1D0
:106D000038001BF06FFC07F11801A5F110038C4649
:106D100013F8010F11F8012B9D4282EA00021A704C
:106D2000F6D199E80F0010348CE80F001035B1E768
:106D30007B69E3187B6007F5A87A07F118097B687F
:106D4000A342ABD099E80F008AE80F004A464946B3
:106D500007F138001BF0A4FDBBF1000F02D123782E
:106D60008AF8103099F8003014F8012B534005F8D8
:106D7000013BBBF1000F01D08AF8103007F251132C
:106D8000CC4607F2611E18685968624603C2083390
:106D900073459446F7D1D2E707F5A87B102200216E
:106DA000584607F1280AF8F7BDFB1022002150468B
:106DB000F8F7B8FB7A694FF00009A3189C423FF43A
:106DC0006DAFB9F1000F0BD01AF8092014F8011BB0
:106DD00009F101094A4005F8012B09F00F09EDE717
:106DE0005946524607F138007B601BF059FD7B681D
:106DF00007F5B07111F8012D0132D2B20A70002AE4
:106E0000E2D18B45F6D1DFE7FA6861192A4407F130
:106E10003800BBF1000F08D01BF042FD10357A6935
:106E200005F10F039A42EFD838E71BF0DBFBF5E7DB
:106E30000025F4E7DFF82C8030E76FF021082DE71C
:106E400008702FE74FF00109CAE54FF00209C7E5C6
:106E50004FF00309C4E54FF00409C1E54FF00509FF
:106E6000BEE500BF80AFFFFF0023FFF75BBD01233E
:106E7000FFF758BD70B500221649054633F034FCC3
:106E800033F0A4FF144B154906460322586833F02B
:106E90002BFC044678B10022B1B231F0E3F9E3896A
:106EA000A3F500739BB2E381E38903F4F05313B9B4
:106EB000204632F0FFF80A4B1C6824B1E38903F541
:106EC00000739BB2E3812846002114F0C3FC2046E6
:106ED00070BD00BFC31406008C2D0020D014060026
:106EE00034D4002008B540B2FFF770FBBDE808407D
:106EF00013F078BE38B5054608460C4631F01DFF44
:106F0000002808BF002422460E49284633F092FB91
:106F10000D4B4FF6FF72198874B18A4204D10020DC
:106F2000BDE8384013F05EBE00221888114615F007
:106F3000EBF90828F4D1F2E78A42F0D0188815F06E
:106F4000E1F9F6E79E140600E22C0020014B1888B8
:106F500014F0F0B8E22C0020014B188814F0EAB8C5
:106F6000E42C002008B5074B1A884FF6FF719142B8
:106F700007D018881321FDF795FDBDE8084013F0F0
:106F800031BE08BDE42C002007B5002308460722C7
:106F900069460093CDF8033034F05EF9094B1A8846
:106FA0004FF6FF71914209D018886A46012115F009
:106FB000D7F913F017FE03B05DF804FB43F20200AB
:106FC000F7E700BFE22C002038B500220E49054645
:106FD00033F08AFB0446A8B90C4928F0F7FC0A49AB
:106FE00004460246284633F025FB2A460849204637
:106FF00033F020FB002031F03DFC064902462046DC
:1070000033F039FB204638BD781406007D140600A5
:1070100097140600B914060010B5044631F075FE49
:10702000224630B92CB107490320BDE810402DF0AD
:1070300095BD054B0549586833F062FFBDE8104027
:1070400014F002BB251906008C2D00204E190600F5
:10705000F8B5044628B9214A136823F48043136025
:10706000F8BD1F4932F06EF90028F4D1204631F006
:1070700074FE054690B1194A1368204643F48043D4
:10708000136034F07DF953EC102B10EE100A194602
:1070900016F04AFCBDE8F84013F0A4BD204631F0DC
:1070A00034FE0028DCD00D4A0E49136843F48043B7
:1070B000136020462A4633F017FB34F0D3F92A46F2
:1070C00006460F462046084933F00EFB34F0CAF955
:1070D00002460B4630463946DAE700BF38D4002076
:1070E000F1170600F617060002180600084B1A688A
:1070F00018B142F400521A60704722F400521A602C
:10710000044B1860044B01221A7013F00DBB00BF32
:1071100038D4002050D400204DD40020F0B583B0E6
:10712000044600AF28B9014613F03AFB0C37BD46C0
:10713000F0BD31F05CFF28B1204633F00BF904219B
:10714000C0B2F1E77860391D204632F09FFB05465A
:10715000F0B920462FF0F0F8064678602CF074FB6A
:1071600006F58073834208D90D4901202DF0F6FC05
:107170000C4901202DF0F2FCD8E7F31D23F00703A2
:10718000ADEB030D6D463246294620462FF0C4F87C
:1071900079680029ECD0284613F034FBC6E700BF1D
:1071A0004D0106000B20060008B5044B0449586841
:1071B00033F08CFEBDE8084013F05CBB8C2D002042
:1071C0004B200600F0B583B0044600AF13F052FB2D
:1071D000002C69D00023391D20467B6032F056FB1D
:1071E000054610BB20462FF0A7F8064678602CF025
:1071F0002BFB06F5807383420CD93A4901202DF010
:10720000ADFC394901202DF0A9FC002420460C37A3
:10721000BD46F0BDF31D23F00703ADEB030D6D4636
:107220003246294620462FF077F878680028E8D0C3
:1072300031F0B0FB044608B92C49E3E72C4B2D494B
:107240000246586833F0F6F9E389A3F500739BB260
:10725000E381E38903F4F05313B9204631F02AFFA8
:10726000204631F09CFD7A68294638F093FE20468E
:1072700031F095FD0546204632F0DFFA01462846FA
:1072800013F008FB0023391D0A207B60F9F73CFE50
:107290007B680446002BB9D0174A11681960516801
:1072A000596012891A81B1E7204631F073FB044618
:1072B00020B90E4901202DF051FCA7E70C4B0D49D8
:1072C0000246586833F0B6F9E389A3F500739BB220
:1072D000E381E38903F4F053002BC8D1204631F059
:1072E000E9FEC4E74D0106000B200600222006003F
:1072F0008C2D00204B200600FFCE0020F0B583B07F
:10730000054600AF48B9424B4249586833F0DEFDAC
:10731000FFF74AFF0C37BD46F0BD0023391D7B60E7
:1073200032F0B4FA0646F0B928462FF005F80446C4
:1073300078602CF089FA04F58073834208D93649C5
:1073400001202DF00BFC354901202DF007FCE1E771
:10735000E31D23F00703ADEB030D6E4622463146D5
:1073600028462EF0D9FF78680028ECD0133031F091
:1073700011FB054608B92A49E6E7254B254902468F
:10738000586833F057F9284631F009FDEB89A3F529
:1073900000739BB2EB81EB8903F4F053044613B9FD
:1073A000284631F087FE1F4B224603F1100153F8A7
:1073B000040B42F8040B8B42F9D11B8813807D68C3
:1073C00031462A4604F1120038F0E4FD6574254484
:1073D000FE23AB740020FFF7F5FE3946054632F078
:1073E00055FA28B1036823604368636003892381E9
:1073F000002D8FD0EB89A3F500739BB2EB81EB8955
:1074000003F4F053002B85D1284631F053FE81E779
:107410008C2D0020032006004D0106000B200600E5
:1074200022200600E40206002DE9F04182B0054664
:1074300000AF50B9594B5A49586833F047FDFFF730
:10744000B3FE0837BD46BDE8F08131F011FD28B923
:107450002A46544903202DF081FBF2E70023391D11
:1074600028467B6032F012FA0446F0B928462EF026
:1074700063FF064678602CF0E7F906F580738342D7
:1074800008D9494901202DF069FB484901202DF018
:1074900065FBD6E7F31D23F00703ADEB030D6C4648
:1074A0003246214628462EF037FF7D68002DECD06D
:1074B00007223F49204638F05FFD60B9073D073499
:1074C0007D604FF0030878681B3031F063FA0646A0
:1074D00080B93849DAE708223749204638F04CFDB0
:1074E00028B9083D08347D604FF00408EBE74FF001
:1074F0000008E8E7294B2A490246586833F09AF811
:10750000304631F04CFCF389A3F500739BB2F38154
:10751000F38903F4F053054613B9304631F0CAFD40
:10752000264B2A4603F1180153F8040B42F8040BCA
:107530008B42F9D11B8813807E6885F8198021461B
:10754000324605F11A0038F025FDF3B203F10802C6
:107550002E440133EB75FE236A740020B376FFF7E7
:1075600031FE3946044632F091F928B103682B60A8
:1075700043686B6003892B81002C3FF462AFE38981
:10758000A3F500739BB2E381E38903F4F053002B6E
:107590007FF457AF204631F08DFD52E78C2D00204F
:1075A00003200600971F06004D010600B21F0600CB
:1075B000C91F0600DA1F0600D11F0600E4020600FC
:1075C00010B5044631F0B9FB084B0949002808BF43
:1075D00000242246186833F02DF8201C18BF012023
:1075E00014F094FEBDE8104013F0FCBA8C2D00207E
:1075F0009E1406002DE9F74F504B514905460322D2
:10760000586833F071F80646002845D000224D49ED
:10761000DFF83081284633F067F831468146684606
:107620002CF00FFC009CECB1204632F072FE0022E0
:107630004146074633F058F8012300224946824666
:10764000F9F7FAF858BBFB8903F500739BB2FB818D
:107650003C465046394632F04FFD68462CF0DCFB84
:10766000002CDFD0009850B1C389A3F500739BB202
:10767000C381C38903F4F0530BB931F01BFD2946D4
:10768000002C57D001A82CF0DCFB019D4DB93246EF
:107690004946204632F004FD03B0BDE8F08F0024D7
:1076A000D7E7EB8903F500739BB2EB81284632F0F4
:1076B00030FE012229460746204633F095F922493B
:1076C0008046284631F03EFE20498246284631F069
:1076D00039FEBAF1000F00D1D0B1404632F019FEA8
:1076E000834610B3BAF1000F1BD00122394630F0A7
:1076F000E5FCBBF80E20A2F5007292B2ABF80E20AA
:10770000BBF80E2002F4F05212B9584631F0D2FC08
:1077100040463A46294632F0C3FC01A82CF07CFBD7
:10772000B3E7394633F0BDF9E3E73946404632F076
:10773000E9FBEDE730462FF0C7FCA8E78C2D0020D1
:10774000A5150600FF160600AC150600B5150600C7
:10775000F8B5064608460C4631F0D7FA074620B37E
:1077600000223949204632F0BFFF33F044FC0022AA
:1077700007463649204632F0B7FF0446E0B131F003
:10778000BCFAC8B9E389A3F500739BB2E381E3892E
:1077900003F4F05313B9204631F08CFC22462C49F7
:1077A0000320BDE8F8402DF0D9B92CB12246294973
:1077B00003202DF0D3F93C46304631F0BEFA0028C4
:1077C0003AD0002E38D048F24801234831F0A1F8D1
:1077D0000546D0B12246002133F02CFA32461F492B
:1077E000284632F027FF1E4B1E4918682A4632F001
:1077F00021FFEB89A3F500739BB2EB81EB8903F4C6
:10780000F05313B9284631F055FC301C18BF012045
:10781000394613F0BFF813F0E5F9A4B1E389A3F5F5
:1078200000739BB2E381E38903F4F0535BB9204614
:10783000BDE8F84031F03EBC094B0A49186833F006
:1078400045FB0026E1E7F8BD18180600C116060042
:107850001F18060053180600217A02006C18060053
:107860008C2D0020711806002DE9F84380460C4647
:1078700031F063FA30B9384942460120BDE8F84397
:107880002DF06CB9204631F068FA05462046C5B1A6
:1078900033F076FD57EC106B002432463B46304601
:1078A000394638F0FDF830B900222C4B30463946C5
:1078B00038F0CEF8C8B12A490120BDE8F8432DF0D0
:1078C0004DB931F022FA50B12A462649204632F00D
:1078D0000BFF40B133F0C6FD06460F46DDE714B19D
:1078E00022462149C9E7214F0026214DD5F80490B1
:1078F00031F019F81F490246484632F0BCFE4246B4
:107900001D49686832F096FE08211C4831F001F8E4
:10791000054670B12146FFF71BFFEB89A3F5007305
:107920009BB2EB81EB8903F4F05313B9284631F095
:10793000C1FB0021124830F0ECFF044648B10021A1
:1079400047EC106B0DF0C8FE2146BDE8F84332F05D
:10795000D3BBBDE8F88300BF3B1506000000244000
:107960008C150600941506006915060000409F401E
:107970008C2D0020A51506009C150600F57502004B
:107980008579020037B5144C00210846FFF7E0FE68
:1079900003221249606832F0A7FE002201901049CC
:1079A000606832F0A1FE0D490546606833F08EFA3A
:1079B0000B49606833F08AFA019B33B12DB1012382
:1079C00001AA2946002026F065F92946019832F0DF
:1079D00093FB03B030BD00BF8C2D0020A515060021
:1079E0009C1506001FB54FF08052D2F8A430D2F893
:1079F000A820D8B20290C3F307200190C2F3072158
:107A0000C3F3074000901B0ED2B241F0C0010348FF
:107A100031F0C4FD05B05DF804FB00BFC1150600E0
:107A20002DE9F04F8BB000AFC7E902011446002AE0
:107A300076D09E49002027F0C9FF00220546386114
:107A40009B49204632F050FE99490246284632F0C2
:107A500012FE002297493D69204632F045FE9549C5
:107A60000246284632F007FE30F05DFF804604F003
:107A70007DFF002283469049204632F035FE814644
:107A8000E8B102468C49386932F0D4FD002307F191
:107A9000240148467B6231F0F9FE044600284ED1AD
:107AA00048462EF049FC054678622BF0CDFE05F5E0
:107AB0008073834238D9814901202DF04FF8B8F105
:107AC000000F07D0D8F8003023B142467C4938690E
:107AD00032F0B0FD584631F0B0FE20B15A46794937
:107AE000386932F0A7FD5A464146484632F0D8FA86
:107AF000FB68002B40F0C08007F110030122002139
:107B0000B86827F091FE386950B1C389A3F50073B6
:107B10009BB2C381C38903F4F0530BB931F0CAFAA5
:107B20002C37BD46BDE8F08FEB1D23F00703ADEB0E
:107B3000030D6C462A46214648462EF0EDFB7B6A33
:107B4000002BBCD0B8F1000FC4D0BBF1000FB6D0F1
:107B5000002514E0092A09D1A91C2144701ED7F878
:107B600010A032F0FDF85849024619E0911E012993
:107B700027D89A4602239E4216DA013635447B6A9C
:107B8000AB429CD96319665D5A78082AE2D1A91CD8
:107B90002144701ED7F810A032F0E2F84B4902469B
:107BA000504632F068FDE8E73AF8021F48487B602B
:107BB00031F0F4FC0146404630F0DEF97B680233D8
:107BC000D9E7911F012908D8A81C20441BF0B8FC54
:107BD0000146404630F0D0F9CFE7162A33D1598814
:107BE0003B4831F0DBFC33F090FE82460028C4D0E5
:107BF00001220146584632F0F7FE291D78602144E3
:107C0000F01E2EF078FE7B6802463BB130B1014693
:107C10003860184632F076F9D7E900231846114645
:107C200032F06AFABAF80E30A3F500739BB2AAF8E4
:107C30000E30BAF80E3003F4F053002B9DD15046AD
:107C400031F038FA99E7FF2A97D1D8789B78D7F89E
:107C500010A043EA002030F015FE1E4902465046AF
:107C600032F009FD291D2144F01ED7F810A02EF096
:107C700042FE1949024693E7D7E9031607F11400BB
:107C80002CF0DFF8786948BB0446786950B1C389A5
:107C9000A3F500739BB2C381C38903F4F0530BB9FE
:107CA00031F008FA002C7FF427AF2CE7E218060029
:107CB000FF160600A41406001D2006004D01060054
:107CC000AC150600B515060073200600F218060074
:107CD000C7780600FC1806000919060032F019FBE7
:107CE0000022BA49054632F0FFFC8046002800F029
:107CF0000F810022B549304632F0F6FC41468146FC
:107D000007F118002CF09DF80124B869002840F014
:107D1000CC804946404632F0EFF90022AC49284673
:107D200032F0E2FC8046E0B10022A949304632F050
:107D3000DBFC8146404631F0E2F8002800F0EA80A2
:107D4000484631F0DCF8002800F0E480494640461F
:107D500031F058FE00284946404608BF002432F062
:107D6000CBF900229B49284632F0BEFC804610B376
:107D700000229749304632F0B7FC8146404631F048
:107D800077F898B1484631F073F878B1404631F051
:107D900020FD8246484631F01CFD824506D801236D
:107DA000002249464046F8F747FD00B10024494605
:107DB000404632F0A1F900228749284632F094FC6F
:107DC000804680B100228449304632F08DFC014665
:107DD0008146404631F016FE49460028404608BF1D
:107DE000002432F089F900227C49284632F07CFCDC
:107DF0008046F0B130F089FF60B1414607F12400C0
:107E00002CF01FF8DFF8D4A1D7F824B0BBF1000F95
:107E100040F09480B8F80E30A3F500739BB2A8F838
:107E20000E30B8F80E3003F4F05313B9404631F079
:107E300041F900226A49284632F056FC8046F0B1EA
:107E400030F063FF60B1414607F124002BF0F9FFE9
:107E5000DFF894A1D7F82490B9F1000F40F0998091
:107E6000B8F80E30A3F500739BB2A8F80E30B8F83E
:107E70000E3003F4F05313B9404631F01BF95DB1F5
:107E8000EB89A3F500739BB2EB81EB8903F4F0530C
:107E900013B9284631F00EF907F114002BF0BCFF9E
:107EA000002C3FF4EFAE0124EFE6B9F1000F12D041
:107EB00032F02FFA014607F11C001BF0BDFA4946CB
:107EC00007F120002BF0BDFF4FF0000A386A40B9DF
:107ED000BAF1000F00D1002407F118002BF09CFF2D
:107EE00013E732F016FA014607F124001BF0A4FA5A
:107EF000BA7F97F826309A4205D1BA8BBB8C9A424A
:107F000008BF4FF0010A07F120002BF085FFDDE7E5
:107F1000012402E7334BA8EB03000011013082B2C9
:107F2000B9F1000F08D0A9EB03000011013080B2B5
:107F3000131A584258410DE74846F9E7BBF80E308E
:107F400003F500739BB2ABF80E3000225146304669
:107F500032F0CAFB814648B900245846494632F0FF
:107F6000CBF807F124002BF057FF4DE700225946CC
:107F700032F03AFD0028EFD0C389A3F500739BB21D
:107F8000C381C38903F4F053002BE6D131F092F89A
:107F9000E3E7B9F80E3003F500739BB2A9F80E3091
:107FA00000225146304632F09FFB83460146484648
:107FB00031F028FD59460028484608BF002432F019
:107FC0009BF807F124002BF027FF43E7AC150600D0
:107FD000732006001A190600FF160600B5150600E4
:107FE00009190600AC2D0020FC1806002DE9F0410F
:107FF00086B000AF00238846391D06467B6031F00D
:1080000045FC0546E0B930462EF096F90446786006
:108010002BF01AFC04F58073834206D93F490120F6
:108020002CF09CFD32463E4938E0E31D23F0070367
:10803000ADEB030D6D462246294630462EF06CF915
:108040007B68002BEED0404630F077FE28B1354BF0
:1080500035491868424632F0EDFA344B1A6812F08E
:10806000400F1E4607D1324901202CF077FD18370A
:10807000BD46BDE8F0812F4A12884FF6FF7191424C
:1080800001D12D49F0E71A6812F0800201D02B4986
:10809000EAE77C68102C05DD2949102201202CF02C
:1080A0005DFDE4E7274B93F800C0274BA4B2BCF179
:1080B000000F23D19A7C62B3B3F8760188422AD0AC
:1080C0009B8A7C80C7F80AC0A7F80EC03B810123B9
:1080D000BB7207F10801BB1CC7E90435FBF7E4FCE0
:1080E00018B97B88A34218BF0C2012F07BFD002832
:1080F000BDD1336843F080033360B8E7B3F876014D
:10810000884208D07C80C7F80A20FA81B3F84E3143
:10811000DCE70720E9E70820E7E700BF4D0106009C
:10812000681706008C2D0020F816060038D40020B1
:1081300002170600E42C002016170600251706007B
:108140003D1706004CD400206CCC00202DE9F04FE8
:10815000B04B91B01B681B0700AF044607D5AE4972
:1081600001202CF0FBFC4437BD46BDE8F08F15F034
:1081700055FC204630F0C9FD8046002800F05E81A5
:10818000214607F114002BF05CFEDFF8ACA2796900
:1081900081B10023BB61CB8903F500739BB2CB8116
:1081A00007F118001BF048F9024698B19B490120DD
:1081B0002CF0D4FC78690028D5D0C389A3F50073CE
:1081C0009BB2C381C38903F4F053002BCBD130F0B1
:1081D00071FFC8E77D691DB1284632F09AF805465F
:1081E000294607F11C002BF02CFEF969B8F1000FAD
:1081F0000FD071B1CB8903F500739BB2CB8107F12E
:1082000020001BF019F9024610B3854901202CF01B
:10821000A5FCF86950B1C389A3F500739BB2C38173
:10822000C38903F4F0530BB930F044FF5DB1EB891F
:10823000A3F500739BB2EB81EB8903F4F05313B900
:10824000284630F037FF07F114002BF0E5FD9EE7DC
:1082500007F128003C8C97F822601BF0B1F908B1B7
:10826000F9F7D0FC4FF00009002207F13001388DFA
:10827000C7F830901BF0A2F9052810D043F2030292
:1082800090420CD0A8B93B8EA34214D197F832305B
:10829000B34210D1B7F82890B9F1000F0FD1386A66
:1082A0001BF064F95F490446024601202CF056FC9D
:1082B00048E0F9F7A7FC3B8D01333B85D4E7FC6927
:1082C0001CB1204632F025F80446002256492046CB
:1082D00032F00AFA002255490646204632F004FAE6
:1082E00032F089FE0022B8605149204632F0FCF994
:1082F00032F081FEF8602EB3002307F124013046EE
:108300007B6231F0C3FA8346002837D130462EF025
:1083100013F8786278602BF097FA7A6802F5807328
:10832000834221D9434901202CF018FCF389A3F59D
:1083300000739BB2F381F38903F4F05313B9304611
:1083400030F0B8FE5CB1E389A3F500739BB2E38122
:10835000E38903F4F05313B9204630F0ABFE07F184
:108360001C002BF059FD40E7D31D23F00703ADEBB4
:10837000030DEB46594630462DF0CEFF7A6A002AAF
:10838000D4D0002179853A85494607F12802BAF808
:108390000000C7F82CB0FDF735FE12F023FCBB68D7
:1083A00080F001005FFA80F813B9FB68002BBDD0A4
:1083B000BAF800204FF6FF719142B7D0FB68BAF8C7
:1083C0000000A7F830900022002BC7F83220FA8670
:1083D0007A6A7A8214BF0222012287F8322007F1DA
:1083E000300107F11202C7E90E2BFBF75DFB30F0FD
:1083F00008029BD043F20402904297D043F201421C
:10840000904293D012F0EEFB002818BF4FF0000806
:108410008CE700BF38D40020BB190600E319060022
:10842000FC1906002C1A0600F63F06001C1A06006E
:10843000231A06004D010600E42C0020002C3FF416
:1084400092AE2246024903202CF088FB8BE600BF47
:10845000501A06002DE9F04F9BB000AF0D460446C0
:108460003C22002107F12C00F7F75CF8022387F883
:108470002C302846062387F82F3030F046FC0028A1
:1084800000F08D8000228E49284632F02DF938B157
:1084900032F0B1FD002814BF0223002387F82C30EE
:1084A00000228849284632F01FF938B132F0A3FD86
:1084B000002814BF0623052387F82F3000228249A5
:1084C000284632F011F9064618B3002307F10C01D3
:1084D000FB6031F0DBF9804600284ED130462DF0AC
:1084E0002BFF8146F8602BF0AFF909F580738342CA
:1084F00037D9764901202CF031FBF389A3F50073BD
:108500009BB2F381F38903F4F05313B9304630F092
:10851000D1FD284600226E4932F0E6F8054690B1BA
:108520003B6D002B36D031F015FF3B6D1880EB8989
:10853000A3F500739BB2EB81EB8903F4F05313B9FD
:10854000284630F0B7FD204630F0D7FB80B3E389F2
:1085500003F500739BB2E38120466C37BD46BDE84E
:10856000F08F09F1070323F00703ADEB030DE84695
:108570004A46414630462DF0CFFEFA68002ABCD06C
:1085800084B06B464FF6FF713B6519809A80C3F843
:108590000880B2E74F4903202CF0E0FAC7E7002D2E
:1085A000D1D04D492A4603202CF0D8FA0024D3E735
:1085B000204630F086FB06460028C8D1204630F021
:1085C000A4FB002876D0204630F00EFE0C23584342
:1085D000073020F00700ADEB000D214607F1080041
:1085E0002BF02FFCE946DFF8E4B04D46B246B86800
:1085F000C0B987F85860C7F854901F2307F10802E4
:1086000007F10C0107F12C003B81FCF7F3FA12F0A3
:10861000E9FA0028CAD107F10C0138892EF06BF96C
:10862000044699E731F075FE07F10C010446C7F8DE
:108630000CA031F02BF9804678B920462DF07CFE55
:10864000F86078602BF000F97A6802F58073834255
:1086500025D9594601202CF081FA5CB1E389A3F5B4
:1086600000739BB2E381E38903F4F05313B920460E
:1086700030F020FDB86820B1C38903F500739BB2C8
:10868000C38132F0A3FBFB682880AB80C5F808806B
:1086900007F108002BF0C0FB01360C35A7E7D31D0E
:1086A00023F00703ADEB030DE846414620462DF0CD
:1086B00033FED2E7002CA0D02246084973E700BF62
:1086C000DF150600E8150600091906004D01060031
:1086D000FC180600F5150600291606005F160600B0
:1086E00008B5054A136823F40073136012F09AFD6D
:1086F000BDE8084012F076BA38D4002008B5054A23
:10870000136843F40073136012F06EF9BDE808407B
:10871000FEF728BC38D4002008B518F0A9FE41ECBB
:10872000100B08BD08B50C4B1B884FF6FF729BB2AF
:10873000934203D1094A1288934208D0084825F091
:1087400035FB084A136843F00803136008BDBDE811
:10875000084014F0C7BE00BFE22C0020E42C00202B
:10876000C916060038D4002038B50F4C0F49002236
:108770000546606831F0B8FF32F028FBC3B27DB126
:1087800043F0010098420ED0646830F07BF807494E
:108790000246204631F06FFFBDE83840FFF7C2BF08
:1087A00003F0FE00EEE738BD8C2D00200E18060009
:1087B0002DE9F0418CB006460F4630F0A6FA40B9DC
:1087C0003EB13246524903202CF0C8F90CB0BDE846
:1087D000F0810023029301934E4B039302AB059368
:1087E0004D4B06934FF003080B23ADF81C300DEBF7
:1087F000080301220893494B8DF803200993424650
:1088000001AB03A93846ADF81080ADF828800B9372
:108810002EF0F0F80028D9D00298414D414C30F0AC
:1088200052FB48B1029A4049686831F003FF23685F
:1088300043F00803236009E0029B002B4AD13A4928
:10884000686832F043FB23685906F0D4029850B1AF
:10885000C389A3F500739BB2C381C38903F4F053AA
:108860000BB930F027FC9DF80330002B37D023687C
:108870002E4968689A065EBF236843F008032360A8
:1088800032F024FB32462A49686832F039FB3A4616
:108890002849686832F034FB019A1AB1236843F022
:1088A000080323602449686832F02AFB019850B11C
:1088B000C389A3F500739BB2C381C38903F4F0534A
:1088C0000BB930F0F7FB236813F0180F1BD0FFF73C
:1088D00029FF7BE7194940462CF040F9B6E72368A9
:1088E000D5F804809B0648BF23684FF0000044BFC2
:1088F00043F0080323602FF0BDFF0C4902464046B9
:1089000031F0B9FEBEE7304614F00EFE5EE700BF60
:10891000501A0600FE160600561906005B190600DE
:108920008C2D002038D4002065190600941906000B
:108930009D190600A7190600B11906006F19060057
:1089400013B5694604461AF08BFD28B90749012082
:108950002CF004F902B010BD054B064958682246B8
:1089600031F068FEFFF7DEFEF4E700BF8017060077
:108970008C2D0020B617060070B50D4D2A780646DE
:108980000C462AB101200B492CF0E8F8002070BDFC
:1089900009F08EFA084B2E70186024B1E38903F5B4
:1089A00000739BB2E381054B01201C60EFE700BF21
:1089B0003CD400205514060034D4002040D40020BC
:1089C00037B50546002105208DF80610FFF7D4FFC6
:1089D00070B1084B1C6824B1E38903F500739BB2A6
:1089E000E3810199284612F075F8204603B030BDA6
:1089F0000446FAE734D4002037B505460C46052076
:108A00000021FFF7B9FFD0B1214601A81AF054FCAC
:108A1000024638B10B4901202CF0A0F80024204672
:108A200003B030BD084B1C6824B1E38903F5007323
:108A30009BB2E3810199284612F04CF8EFE7044617
:108A4000EDE700BFF637060034D4002013B500214F
:108A500004208DF80610FFF78FFF68B1074B1C68E4
:108A600024B1E38903F500739BB2E381019812F00E
:108A700081F8204602B010BD0446FAE734D4002045
:108A800013B50C4604200021FFF776FFC8B121463C
:108A900001A81AF011FC024638B10B4901202CF054
:108AA0005DF80024204602B010BD084B1C6824B1BC
:108AB000E38903F500739BB2E381019812F05AF841
:108AC000F0E70446EEE700BFF637060034D4002096
:108AD00038B5124D2A8801464FF6FF70904215D0E6
:108AE0000320FFF749FF78B10D4B1C6824B1E389DF
:108AF00003F500739BB2E38113212888FBF7D2FFB3
:108B000012F070F8204638BD0446F5E7FDF75CFD2D
:108B1000BDE83840084609F03FBA00BFE22C00200B
:108B200034D400202DE9FF4100220F463149804610
:108B300031F0DAFD00223049064631F0D5FD6946B4
:108B400005461AF08DFC044658B92946304631F0E6
:108B5000D3FA2A4903202CF001F8204604B0BDE8DE
:108B6000F0815EB1F389A3F500739BB2F381F389C1
:108B700003F4F05313B9304630F09CFA414602201A
:108B8000FFF7FAFE80B90024002DE6D0EB89A3F5AB
:108B900000739BB2EB81EB8903F4F053002BDCD123
:108BA000284630F087FAD8E7482115482FF0B1FE63
:108BB00004460028E7D00223014602AA0020CDE99E
:108BC000025725F067F8E389A3F500739BB2E381B0
:108BD000E38903F4F05313B9204630F06BFA094BE4
:108BE0001C68002CD0D0E38903F500739BB2E381AD
:108BF000CAE700BF97140600FF160600F714060028
:108C0000B9BA020034D4002070B504460E460020E4
:108C1000184926F0DBFE054610B90025284670BD30
:108C20002246154931F006FD2846FEF7CDF9EB89BD
:108C3000A3F500739BB2EB81EB8903F4F053044678
:108C400013B9284630F036FA002CE6D031462046DB
:108C5000FFF768FFE389A3F500739BB2E381E38923
:108C600003F4F0530546002BD8D1204630F022FA09
:108C7000D4E700BFE2180600FF1606002DE9704396
:108C8000064658B130F041F8044638B932464E49EC
:108C900003202BF063FF2046BDE8708300224B4980
:108CA000304631F021FD044630F027F898B95CB128
:108CB000E389A3F500739BB2E381E38903F4F053E6
:108CC00013B9204630F0F6F92246414903202BF033
:108CD00045FF0024DFE75CB1E389A3F500739BB295
:108CE000E381E38903F4F05313B9204630F0E2F94D
:108CF00000223849304631F0F7FC32F0B3FB02462F
:108D00000B468046894636F0CBFE30B90022002360
:108D10004046494636F0A6FE18B1DFF8C8904FF03D
:108D2000000800212C482FF0F4FD0446002846D00E
:108D3000002149EC108B0CF0CFFCE389A3F5007304
:108D40009BB2E381E38903F4F053054613B920464F
:108D500030F0B0F929460120FFF70EFE002830D090
:108D600008211E482FF0D5FD044670B13146FEF7AC
:108D7000EFFCE389A3F500739BB2E381E38903F47D
:108D8000F05313B9204630F095F9154B1C6824B107
:108D9000E38903F500739BB2E381002D3FF47BAFC1
:108DA000EB89A3F500739BB2EB81EB8903F4F053DD
:108DB000002B7FF470AF284630F07CF96BE7054656
:108DC000C8E70446E9E700BF8C160600C116060096
:108DD0001F18060094150600CDB6020025BC02003F
:108DE00034D4002000409F4030B5154691B0002299
:108DF00031F07AFC0446C0B16946402232F02CFAC8
:108E00000C49684637F0EEF888B168461FF04CFB15
:108E10002860E389A3F500739BB2E381E38903F43F
:108E2000F05313B9204630F045F911B030BD024877
:108E3000EEE700BF101406007F0000012DE9F04F9F
:108E4000B64B1B78B5B0022B0D460C924FF00004C8
:108E500007D00120B2492BF081FE204635B0BDE895
:108E6000F08F17A81FF05AFB0028F7D011A81BF0AD
:108E7000F3F99DF845209DF8443013439DF84620B2
:108E800013439DF8472013439DF8482013439DF852
:108E9000492013430AD108238DF845304FF4EE736F
:108EA000ADF8463040F20233ADF8483028462FF096
:108EB0002CFF0746002855D00DF14A029949284653
:108EC000FFF792FF0DF14E0297492846FFF78CFFFE
:108ED0000DF1520295492846FFF786FF0DF1560223
:108EE00093492846FFF780FF00229249284631F037
:108EF000FBFB0646D8B1402224A932F0ADF900248C
:108F000024AF254617F8018BB8F1000F14D134AB0C
:108F10001C4404F88C5CF389A3F500739BB2F381C5
:108F2000F38903F4F05313B9304630F0C3F801234A
:108F30008DF85A30002459E040462AF0DCFD0F2815
:108F400004D800EB051523461C46DBE7B8F13A0FC1
:108F5000E1D134AA631C1444052B04F88C5CDADCE0
:108F60000025F1E71BF00AFC734B744A1A600646B1
:108F7000062211A909201AF025FB042210A90F20AE
:108F800010971AF01FFB042210A901201AF01AFBF7
:108F9000042210A905201AF015FB3B4644220221A9
:108FA00030461BF09DF8664D11A930461BF0DCFAE7
:108FB00001232B70634B1F7018F0B6FD624B10F548
:108FC000200041F10001C3E90001604B1F7095F9D9
:108FD0000030032BAED05B4B1B78012B2ED15C48AD
:108FE0005C4C24F0E3FE5B482BF066FD11A81BF0FF
:108FF0005DF917A81FF078FA0C982FF09EFEC8B103
:10900000002C00F0F481204630F010FF2490012362
:10901000002024AA0C9924F03DFE249850B1C38965
:10902000A3F500739BB2C381C38903F4F0530BB95A
:1090300030F040F8B4FA84F040090FE72AF0E0FB82
:1090400007460028CBD130461AF04CFB02460028D8
:1090500000F02A810DF13E0300933F4924AB3046D6
:109060001AF09AFDBDF83E303B4A432B40F0B080E9
:1090700002F11C0111AC3B4611F801CB14F8017B45
:10908000BC4540F00F8101339BB2062BF4D1138A0B
:10909000ADF84A30538AADF84C3080B22F4BF038DF
:1090A00003440D932E4B1A7807925A780A9293F83C
:1090B00003C09A782B4B03925A780B920022DF78E8
:1090C00098781B780593CDE90822244B06920492E8
:1090D00014460D9999420AD8049B002B65D0214B68
:1090E0000B9959700599DF70987019705DE093F8CD
:1090F00000E0BEF1060F00F0AA8035D8BEF1010FE6
:109100007AD0BEF1000F6FD0BEF1030F00F0838064
:1091100003F102085B78984468E000BF58D400204F
:109120007D1B06009C3806009B1B0600A21B060048
:10913000AA1B0600AE1B060004D20020785634128B
:1091400044D4002008D2002060D4002068D400203D
:10915000B21B0600711B06000CD20020FCD20020BE
:10916000FFD1002048D40020BEF1350F40D00DD8EB
:10917000BEF1330FCCD119799F78D8780B9103F1D8
:1091800006085B790593012304932FE0BEF1360FA7
:1091900079D0BEF1FF0FBBD1049B33B1994B9870CE
:1091A0000B9858700598DF701870099B13B1964B97
:1091B00007991970089B13B1934B0A995970069B34
:1091C00013B1914B0399997012B18F4B83F803C07F
:1091D00095F90030013B032B3FF6F9AEDFE813F0C1
:1091E00066007700A300E40003F10108434670E73E
:1091F00003F103089C78F9E703F1020E0DF14E0824
:1092000003F106091EF801AB08F801ABCE45F9D110
:1092100003F10608EAE793F801E003F102080DF113
:10922000520903F1060A18F801BB09F801BBD04541
:10923000F9D14FF000090633AEF1040E1FFA89FA96
:10924000F24503EB090809F10109F7DBCEE793F8D2
:1092500001E003F102080DF1560903F1060A18F8BE
:1092600001BB09F801BBD045F9D14FF00009063325
:10927000AEF1040E1FFA89FAF24503EB090809F171
:109280000109F7DBB2E79A780792DA780A921A793D
:109290000392012203F1060893F805C00692CDE976
:1092A0000822A3E7002493E7044691E7022C40F04C
:1092B0009980564824F07AFD4FF0FF33249324AA76
:1092C00011AB534930461BF051F82C707FE6052C4A
:1092D00016D1504824F06AFD1BF012F811A81AF0BC
:1092E000E5FF18F021FC4C4B10F5200041F1000186
:1092F000C3E90001494B00221A7003232B7066E674
:10930000062C6FD1464824F051FD18F00DFC424B5D
:1093100010F5200041F10001C3E900013F4B00229C
:109320001A700123EAE7374B1F687B1C3FF44FAEEE
:1093300018F0FAFB7A08002382428B41BFF647AE51
:10934000384824F033FD384B9DF84A201A709DF8B8
:109350004B205A709DF84C209A709DF84D20DA7081
:10936000294B1A788DF890205A788DF891209A78A8
:109370008DF892202D4ADB788DF8933013680133F5
:1093800013600DF14A0111AB24AA30461AF0EEFF2A
:1093900004232B7018F0C8FB1F4B10F5200041F17F
:1093A0000001C3E9000112E6052C19D11B4A1E4930
:1093B000002313700DF14A0211F8017B12F8010B22
:1093C000874218D101339BB2042BF5D118F0ACFBC6
:1093D000114B10F5200041F10001C3E900018CE7B9
:1093E000062C92D011A930461BF05EF9EFE5022061
:1093F0002FF0E0F90AE61AF083FF11A81AF056FFE1
:10940000E4E700BF48D40020FFD10020CF1B0600B6
:10941000FBD10020E61B060060D4002068D40020A9
:10942000FB1B0600111C060030D4002004D20020D3
:109430002DE9F041364B1F78022F98B0884608D0AE
:10944000344901202BF08AFB0024204618B0BDE8E7
:10945000F0810BA81FF062F8002857D005A81AF079
:10946000FBFE03F083FA0A252E26044604230DF1A1
:109470001A022949CDE900561FF07BF904230DF1AA
:109480001E0226492046CDE900561FF072F904233A
:109490000DF1220222492046CDE900561FF069F95C
:1094A00004230DF126021F492046CDE900561FF086
:1094B00060F910233A22CDE900321B49062305AAA0
:1094C00020461FF056F90BA81FF00EF840462FF06B
:1094D00034FC0028B9D038462FF06CF93B46CDE972
:1094E000030403AA0020414624F0D4FB039800287B
:1094F000ABD0C389A3F500739BB2C381C38903F4C6
:10950000F053002BA1D12FF0D5FD9EE704469CE738
:1095100058D400207D1B06009C3806009B1B0600CB
:10952000A21B0600AA1B0600AE1B060010B58EB0DB
:109530000446032101A81FF097F801A81EF0E8FFD8
:1095400001A81EF0D1FF084B08495868224631F0A7
:1095500071F8074B02221A70E38903F500739BB27E
:109560002046E3810EB010BD8C2D0020931F060015
:1095700058D40020024B1B680021987926F004B9CA
:1095800054D40020024B1B680121987926F0FCB8C6
:1095900054D40020F0B50E4693B0044658B125F0DF
:1095A000FBF9132805460DD02246574901202BF020
:1095B000D5FA002403E0554901202BF0CFFA2046CC
:1095C00013B0F0BD022105A81FF04EF805A88DF8D4
:1095D00019508DF81A601EF09BFF4D49002026F0AF
:1095E000F5F9002104469DF81A0025F0E1F9012162
:1095F0009DF81A0026F0C8F8464B474A1A61474AB8
:109600005A611A88920500D4FEE7454A9A61454A94
:10961000DA61454B01AA03F110071546186859682D
:10962000164603C60833BB423246F7D11AF068FE2D
:109630009DF804305AB2102A5EDC9DF805201344D0
:10964000DBB25AB2102A57DC9DF806201344DBB275
:109650005AB2102A50DC9DF8072013445BB2102B3D
:109660004ADC2E46032700251B2019F0D7FF16F8E9
:10967000013B07FA05F1AB4020EA01011943C9B2E9
:109680001B2002351AF06EF8082DEDD19DF8083038
:109690005AB2102A30DC9DF809201344DBB25AB2CA
:1096A000102A29DC9DF80A201344DBB25AB2102A92
:1096B00022DC9DF80B2013445BB2102B1CDC0DF157
:1096C0000706002503271A2019F0A8FF07FA05F15D
:1096D00020EA010116F8010FA8400143C9B21A207F
:1096E00002351AF03FF8082DEDD105A81EF0FCFE5A
:1096F0000E4B02221A7062E70D4824F0D9FB05A830
:109700001EF0F2FE55E700BF8A200600A7200600E3
:10971000DF200600B82C0020759502008595020018
:109720005D97020063970200FF02060058D40020F4
:10973000E820060010B5084C23680146587918F057
:1097400003F8002805DA23684FF0FF31587917F045
:10975000FBFFC0B210BD00BF54D40020FF20FFF7B4
:10976000E9BFFFF7E7BF1BF0EFB91BF001B900003D
:1097700038B5054609B11BF089F90022124928467F
:1097800030F0B2FF31F037FC10B1104830F04EFB32
:109790000446014628461BF079F95CB1E389A3F53C
:1097A00000739BB2E381E38903F4F05313B92046BD
:1097B0002FF080FC01202FF05DF805490246284675
:1097C000BDE8384030F057BF4F02060026B606000D
:1097D000261E060008B51BF059F9002008BD000040
:1097E00070B58EB0044601A80E4615461EF022FF45
:1097F000D8B1204600220E4930F076FF0446A0B1D1
:1098000032460C4930F016FF2A460B49204630F00C
:1098100011FFE389A3F500739BB2E381E38903F4AD
:10982000F05313B920462FF045FC0EB070BD00BFB9
:10983000521B0600561B0600651B060010B58EB0B5
:10984000044601A81EF0F6FE30B101A821461BF027
:1098500091FB01A81EF048FE0EB010BD38B50546BC
:1098600030F057FD04462FF068FAA0B92146184899
:109870002BF042F914B90024204638BDE389A3F542
:1098800000739BB2E381E38913F4F055F3D12046D2
:109890002FF010FCEFE75CB1E389A3F500739BB2F6
:1098A000E381E38903F4F05313B920462FF002FC5F
:1098B0000849002026F08AF804460028DCD001215F
:1098C0001EF094FD2A460449204630F0B3FED3E74B
:1098D0002A1E0600511E0600591E060038B5054610
:1098E00030F017FD04462FF028FAA0B92146184899
:1098F0002BF002F914B90024204638BDE389A3F502
:1099000000739BB2E381E38913F4F055F3D1204651
:109910002FF0D0FBEFE75CB1E389A3F500739BB2B6
:10992000E381E38903F4F05313B920462FF0C2FB1F
:109930000849002026F04AF804460028DCD000211F
:109940001EF054FD2A460449204630F073FED3E74A
:109950002A1E060090140600591E060030B591B06C
:10996000044603A80D461EF065FE48B1002303A877
:1099700000932A4621461BF097F903A81EF0B4FD78
:10998000002011B030BD30B58FB0044601A80D469F
:109990001EF050FE58B11DB129462046FFF7DEFFEC
:1099A00001A821461BF0E6FA01A81EF09DFD0FB0AC
:1099B00030BD000030B58FB0054601A81EF03AFE5C
:1099C00078B300211A481EF02BFD044630B3294617
:1099D00001A81BF027FB2946012220462EF04BFB55
:1099E000054600B30146204631F004FAEB89A3F5A1
:1099F00000739BB2EB81EB8903F4F05313B9284653
:109A00002FF058FBE389A3F500739BB2E381E38950
:109A100003F4F05313B920462FF04CFB01A81EF0BD
:109A200063FD0FB030BD03482BF046F8EAE700BFF6
:109A30004F1F0600551F06002DE9F04391B08146E7
:109A400003A8884616461F461EF0F4FDB8B1002153
:109A500018982EF085FC04462FF07FF980B330462D
:109A600030F078FC0646384630F074FC07461B2080
:109A70002EF0A0FE054628B903A81EF035FD11B052
:109A8000BDE8F0833B46324641462FF034FD0121CC
:109A900018982EF065FC26460746304630F05AFCF2
:109AA00080B200903B462A46494603A81BF0FCF8CA
:109AB0004545E1D03A463146284630F0F1FADBE739
:109AC0000CB94546E9E7E389A3F500739BB2E3814E
:109AD000E38903F4F053002BF3D120462FF0EAFA88
:109AE000EFE700002DE9F04F8BB0824601912FF097
:109AF000BFF920B9002630460BB0BDE8F08F02F068
:109B000035FF06460028F5D04FF000094FF0FF352D
:109B10000022514605A82AF03DFDCB462C46A8461A
:109B20002F464A464946DDE905308342C0F0D780DA
:109B3000089850B1C289A2F5007292B2C281C2895E
:109B400002F4F0520AB92FF0B5FAB4F1FF3F08BFA2
:109B50005C46B8F1FF3F08BFA046002F09DD7A1E22
:109B6000002150462FF00AFDBB490246304630F036
:109B700082FDBA4830F05AF9B9490246304630F011
:109B80007AFD791CA8EB010250462FF0F7FCB5498D
:109B90000246304630F06FFD6FF0004221465046DD
:109BA0002FF0ECFC07462FF014FE18B9AE493846EA
:109BB0002FF06DFD3A46AD49304630F05CFD691C32
:109BC00014BF2A1B6FF00042214650462FF0D6FCEE
:109BD00004462FF0FEFD18B9A34920462FF057FD8B
:109BE0002246A349304630F046FD6A1C00F0B98099
:109BF0006FF00042294650462FF0C0FC02469D49B6
:109C0000304630F038FD09F1FF324FF6FE739A42CC
:109C100040F2AB8002202EF0CDFD02469649304640
:109C200030F029FD6B1C00F0A4806FF00042691C2D
:109C300050462FF0A3FC019B0446002B49D02FF087
:109C400021F80546002844D10246214605A82AF0FD
:109C5000A1FC02F08BFE81461B202EF0ABFD0746D7
:109C60001B202EF0A7FD8046DDE905239A42C0F0B7
:109C70008480089850B1C389A3F500739BB2C38157
:109C8000C38903F4F0530BB92FF014FA5CB1E389E4
:109C9000A3F500739BB2E381E38903F4F05313B996
:109CA00020462FF007FA38462FF093FD002800F0E9
:109CB0009780384631F029FE414607462FF044FF91
:109CC0003946484630F0BCFB4146384630F014FA7D
:109CD0004C4622466949304630F0CDFC0BE70998E6
:109CE00088B1C05C2F2812D1B4F1FF3F08BF5C4699
:109CF000012A01F1010106D1022904D17B1C02D104
:109D00003D463C465F46B8F1FF3F0DD119E03A2889
:109D100007D17B1C02F10102F5D0631CF3D1D846B8
:109D20000FE0B8F1FF3F16D0D84514DA631C40F0BD
:109D300090802F2805D9392803D830380A2303FB0F
:109D4000090905A8CDE902210BF1010B2AF0FCF865
:109D5000DDE90221E7E63F28F3D1601CF1D05D4642
:109D6000EFE702202EF026FD48E748462EF08AFD58
:109D700053E702202EF01EFD5DE7099B002B53D018
:109D80009B5C262B25D138462FF023FDC0B13846E9
:109D900031F0BBFD414605462FF0D6FE2946484628
:109DA00030F04EFB4146284630F0A6F91B202EF03D
:109DB00001FD07461B202EF0FDFC8046002504E037
:109DC00040462FF006FD0028E1D105A82AF0BCF896
:109DD0004AE765B93D2B31D1019DF6E7824611E096
:109DE00040462FF0F6FC00287FF463AF6CE7252B8C
:109DF0001BD105A82AF0A8F809980028EED0059BE9
:109E000010F803A005A82AF09FF8504629F073FE29
:109E100000014FFA80FA099808B1059BC05C29F04F
:109E20006AFE4AEA0000C3B255B101220DF11301E6
:109E300040468DF813302FF007FCCDE7252BD8D006
:109E400001220DF1130138468DF813302FF0FCFB81
:109E5000B4E73F2883D074E7562006005F20060051
:109E60006320060015140600CF1F06006A200600B6
:109E70006F200600782006007F2006008420060060
:109E800070B58EB004460D460146684616461FF072
:109E90003BF878B13246294668461EF0BBFD68465D
:109EA0001EF0F8FFE38903F500739BB2E3812046BF
:109EB0000EB070BD0446FAE730B58FB00D460146CE
:109EC00068461FF021F800284CD0BDF91B20BDF9D1
:109ED0001F309A4244DC02F049FD044618B3BDF934
:109EE0001B002EF0CFFC20490246204630F0C3FB79
:109EF000BDF91D002EF0C6FC1C490246204630F07C
:109F0000BAFBBDF91F002EF0BDFC194902462046E0
:109F100030F0B1FBBDF921002EF0B4FC154902462A
:109F2000204630F0A8FBC5B100226FF07F038DF80A
:109F30001F208DF820308DF821208DF822304FF031
:109F4000FF327F2368468DF81B208DF81C308DF87A
:109F50001D208DF81E301EF09DFF20460FB030BD35
:109F60000024E0E70446F8E7931D0600961D06006E
:109F7000991D06009C1D060070B58EB004460D4666
:109F80000146684616461EF0BFFF50B3BDF80530C7
:109F9000022D23F070039BB21DD0032D1ED0012D86
:109FA00008BF43F03003ADF805304EB1BDF80530C1
:109FB000DA064CBF83F0400383F02003ADF8053090
:109FC00068461EF067FFE38903F500739BB2E381E7
:109FD00020460EB070BD43F06003E4E743F0500349
:109FE000E1E70446F4E770B58EB004460E4601463C
:109FF000684615461EF088FF70B16846ADF81660D9
:10A00000ADF818501EF046FFE38903F500739BB2CC
:10A01000E38120460EB070BD0446FAE7F0B58FB07C
:10A0200004460E460146684615461F461EF06CFF64
:10A0300000B3012E9DF81A10A8BF0126012DA8BF5C
:10A04000012546EAE67666F3010145EAE57565F322
:10A05000830187F3020767F3051168468DF81A102C
:10A060001EF018FFE38903F500739BB2E3812046DD
:10A070000FB0F0BD0446FAE72DE9F0438FB0044677
:10A0800088460146684616461D46169F1EF03CFF50
:10A09000002846D040462EF0EBFE40B92249012070
:10A0A0002AF05CFD002420460FB0BDE8F083FF2EAF
:10A0B00001D91E49F3E728462EF0DAFE28B92846D2
:10A0C0002EF095FF08B91A49E9E77B1EFE2B01D94E
:10A0D0001849E4E742461849204630F0ABFA2A46D0
:10A0E0001649204630F0A6FA38462EF0CBFB14492C
:10A0F0000246204630F0BFFA30462EF0C3FB11492D
:10A100000246204630F0B7FA4FF6FE736846ADF8C7
:10A1100014301EF0BFFEE38903F500739BB2E381A8
:10A12000C1E70446BFE700BF9F1D0600BC1D060037
:10A13000D91D0600031E0600121E0600171E06008B
:10A140001C1E0600211E06002DE9F04F93B00146AB
:10A1500004A81EF0D9FE28B94FF0000B584613B0E2
:10A16000BDE8F08F9DF81B80B8F1010F07D0B8F162
:10A17000180F04D04B4901202AF0F0FCECE7BDF8A1
:10A180001530BDF81950BDF81760DB0642BF2B46ED
:10A1900035461E4606FB08F31F33B8F1010F4FEAA0
:10A1A00063134FEA83030CBF20271A2703FB0579AB
:10A1B000484600932EF0EEFB83460028CCD02EF0CC
:10A1C000EEFD422303704D2343700C23837333123F
:10A1D00080F80290C3744FEA29292B12877280F805
:10A1E000039043750123B8F1010F83759DF81B306F
:10A1F0000376009A867401BFFF238376C3760377C4
:10A200006B1E0446057502FB03774FF000084545B9
:10A21000A4D09DF81B30012B3BD04FF000090FFA62
:10A2200088FAB14530D052460FFA89F104A81EF0E1
:10A23000FDFD9DF81B30DB0809FB0373020AE054A7
:10A240002344000C5A70987009F10109E9E70023D2
:10A250005B000FFA89F1019A039304A81EF0E6FD52
:10A2600009F10109039B00F00100CA4543EA00031C
:10A27000EED1029A02EBEA020AF1080A02F8013C66
:10A28000AAF10809B145E2DB009B08F10108FF1AB9
:10A29000BDE70FFA88F30193E3194FF0080A029320
:10A2A000EEE700BF291C060038B5FFF74DFF054655
:10A2B00010B90025284638BD0BF0A8FCEB89A3F5A2
:10A2C00000739BB2EB81EB8903F4F053044613B99E
:10A2D00028462EF0EFFE002CEBD0214608482FF048
:10A2E0005DF9E389A3F500739BB2E381E38903F48D
:10A2F000F0530546002BDDD120462EF0DBFED9E7DA
:10A30000571C060010B5FFF7CFFF044668B123F0D5
:10A31000CBFDE389A3F500739BB2E381E38903F4EA
:10A32000F05313B920462EF0C5FE0248BDE8104098
:10A3300023F0BEBD25B6060030B58FB00C460146F1
:10A34000684615461EF0E0FD20B12AB221B26846EB
:10A350001EF06CFD0FB030BDF0B58FB004460E4658
:10A360000146684615461F461EF0CEFDE0B1B7B95E
:10A37000039B36B22DB22A46314668461EF076FD62
:10A380006846ADF81660ADF818501EF083FDE389FD
:10A3900003F500739BB2E38120460FB0F0BD384651
:10A3A0002FF0D8FF0346E4E70446F5E72DE9F04F28
:10A3B0009DB004460D4601460EA8CDE905231EF0CA
:10A3C000A3FD20B9002420461DB0BDE8F08F28462B
:10A3D0002EF09BFC20B9764901202AF0BFFBF1E763
:10A3E00000227449284630F07FF930F0EFFC00225B
:10A3F00071490290284630F077F930F0E7FC0022EE
:10A400006E490090284630F06FF930F0DFFC0022F2
:10A4100001906B49284630F067F980462FF09AFF8B
:10A420000390B8F1000F0ED0B8F80E30A3F500730A
:10A430009BB2A8F80E30B8F80E3003F4F05313B9FD
:10A4400040462EF037FE284600225E4930F04CF997
:10A4500005462EF036FCA8B1029B002B18DC5A49A9
:10A4600001202AF07BFB002DACD0EB89A3F5007313
:10A470009BB2EB81EC8914F4F054A3D128462EF062
:10A4800019FEA0E728462EF0F3FC0028E4D1E6E709
:10A49000009B002BE3DD019B202BE0DC28462EF007
:10A4A0005BFF07465DB1EB89A3F500739BB2EB81BF
:10A4B000EB8903F4F05313B928462EF0FBFD019B02
:10A4C000012BB8BF01239B4609AB00221846394631
:10A4D0002AF060F8012202FA0BF2531E00250493C1
:10A4E00009AB2E46A946AA4607935E455BDADDE92D
:10A4F00009239A4202D2009B994522DB0C9850B165
:10A50000C389A3F500739BB2C381C38903F4F053DD
:10A510000BB92EF0CFFD5FB1FB89A3F500739BB2A1
:10A52000FB81FB8903F4F05313B938462EF0C2FDCA
:10A530000EA81EF0AFFCE38903F500739BB2E38124
:10A5400041E72B020D9D0DB1099AAD5C07980836C5
:10A550001D4329F0F9FCB345F3DCA6EB0B06049A86
:10A5600025FA06F31340B8F1000F02D0039A9A427D
:10A570000DD0019A012A01DC9BB1119B069A059925
:10A580004A44514412B209B20EA81EF06FFC029B5D
:10A590000AF1010A5345DCBF09F101094FF0000A35
:10A5A000A3E7129BEAE7009B9945D6DBA6E700BF2D
:10A5B000F61C06001F1D06000B1E0600251D0600CA
:10A5C000291D060044430600351D0600F0B5DBB02A
:10A5D00004460D4601460CA81EF096FC18B900244E
:10A5E00020465BB0F0BD28462EF06DFC0028F6D06A
:10A5F0002946012201A82BF0BEFC1AAE00253746E1
:10A6000001A829F0CEFB08B1802D16D101A829F0B0
:10A6100089FB802D03D140210D482AF04DFA3A469E
:10A6200069100CA81EF062FA0CA81EF033FCE38936
:10A6300003F500739BB2E381D2E701A829F0A9FDDD
:10A6400026F8020B01A8013529F0DEFCD8E700BF8F
:10A650005F1D06002DE9F04F9FB004460E460146EF
:10A6600010A803921EF050FC20B9002420461FB011
:10A67000BDE8F08F30462EF026FC0028F5D031469C
:10A68000012205A82BF077FC002605A829F089FBFC
:10A69000C0B905A829F046FB039B53B12DB2009524
:10A6A0000FFA8AF3BDF95820BDF9561010A81EF014
:10A6B00023FB10A81EF0EEFBE38903F500739BB2A9
:10A6C000E381D3E705A829F064FDF307834616D597
:10A6D000012E0FFA87F90FFA80F816D0CDF8008016
:10A6E0004B46BDF95820BDF9561010A81EF004FBCA
:10A6F000AB465D46ADF85690ADF85880BB4605A810
:10A70000013629F081FC5F46BFE7BA46F1E770B534
:10A7100090B004460E46014602A815461EF0F4FB12
:10A72000C8B136B22DB23346BDF92020BDF91E1096
:10A73000009502A81EF0E0FA02A8ADF81E60ADF880
:10A7400020501EF0A7FBE38903F500739BB2E38161
:10A75000204610B070BD0446FAE7F0B591B004464B
:10A760000D46014602A816461F461EF0CDFB98B1C5
:10A77000BDF95830009332B23BB229B202A81EF0A4
:10A78000BBFA02A81EF086FBE38903F500739BB2B7
:10A79000E381204611B0F0BD0446FAE72DE9F04F01
:10A7A00095B004460D46014606A81EF0ADFB0028F4
:10A7B00039D0BDF92C30023338D100223749204638
:10A7C0002FF092FF00223649064620462FF08CFFDC
:10A7D00030F0FCFA8046284630F068FC0022014642
:10A7E000814601A829F0D6FE0027DFF8B8A03C4634
:10A7F0004FF0C00BDDE9013293421BD3049850B1F6
:10A80000C389A3F500739BB2C381C38903F4F053DA
:10A810000BB92EF04FFC484631462FF06DFCBC4280
:10A820002046B8BF384615B0BDE8F08F4FF000089D
:10A830004646D0E7059D35B1ED5C0A2D03D1A74210
:10A84000B8BF27460024BDF92C20002A0FDD203D8B
:10A85000EBB25E2B97BF1AF81530002313FB02F3FF
:10A86000B3FBFBF31C4401A829F06EFBC2E7531CA9
:10A8700001D10434F7E70232F5D130462EF0F8FA70
:10A8800040B14545EFDBA5EB080130462EF012FE46
:10A890000444E8E730462FF05DFDF9E7171E060097
:10A8A000211E0600653506002DE9F04FA5B000AF6A
:10A8B0000D46F862014607F15800BA621C461EF0C8
:10A8C00023FB002800F01F82B7F96C30002B05DD58
:10A8D0007B624FF0000BC7E907BB21E05E1C00F074
:10A8E0008380023340F085800022A849F86A2FF067
:10A8F000FBFE0022F861A649F86A2FF0F5FE00225F
:10A90000A4493862F86A2FF0EFFE30F05FFA0022B7
:10A910007862A149F86A2FF0E7FE30F057FA8346D3
:10A9200097F87220B7F85D303B8102F030011029B2
:10A930009BB263D183F03003A7F85D30BB6AB7F8F0
:10A940005F10BC620133CC1A02F00302012A0FD857
:10A950002946F86AFFF722FF97F8723003F00303E5
:10A9600003FB0000BB6A00EBD070A3EB6003BB628B
:10A9700097F87230C3F38102012A08D87A6A03F08B
:10A98000030303FB022303EBD373A4EB6304B7F8C5
:10A990005F307B61B7F86130BB61B7F85D30D806D6
:10A9A00048BFD7E90523284648BFC7E9053230F03C
:10A9B0007DFB0022F860014607F1300029F0EAFD36
:10A9C000BD6AD7E90C239A4280F0A3803B6C9BB30D
:10A9D00013F80290B9F10A0F2FD17B6A07F130000A
:10A9E0001C4429F0B1FAEBE706234FF0000B7B6221
:10A9F00071E74FF0000BC7F824B06CE720290ED1A7
:10AA000083F06003A7F85D30BB6AB7F85F100133CD
:10AA1000CB1ABB62B7F8613001341C1B94E73029B4
:10AA200092D183F05003B7F86110A7F85D30631C32
:10AA3000CB1ABC6ABB6287E79946B7F96C80B8F15C
:10AA4000000F40F38C80A9F120095FFA89F25E2A99
:10AA50009BBF524B13F81930002313FB08F39CBF24
:10AA6000C021B3FBF1F33B613B695B42AB4249DA86
:10AA70007B699D4246DAC8F10003A34242DABB6912
:10AA80009C423FDA5E2A3DD8002244491646914551
:10AA90005BDC01EB4901C7F800D04B787B60404B91
:10AAA00088B000201E44EA46814660237A689145BA
:10AAB00026DA327896F801C04FF0300E02F07F02AD
:10AAC00018FB02E2B2FBF3F22A442AF810200AEB48
:10AAD00040010CF07F0218FB02E21CF0800FB2FB79
:10AAE000F3F222444A8000F1020034D04110524671
:10AAF00007F158001DF0FAFF28F082FE602350B3E2
:10AB0000D7F800D03B691D4428F07AFE002800F0F9
:10AB1000E780F86B002840F0E880D7E90712F86872
:10AB20002FF0BEFA3B89A7F85D3007F158001EF000
:10AB3000B1F9FB6AFA6ADB8903F500739BB2D38132
:10AB4000F86A9437BD46BDE8F08F01EB420301324D
:10AB50005B781E449BE709F102090236A6E7B8F1CB
:10AB6000FF3F1FD1E91C0EDB7B699D420BDA621DA2
:10AB700009DBBB699C4206DA4B4622B229B207F1D7
:10AB800058001EF099FA0435BEE700BF121E0600F9
:10AB9000171E06001C1E0600211E06006535060055
:10ABA0004921060018F1020FAED1386A2EF060F983
:10ABB00000285DD0CB4500F3918007F144060022C8
:10ABC000396A304629F0E6FC4FF00008A9EB0B0982
:10ABD000786CBB6C796D984203D2FA6C02444A459A
:10ABE0003DDB002942D00E5C386D50B1C389A3F51E
:10ABF00000739BB2C381C38903F4F0530BB92EF0E9
:10AC000059FA7342AB423DDA7B699D423ADA7B6A7C
:10AC10005B42A34236DABB699C4233DA7B6AF9694C
:10AC200008FB03F807F1440A4FEAD802504629F01E
:10AC3000B1FC08F007084FF00009C7F804A0B145BF
:10AC400045DB386DF0B1C389A3F500739BB2C381B6
:10AC5000C38903F4F053ABB92EF02CFA12E001B122
:10AC6000095C3046884429F06FF9B1E70E46BBE72E
:10AC7000386A2FF06FFBA9EB0B08CB45064600FBAB
:10AC800008F8BEDD35443FE77B6D73B17A6C9B5CA1
:10AC900003FA08F31B0608D50AEB04027B6E396938
:10ACA00012B207F158001EF0E1F808F10108B8F1FE
:10ACB000080F04D1786829F047F94FF000080AF12D
:10ACC000010A7B6A5345DFDC09F10109B7E709EBAB
:10ACD00005031BB24FF0000A3B61F2E70026D1E703
:10ACE00007F1300029F030F96BE6C389A3F5007352
:10ACF0009BB2C381C38903F4F053002B7FF40DAFE3
:10AD00002EF0D8F909E7F8621AE700BF2DE9F04FF5
:10AD10009DB00EAD03900F460146284616461C46D0
:10AD20001EF0F2F8002800F0C680269BADF8363001
:10AD30000DF132020CA92846ADF83070ADF8344060
:10AD4000ADF832601DF046FE0DF136020DA9284621
:10AD50001DF040FEBDF93040BDF93420BDF9320090
:10AD6000A31803EBD3734FEA630ABDF93630C11859
:10AD7000121B01EBD1711B1A491002EBD274641043
:10AD80000491013203EBD371B8BF64424FEA610B07
:10AD90000133B8BFCBF1000B0BFB0BF30793079A02
:10ADA00004FB04F3089353430B93049A119BAAEBFF
:10ADB000040128461DF06AFD119B049A0AEB040168
:10ADC00028461DF063FD002301270993BB450DDADA
:10ADD0000EA81EF05FF8039B039ADB8903F500734E
:10ADE0009BB2D38103981DB0BDE8F08F099B089AF0
:10ADF0005E1E07FB07F3A61B5343002E2BDCA31B91
:10AE00000993AAEB06030593049BA3EB07090AEB3E
:10AE100006030693049B03EB0708A31B012B24DC0A
:10AE2000119B05994A4628461DF030FD119B069955
:10AE30004A4628461DF02AFD119B059942462846A0
:10AE40001DF024FD119B0699424628461DF01EFD6B
:10AE500001373446BAE7079906FB06F201FB0232D6
:10AE60000B999142CBDA013EC7E7AAEB04035444A5
:10AE700001334A460599CDF800902846013C0A93D3
:10AE80001DF0A2FC23464A460699CDF800902846BC
:10AE90001DF09AFC0A9B0599CDF800804246284691
:10AEA0001DF092FCCDF800802346424606992846C4
:10AEB0001DF08AFCCCE7039094E737B505461C46A5
:10AEC00013440093121B0B19091BFFF71FFFEB899B
:10AED00003F500739BB22846EB8103B030BD2DE92A
:10AEE000F04F99B00AAC81460F46014620461646FF
:10AEF0001D461EF009F8002800F08980229BADF85D
:10AF000026300DF1220208A92046ADF82070ADF8D8
:10AF10002260ADF824501DF05DFD0DF1260209A957
:10AF200020461DF057FDBDF92000BDF92420BDF9D4
:10AF30002210BDF926308518121ACE1802EBD27AEB
:10AF40005B1A4FEA6A0A013203EBD378B8BFCAF141
:10AF5000000A4FEA68080133B8BFC8F1000808FBCF
:10AF600008F30393039A0AFB0AF305EBD57506EB86
:10AF7000D6766D107610049353430793009605EB35
:10AF80000A033246A5EB0A0120461DF01DFC0023F2
:10AF9000CDE905340127B8450DDA0AA81DF07AFF7E
:10AFA000B9F80E3003F500739BB2A9F80E3048468D
:10AFB00019B0BDE8F08F059B049A5C1E07FB07F3F0
:10AFC000AAEB04045343002C17DCF21BAAEB040386
:10AFD00005EB040BA5EB040A5146059300925B4672
:10AFE00006981DF0F1FBF219514600925B46069857
:10AFF0001DF0EAFB0137A246CDE7039904FB04F2FA
:10B0000001FB023207999142DFDA013CDBE781461E
:10B01000CDE737B505461C4613440093121B0B19A8
:10B02000091BFFF75CFFEB8903F500739BB2284611
:10B03000EB8103B030BDF0B593B004460F46014636
:10B0400004A816461D461DF05FFF002849D0189B36
:10B05000ADF80E300DF10A0202A904A8ADF808708F
:10B06000ADF80A60ADF80C501DF0B4FC0DF10E0205
:10B0700003A904A81DF0AEFCBDF90A200092BDF999
:10B080000C30BDF9081004A81DF09EFBBDF90C3072
:10B09000BDF90E2000921946BDF90A2004A81DF042
:10B0A00093FBBDF90E200092BDF90C30BDF90810DC
:10B0B00004A81DF089FBBDF90830BDF90A200092F3
:10B0C0001946BDF90E2004A81DF07EFB04A81DF052
:10B0D000E1FEE38903F500739BB2E381204613B0E0
:10B0E000F0BD0446FAE7F0B591B004460D460146BE
:10B0F00002A816461F461DF007FF98B1BDF958304B
:10B10000009332B23BB229B202A81DF071FE02A830
:10B110001DF0C0FEE38903F500739BB2E381204676
:10B1200011B0F0BD0446FAE730B58FB004460D46C5
:10B13000014668461DF0E8FE00B38DB100234FF0D4
:10B14000FF32CDE90323ADF818309DF81A3023F013
:10B150003F034FF6FF7243F00F0305928DF81A304C
:10B1600068461DF07EFB68461DF094FEE38903F5FA
:10B1700000739BB2E38120460FB030BD0446FAE76E
:10B180002DE9F0478AB080462DF072FE044638B9AA
:10B190006149032029F0E2FC20460AB0BDE8F087AF
:10B1A00000224146684629F0F5F900273C463E4614
:10B1B000B9463D46DDE90032934212D3039850B1BF
:10B1C000C389A3F500739BB2C381C38903F4F05311
:10B1D0000BB92DF06FFF01F0C9FB0546D8B900246B
:10B1E000DAE7049A6AB1D35C0A2B0AD155EA09035B
:10B1F00008BF012709F101090025684628F0A4FECF
:10B20000D8E7A14505F10105A8BF09F10104AE4247
:10B21000B8BF2E46F1E730462DF034FB3F490246D9
:10B2200028462FF028FA20462DF02CFB3C490246F8
:10B2300028462FF020FA04FB06F007300021C0104A
:10B240002EF08EFD044668B9EB89A3F500739BB21E
:10B25000EB81EB8903F4F053002BC0D128462DF08D
:10B2600029FF99E73A464146684629F093F94FF09D
:10B27000000847464FF08009DDE90032934213D3BE
:10B28000039850B1C389A3F500739BB2C381C389EE
:10B2900003F4F0530BB92DF00DFF22462149284647
:10B2A0002FF0E9F92C4677E7049A5AB1D35C0A2BC0
:10B2B00006D108F101080027684628F045FEDBE7C3
:10B2C000202B26D020462DF0D3FD10B306FB087AA4
:10B2D00021464FEADA0205A829F05CF9099909B17B
:10B2E000059BC95C0AF0070A49FA0AFA41EA0A0111
:10B2F00005A8C9B229F006F8089850B1C389A3F58A
:10B3000000739BB2C381C38903F4F0530BB92DF0D2
:10B31000D1FE0137D0E700BFE31C06001F1D060069
:10B320000B1E0600444306002DE9F04316461D4659
:10B33000421E47F6FE739A428FB080460F4602D8EF
:10B340004A1E9A4208D93349012029F007FC0024FB
:10B3500020460FB0BDE8F083304604F085FD04467A
:10B3600020B92D49012029F0F9FBF1E728462DF0FD
:10B37000CCFCD8B10022294928462FF0B5F900228B
:10B380000446274928462FF0AFF92546814628462E
:10B390002DF0D3FC044680B92A462249012029F029
:10B3A000DDFB494628462EF0A7FED1E7EB8903F5E1
:10B3B00000739BB2EB818146E9E7B9F1000F06D03B
:10B3C00048462DF0BAFC044608B94A46E5E7164956
:10B3D000002024F0FBFA04460028B9D068461DF08E
:10B3E00043FE01232A4611498DF80430204600947B
:10B3F000ADF80780ADF809708DF80B602FF01AF9E1
:10B400004A460B4900982FF015F968461DF042FD99
:10B41000C7E700BF701C06007D1C0600891C0600E3
:10B42000921C06009B1C06004E1C0600CF1C06004A
:10B43000D91C06002DE9F0439DB000AF00230E4655
:10B4400007F108018046BB602EF020FA0546F8B9E6
:10B4500040462AF071FF0446B86028F0F5F904F57B
:10B460008073834209D96149012029F077FBA846FE
:10B4700040467437BD46BDE8F083E31D23F0070363
:10B48000ADEB030D6D462246294640462AF044FFA7
:10B49000012E01D1142000E0F0104FF00009391DF9
:10B4A000C7F80490F5F730FD7C68804624B9504811
:10B4B00029F022FBA046DBE7012E78D15C22494629
:10B4C00007F11400BE68F4F72DF84A4BFB6103F155
:10B4D00088333B6203F12943A3F59613A3F68B63EC
:10B4E0007B62A3F18833BB62434BFB622EB13246D1
:10B4F000294607F1140017F063FE7A69B969530F02
:10B5000043EAC1031BBAFB60D30002F03F02372AB3
:10B510001BBA94BFC2F13802C2F1780237493B61CD
:10B5200007F1140017F04CFE082207F10C0107F197
:10B53000140017F045FEFB7F2370FB8B6370FB69E3
:10B540001B0AA370FB69E37097F8233023717B8C8F
:10B5500063713B6A1B0AA3713B6AE37197F827305A
:10B560002372FB8C63727B6A1B0AA3727B6AE37291
:10B5700097F82B3023737B8D6373BB6A1B0AA3730D
:10B58000BB6AE37397F82F302374FB8D6374FB6AF7
:10B590001B0AA374FB6AE37400231A4607F1140123
:10B5A000194401335D2B3FF463AF0A70F6E7E02ED8
:10B5B00006D101232246B968284617F037FD57E720
:10B5C000B6F5807F01D14B46F4E7B6F5C07F06D1D2
:10B5D00001232246B968284617F096FB48E7B6F5DE
:10B5E000007F7FF445AF4B46F3E700BF4D010600F7
:10B5F000CE1A060001234567F0E1D2C304210600FC
:10B60000024B0349586800222FF06EB88C2D0020A1
:10B610004B14060010B51D4C2378834206D0024619
:10B620001B490420BDE8104029F098BA002323707C
:10B63000184C206890B129B3114603F01DFD206815
:10B6400050B1C389A3F500739BB2C381C38903F4CE
:10B65000F0530BB92DF02EFD002323600E4C206813
:10B6600050B1C389A3F500739BB2C381C38903F4AE
:10B67000F0530BB92DF01EFD00232360074B012270
:10B680001A7010BD114603F057FDD8E73CD40020D6
:10B690001A14060034D4002040D4002045D40020E1
:10B6A00010B50A460C460021FFF7B4FF6CB1E389E0
:10B6B000A3F500739BB2E381E38903F4F05323B94C
:10B6C0002046BDE810402DF0F5BC10BD10B5094B6B
:10B6D0001C78012C0CD100210846FCF739F80648EB
:10B6E0002EF0A4FB01462046BDE81040FFF7D8BF6E
:10B6F00010BD00BF3CD40020A81606000A46002159
:10B70000FFF788BF73B50022414905462EF0ECFFD4
:10B710002FF05CFB3F4B40490646032258682EF051
:10B72000E3FF044678B12A46B1B22CF09BFDE389D1
:10B73000A3F500739BB2E381E38903F4F05313B9DB
:10B7400020462DF0B7FC0022344928462EF0CCFFCD
:10B750002FF03CFB80B2002846D129460820FDF797
:10B760000BF918B90024204602B070BD2C4B1C68A0
:10B7700024B1E38903F500739BB2E381294E33883A
:10B780004FF6FF729A4207D127482EF04FFB014631
:10B790000820FFF785FFE6E700221D4928462EF026
:10B7A000A3FF2FF013FB013080B2ADF80400ADF819
:10B7B000060001A9308810F0A1FD0FF02DF9054613
:10B7C0000028D0D001460820FFF798FFEB89A3F5A9
:10B7D00000739BB2EB81EB8903F4F053002BC2D1D1
:10B7E00028462DF067FCBEE700210920FDF7C4F8CC
:10B7F0000028B7D00A4B1C6824B1E38903F5007315
:10B800009BB2E3810121284610F024F8ABE700BF8A
:10B81000C31406008C2D0020D0140600A9140600C5
:10B8200034D40020E22C0020B514060070B5014687
:10B8300006460720FDF7A0F800283AD01E4B1C68EA
:10B8400024B1E38903F500739BB2E3811B4D2B8880
:10B850004FF6FF729A4208D119482EF0E7FA0146D6
:10B860000720FFF71DFF204670BD00221549304616
:10B870002EF03AFF2FF0AAFA2B8881B20022184648
:10B8800010F03AFD0FF0C8F805460028EBD001464D
:10B890000720FFF733FFEB89A3F500739BB2EB8121
:10B8A000EB8903F4F053002BDDD128462DF002FC88
:10B8B000D9E70446D7E700BF34D40020E22C0020AB
:10B8C000B5140600C31406002DE9F04F85B0884674
:10B8D00000AF00230646394640463B602DF0D6FFB8
:10B8E0000546F8B940462AF027FD0446386027F09F
:10B8F000ABFF04F58073834209D94249012029F046
:10B900002DF92C4620461437BD46BDE8F08FE31DC7
:10B9100023F00703ADEB030D6D4622462946404652
:10B920002AF0FAFC00210620FDF726F808B90446A3
:10B93000E8E7354B1C6824B1E38903F500739BB23B
:10B94000E381324B1A884FF6FF719142984607D136
:10B950002F482EF06BFA01460620FFF7A1FED1E733
:10B9600000222C49D7F8009030462EF0BDFE2FF073
:10B970002DFA00221FFA80FA274930462EF0B4FE35
:10B98000064600283CD0002224492EF0ADFE2FF0C0
:10B9900032FBF389A3F500739BB2F381F38903F4BF
:10B9A000F053834613B930462DF084FB00239B45AA
:10B9B0003B8114BF022301233B71391D0123B8F8D9
:10B9C00000007B71FD60A7F806A0A7F80A900FF0B1
:10B9D0003FFF0FF021F80546002893D001460620CE
:10B9E000FFF78CFEEB89A3F500739BB2EB81EB892B
:10B9F00003F4F053002B85D128462DF05BFB81E743
:10BA00008346D3E74D01060034D40020E22C002009
:10BA1000B5140600C3140600D7140600E21406008D
:10BA200038B50D4601460A20FCF7A6FF002839D09C
:10BA30001D4B1C6824B1E38903F500739BB2E381BD
:10BA40001A4B1A884FF6FF71914208D118482EF010
:10BA5000EDF901460A20FFF723FE204638BD18887D
:10BA6000144B1B7880B2DBB100232A461946F8F745
:10BA7000E1FD0EF0D1FF05460028EED001460A2078
:10BA8000FFF73CFEEB89A3F500739BB2EB81EB89DA
:10BA900003F4F053002BE0D128462DF00BFBDCE73C
:10BAA0000820E6E70446D8E734D40020E22C002042
:10BAB000B5140600ECCD0020F0B58BB06D460C46F9
:10BAC000294617F0CDFC002800F08D8000220123CC
:10BAD00095E80300ADF818208DF81830A023ADF8D4
:10BAE0001A30454BADF80C10CDE90732434B0290AC
:10BAF000090C58688DF80E10414909922EF0F4FD9A
:10BB00002FF064F9C3074CBF3E4B3F4B08932046D0
:10BB10004FF0C87309932DF0F8F8002841D00022A7
:10BB20003A4920462EF0E0FD2FF09CFC02460B46E1
:10BB300006460F4633F0B4FF90B90022344B30462E
:10BB4000394633F013FD2AA3D3E9002333F038FE3E
:10BB50000022304B33F054FB33F0E0FFADF820000F
:10BB600000222D4920462EF0BFFD2FF07BFC02461F
:10BB70000B4604460D4633F093FF90B90022244B48
:10BB80002046294633F0F2FC19A3D3E9002333F011
:10BB900017FE00221F4B33F033FB33F0BFFFADF82D
:10BBA000220002AB93E80300ADF81410090C0490D6
:10BBB0008DF8161008AA06A904A810F0A1FB0EF033
:10BBC0002BFF044678B101460220FFF797FDE38979
:10BBD000A3F500739BB2E381E38903F4F05313B937
:10BBE00020462DF067FA0BB0F0BD00BFAFF3008028
:10BBF0000000000000889340900004008C2D00207D
:10BC00000E180600900120031000A000F617060091
:10BC100000408F400000E03F021806000A46012164
:10BC2000FFF7F8BC38B5124B1C78012C05461DD126
:10BC300000210846FBF78CFD21460E482CF076FECD
:10BC4000044609F095FC5CB1E389A3F500739BB24F
:10BC5000E381E38903F4F05313B920462DF02AFA67
:10BC600029460120BDE83840FFF7D8BF38BD00BFE6
:10BC70003CD4002040D400207CDF70472DE9F04FF9
:10BC8000AC4D85B02B6800AF044603F004030846B2
:10BC90000E463B602DF039F8002800F0BC800022F1
:10BCA000A54930462EF020FDB0B12FF08FF84FF4AB
:10BCB0007A73584340F2712390FBF3F080B2B0F5F1
:10BCC000804F9E4B28BF4FF4804020281A8838BFF1
:10BCD0002020824218BF18800022994930462EF059
:10BCE00003FD38B12FF087F92B68002875D023F4B5
:10BCF00000632B600022934930462EF0F5FC38B1EA
:10BD00002FF079F92B6800286AD023F480532B6038
:10BD100000228D4930462EF0E7FC8146002800F0D5
:10BD20008480002307F10C01FB602DF0AFFD8046FD
:10BD3000002864D148462AF0FFFA8246F86027F0CE
:10BD400083FD0AF5807383424DD98049012028F094
:10BD500005FFB9F80E30A3F500739BB2A9F80E30B9
:10BD6000B9F80E3003F4F05313B948462DF0A2F998
:10BD700020462CF0CAFF824608B9002C58D1314623
:10BD80002046FCF767FB002C40F0D2800024704D69
:10BD90007049686822462FF0B3F832466E496868E9
:10BDA0002FF0AEF85CB1E389A3F500739BB2E38199
:10BDB000E38903F4F05313B920462DF07BF93B6877
:10BDC0000BB10EF011FE40460EF00CFF3B6843B382
:10BDD0000FF028FA0EF006FF23E043F4006388E733
:10BDE00043F4805393E70AF1070323F00703ADEB15
:10BDF000030DE8465246414648462AF08DFA112383
:10BE00004146BA893B7207F10800FFF735FF8046CB
:10BE10000EF0E8FE9DE746B132465049032028F077
:10BE20009DFE1437BD46BDE8F08F4FF000089FE738
:10BE300020462CF062FF7860002868D0E38903F583
:10BE400000739BB2E3812B6823F47F0323F4004348
:10BE5000214607F10C002B6027F0F3FFD346F8686A
:10BE600050B9BAF1000F92D0BBF1010F8FDD2B68F2
:10BE700043F400432B608AE72EF04BFA81462CF006
:10BE800044FF10B9B9F1000F1ED131464846FCF706
:10BE9000E1FA8246F86810B151462EF033F8BAF153
:10BEA000000F0ED0BAF80E30A3F500739BB2AAF8BB
:10BEB0000E30BAF80E3003F4F05313B950462DF09B
:10BEC000F9F8D7F804A009E048462CF016FF00283E
:10BED000F7D148462CF0F5FE0028F2D10BF1010B0A
:10BEE000B9F1000F0ED0B9F80E30A3F500739BB274
:10BEF000A9F80E30B9F80E3003F4F05313B94846E0
:10BF00002DF0D8F807F10C0027F086FFA7E72046B0
:10BF10002CF0D7FE00283FF439AFE38903F5007316
:10BF20009BB2E3812B6823F47F0323F40043A1E752
:10BF300004462CE738D40020BE170600E02C002071
:10BF4000C7170600D3170600732006004D01060030
:10BF50008C2D0020DD170600E717060029160600C5
:10BF600072DF7047F0B5264B264983B0044600AF18
:10BF7000024658682EF0C4FF20462CF0BEFEE8B101
:10BF80000023391D20467B602DF080FC054668BBF0
:10BF900020462AF0D1F90646786027F055FC06F5D0
:10BFA0008073834217D91849012028F0D7FD17491B
:10BFB000032028F0D3FD0C37BD46F0BD20462CF001
:10BFC00080FE0028DCD1002CF5D022461049032049
:10BFD00028F0C4FDEFE7F31D23F00703ADEB030DDD
:10BFE0006D463246294620462AF096F900213B79D3
:10BFF0002A460846FFF7B4FF0EF0F4FDDBE700BF6A
:10C000008C2D00207C1806004D01060085180600C6
:10C01000B118060070B5384C3849206800222EF05F
:10C0200063FB054678B1002101200EF0B3FCEB89DB
:10C03000A3F500739BB2EB81EB8903F4F05313B9C2
:10C0400028462DF037F800222D4920682EF04CFBB1
:10C05000054670B1012010F059F9EB89A3F5007382
:10C060009BB2EB81EB8903F4F05313B928462DF012
:10C0700021F80022234960682EF036FB0022054695
:10C08000214960682EF030FB064605B918B13146EB
:10C090002846FFF7F3FD284631462EF02DF8002202
:10C0A0001A4960682EF020FB054668B111F03CFA91
:10C0B000EB89A3F500739BB2EB81EB8903F4F0539A
:10C0C00013B928462CF0F6FF6068114900222EF0C3
:10C0D0000BFB044678B1FFF745FFE389A3F5007336
:10C0E0009BB2E381E38903F4F05323B92046BDE812
:10C0F00070402CF0DFBF70BD8C2D00207118060041
:10C100009E140600DD170600E71706009D190600BD
:10C110007C1806002DE9F043C38903F5007391B044
:10C120009BB20446C38103A8884615461CF082FAD8
:10C1300090B301212E481CF073F9064648B31FFA4C
:10C1400088F02CF09FFB2B49024620462EF093FAF4
:10C150000022294920462EF0C7FADDF826900090EB
:10C1600007461FFA88F30022294603A8C84700287B
:10C1700016DA2249042028F0F1FC01202CF07AFB89
:10C180001F49024620462EF076FA314638462DF0F9
:10C19000B3FF03A81CF0A8F9204611B0BDE8F08356
:10C1A00001302CF06FFB1749024620462EF063FA4F
:10C1B000022D17D1012114481CF032F90546002840
:10C1C000E3D021462AF080FFEB89A3F500739BB2F0
:10C1D000EB81EB8903F4F053002BD6D128462CF0E9
:10C1E00069FFD2E7214630462AF06EFFCDE700BF57
:10C1F0004F1F06007F200600521B0600671F060027
:10C20000801F0600871F06008C1F060013B5C38918
:10C21000019003F500739BB20C46C3810E492EF0CA
:10C2200009FA022221460198FFF774FF50B1C38931
:10C23000A3F500739BB2C381C38903F4F0530BB918
:10C240002CF038FF01980449012301AA21F070FD68
:10C25000019802B010BD00BF4A1B06002DE9F0474F
:10C260008EB005468A4617462CF002FE814620B164
:10C2700028460021FDF736FC054628462CF045FDF2
:10C28000044638B95748294628F036FC20460EB0F7
:10C29000BDE8F087BAF1000F07D050462CF04DFDF5
:10C2A000044610B951465048EEE7022F16D101A8B6
:10C2B0001CF034F990B100224C4928462EF014FAB3
:10C2C0002EF084FDDDF80D30834204DACDF80D0048
:10C2D00001A81CF01DF901A81CF006F90121444831
:10C2E0001CF09EF8064600287AD0012F6DD14149F6
:10C2F000002023F06BFB044690B9F389A3F500738B
:10C300009BB2F381F38903F4F05313B930462CF058
:10C31000D1FEB9F1000FB9D0002D39D12C46B5E7C7
:10C320003549002023F052FBA046044644B3394669
:10C3300020461CF05BF8BAF1000F10D02F4A51468E
:10C3400020462EF00AFA50B1C389A3F500739BB2C0
:10C35000C381C38903F4F0530BB92CF0ABFE214623
:10C3600030462AF0B1FEB8F1000F04D0424624490D
:10C3700020462EF05FF92A46224920462EF05AF92F
:10C38000314640462DF0B8FEB9F1000F0CD05DB13A
:10C39000EB89A3F500739BB2EB81EB8903F4F053B7
:10C3A00013B928462CF086FE002F7FF46FAF01A84A
:10C3B0001CF040F900283FF469AF01A8214618F0AD
:10C3C000E5FB01A81CF090F860E7022F0CBF0E49B6
:10C3D0000E49002023F0FAFA4FF000080446A5E7C2
:10C3E0000446D1E7ED1E06002A1E06001D1F0600AA
:10C3F0002C1F0600331F06003B1F0600591E0600B7
:10C40000ED3D0600521B0600431F0600481F0600B4
:10C4100070B58EB0044601A80E461CF00BF918B991
:10C42000002420460EB070BD20462CF06EFC58B1A2
:10C430001F482DF0FBFC1F4A0146054620462EF002
:10C440007FF929462DF058FE30462DF062FF054653
:10C45000F8B12CF072FC80B92946174828F04CFB43
:10C46000EB89A3F500739BB2EB81EC8914F4F054D3
:10C47000D6D128462CF01EFED3E7EB89A3F5007336
:10C480009BB2EB81EB8903F4F05313B928462CF0EF
:10C4900011FE204601223146FFF7E0FE044618B1A6
:10C4A000014601A818F066FD01A81CF01DF8B8E7C8
:10C4B0005F200600632006002A1E060038B50446E9
:10C4C0001CF0E8FC00220F4920682EF00DF905460B
:10C4D00038B1002321681A4623F0A6F929462DF029
:10C4E0000BFE206860B1C389A3F500739BB2C381C2
:10C4F000C38903F4F0531BB9BDE838402CF0DABD12
:10C5000038BD00BF4421060038B5054600F0A0FA4A
:10C51000044610B90025284638BD014628461CF0BF
:10C52000F3FC05460028F6D1E389A3F500739BB21E
:10C53000E381E38903F4F053002BEBD120462CF088
:10C54000B9FDE8E700B50A4A13788FB0013B6846A9
:10C550001370FFF7D9FF40B168466FF00502002164
:10C560001CF058FA6846FFF7A9FF0FB05DF804FB0E
:10C57000E62C0020034B00221A705A709A70DA7071
:10C58000704700BF69D4002070B58EB004460D46D8
:10C590000146684616461CF0B7FC48B33EB140F26F
:10C5A000FF339D42A8BF1D46012DB8BF0125BDF92F
:10C5B000143002330FD10F4920462EF087FC0E496C
:10C5C00020462EF083FC0D4920462EF07FFC0C49BE
:10C5D00020462EF07BFC6846ADF814501CF05AFC47
:10C5E000E38903F500739BB2E38120460EB070BD72
:10C5F0000446FAE7121E0600171E06001C1E06005F
:10C60000211E06002DE9F04D2DED028B90B0044661
:10C610000E46014602A890461F469DF868501CF041
:10C6200073FC002800F0998030462EF0A9FE4046A9
:10C63000B0EE408AF0EE608A2EF0A2FE38465BEC47
:10C6400010AB2EF09DFE8DED000BB8F1000F7ED0EB
:10C65000002F7CD00022424B51EC180B32F086FFA9
:10C6600033F034FA00223E4B07465946504632F02A
:10C670007DFF33F02BFA9DED000B0022384B064670
:10C6800051EC100B32F072FF33F020FABDF80D20A0
:10C6900012F4607287F3080386F3080680F308003B
:10C6A00008D0B2F5C07F29D020D8802A2AD0B2F590
:10C6B000807F2CD09DF81320102A2FD1D910B210D2
:10C6C000C90241EA421141EAE000002D43D0059041
:10C6D00002A81CF0DFFBE38903F500739BB2E38142
:10C6E000204610B0BDEC028BBDE8F08DB2F5007FA6
:10C6F00011D0B2F5207FDDD1324601E01A46334633
:10C70000064606E01A46034630461646D2E71A4663
:10C7100003461046CEE71A463346F6E7202A06D1EE
:10C720001A0442EA0622104340F07F40CDE7182A5F
:10C7300004D1190441EA06210843C6E733441844EA
:10C74000B0F5C07F4FF0FF30B8BF0020BDE73046E6
:10C750002DF000FEB9E70690BAE70446C0E700BF37
:10C760000000704010B58EB00C46014668461CF0C3
:10C77000CBFB40B1BDF80530DB0648BF84F00104B7
:10C780001CB1BDF809000EB010BDBDF80700FAE7F6
:10C790002DE9F04F97B00546014608A81CF0B4FB00
:10C7A00028B94FF00009484617B0BDE8F08F00F0F7
:10C7B000DDF804460028F4D000212846FFF7D2FF18
:10C7C000012107462846FFF7CDFF054638469DF86C
:10C7D0002B602CF057F83D49024620462DF04BFFC8
:10C7E00028462CF04FF83A49024620462DF043FFE8
:10C7F000012E07D030462CF045F836490246204637
:10C800002DF039FF05FB07F0704307300021C01001
:10C810002DF0A6FA814668B9E389A3F500739BB2AF
:10C82000E381E38903F4F053002BBAD120462CF0C6
:10C8300041FCB8E70146002203A827F0ABFE002523
:10C84000A846AB46AA46DDE90312914213D30698E7
:10C8500050B1C389A3F500739BB2C381C38903F4AC
:10C86000F0530BB92CF026FC4A461B4920462DF00C
:10C8700002FFA14697E70FFA8BF20FFA8AF108A898
:10C880001CF0D4FA0AF1010A08FA06F8574548EAFA
:10C89000000806EB050203DC0BF1010B4FF0000A68
:10C8A00015460AE0083D28FA05F1C9B203A801922D
:10C8B00027F0DCFC019A4FEA1828072DF2D8D5089A
:10C8C0006FF0070303FB0525BDE700BF1F1D060032
:10C8D0000B1E0600251D06004443060030B551EC32
:10C8E000100B85B053EC112B8DED000B55EC124B5A
:10C8F0008DED021B33F0ACF89DED000B28B19DEDE2
:10C90000021BB0EE410AF0EE610A53EC102B2046F8
:10C9100029468DED000B33F09BF89DED000B08B11F
:10C9200045EC104B05B030BD38B555EC104B00222E
:10C93000002310EE100A294633F08AF810B105F1F1
:10C9400000431D4645EC104B38BD436833B1013BF5
:10C95000436003685A1C0260187870474FF0FF303C
:10C9600070470B685A1C0A601870704705202BF03E
:10C9700021BFFFF7FBBFFFF7F9BF0000024621B35D
:10C98000012924D0022924D0032924D0042924D029
:10C99000052924D0062924D0072924D0082924D009
:10C9A000092924D00A2924D00B2924D00C2924D0E9
:10C9B0000D2924D00E2924D0134B14480F2908BF69
:10C9C00003461349012028F0C9B8124BF9E7124B6E
:10C9D000F7E7124BF5E7124BF3E7124BF1E7124B77
:10C9E000EFE7124BEDE7124BEBE7124BE9E7124B87
:10C9F000E7E7124BE5E7124BE3E7124BE1E7124B97
:10CA0000DFE7124BDDE700BF52370600E9370600CB
:10CA1000F13706005A3706005D3706006637060014
:10CA20006E37060078370600803706008837060024
:10CA3000953706009C370600A2370600B13706007E
:10CA4000C1370600CF370600DB3706004537060042
:10CA5000024B0349586800222DF046BE8C2D002061
:10CA60004F8406000000000008B500222DED028B67
:10CA7000B0EE408AF0EE608A002351EC100B32F0E9
:10CA8000FBFF98B1B0EE480AF0EE680A30F0BCFD4A
:10CA90000B4B51EC100B002232F068FDBDEC028B09
:10CAA00041EC100BBDE8084030F02ABDBDEC028B14
:10CAB0009FED010B08BD00BF000000000000F87FE3
:10CAC0000000E03F00000000F8B555EC104B25F0E9
:10CAD00000474FF0FF32284B2046394632F0E0FF46
:10CAE00060B94FF0FF32244B2046394632F0CEFF7A
:10CAF00020B9B5F1004F08BF002C05D145EC104B13
:10CB0000BDE8F8402BF0ACBE0022002320462946A9
:10CB100032F09EFFC8B912A1D1E900012B4622468E
:10CB200032F06EFB06460F4633F080F804460D46A1
:10CB300054EA05030DD1002200233046394632F075
:10CB400087FF30B19FED080BDAE709A1D1E90001B9
:10CB5000E4E720462946BDE8F8402BF006BF00BFB9
:10CB60002083E4FFFFFFDF3F0000000000000080A3
:10CB70002083E4FFFFFFDFBFFFFFEF7F30F0BCBC8F
:10CB800030F09EB930F058BC08B50B464022014643
:10CB900018462EF061FB402805D10120034927F0FB
:10CBA000DDFF002008BD0120FCE700BFEA360600DB
:10CBB000F8B50F4606460022114938462DF094FD7F
:10CBC0000546D8B12CF0E2F8044648B128462CF0CE
:10CBD000E6F83760706090F82642631E5C425C4164
:10CBE000EB89A3F500739BB2EB81EB8903F4F0535F
:10CBF00013B928462CF05EFA2046F8BD0446FBE740
:10CC0000BE360600F0B585B000AF0023391D0646DC
:10CC10007B602CF03BFE0446F0B9304629F08CFBDB
:10CC20000546786026F010FE05F58073834208D92A
:10CC30001949012027F092FF254628461437BD46A2
:10CC4000F0BDEB1D23F00703ADEB030D6C462A4648
:10CC50002146304629F060FB7B681048FB600022CB
:10CC600007F10801BC601CF08EFB002339463B60D5
:10CC7000F4F74AF93E68054626B9094827F03CFF13
:10CC80003546DAE77B680548BC60324607F10801A3
:10CC9000FB601CF078FBD0E74D0106004BC9020099
:10CCA000CE1A0600F0B583B000AF0023391D06464A
:10CCB0007B602CF0EBFD0446F0B9304629F03CFBDC
:10CCC0000546786026F0C0FD05F58073834208D9DB
:10CCD0001649012027F042FF254628460C37BD465D
:10CCE000F0BDEB1D23F00703ADEB030D6C462A46A8
:10CCF0002146304629F010FB00231A467968204669
:10CD00001CF034FC002339463B60F4F7FDF83E6824
:10CD1000054626B9064827F0EFFE3546DDE73B46D7
:10CD2000044A796820461CF021FCD6E74D01060034
:10CD3000CE1A060063C90200F8B5051E0C4606DCD3
:10CD40002949012027F00AFF00242046F8BD0846A3
:10CD50002BF0DBFF0646A8B10022244920462DF027
:10CD6000C3FC2EF048F900222149064620462DF04A
:10CD7000BBFC2EF02BF830F0080309D0102809D0A6
:10CD80001C49DEE724B122461B49012027F0E6FEBC
:10CD9000012400E002242946204629F00DFE074622
:10CDA0009EB12946204629F007FE0546134900207A
:10CDB00022F00CFE044610B10FB146B13DB92A462F
:10CDC000394620462DF06CF9BEE73546EEE73A4687
:10CDD0000B4920462DF04FFC002DB6D02A460949BC
:10CDE00020462DF048FCB0E7FC3F06001B40060043
:10CDF0003A400600284006003F4006007640060004
:10CE0000444306007F40060070B50D1E064606DA54
:10CE10000B49012027F0A2FE0024204670BD1B20F4
:10CE20002BF0C8FC044615F1FF35F6D326F0E8FCDC
:10CE30000028F2D1314620462CF09BFBF3E700BFDF
:10CE4000E83F060038B504462BF05FFFD8B100225A
:10CE50000E4920462DF048FC05462CF009F810B18B
:10CE600028462CF0B6FC04465DB1EB89A3F50073AF
:10CE70009BB2EB81EB8903F4F05313B928462CF0F5
:10CE800019F9204638BD0446FBE700BFA73F06005E
:10CE9000F8B506460F4614462BF0EAFF0546E8B102
:10CEA00020462BF05AFFD8B120462DF053FA054604
:10CEB00038462EF0FBF804462CF08BFC2D1A13D5C7
:10CEC00000255CB1E389A3F500739BB2E381E3899C
:10CED00003F4F05313B920462CF0ECF82846F8BDC3
:10CEE00030462CF076FCE2E720462CF072FC2F183E
:10CEF00030462CF06EFC8742E2D82A4601232146B8
:10CF00003046F3F799FCB0FA80F56D09D9E7F8B52A
:10CF100007460D4616462BF0ABFF044698B128464F
:10CF20002EF0C4F8002E05460FDA00245DB1EB891F
:10CF3000A3F500739BB2EB81EB8903F4F05313B9B3
:10CF400028462CF0B7F82046F8BD2CF042FC841996
:10CF500038462CF03EFC8442E7D80123324629466D
:10CF60003846F3F769FCB0FA80F46409DEE70000A4
:10CF700070B5002286B00E461D492DF0B5FB044663
:10CF80002BF076FF0546B0B10022214601A827F01C
:10CF900001FB0025DDE9013293421CD3049850B116
:10CFA000C389A3F500739BB2C381C38903F4F05313
:10CFB0000BB92CF07FF85CB1E389A3F500739BB249
:10CFC000E381E38903F4F05313B920462CF072F89F
:10CFD000284606B070BD059800B1C05C864214BFFB
:10CFE000284645F00100C5B201A826F0ADFFD1E703
:10CFF0003A3E0600F0B587B02EF058F805460028F6
:10D0000042D00146002201A827F0C4FA4FF0FF34B5
:10D010000027DDE901639E4225D3049850B1C389FE
:10D02000A3F500739BB2C381C38903F4F0530BB91A
:10D030002CF040F8A742DABFE21B01320022394649
:10D0400028462CF09BFAEB89A3F500739BB2EB8189
:10D05000EB8903F4F053044613B928462CF02AF860
:10D06000204607B0F0BD059800B1805D26F0B0FD08
:10D0700030B9039B1E4437EA240728BF374634469D
:10D0800001A826F061FFC4E70446E9E7F8B50646C3
:10D090000D460AB310462DF05DF9002D044603DA63
:10D0A00030462CF096FB0544002C03DA30462CF079
:10D0B00090FB04441B202BF07DFB25EAE57524EA58
:10D0C000E474074630B1A54204DA631B2A463146B0
:10D0D0002CF011FA3846F8BD00296FF00044E9DA67
:10D0E000DEE7F8B505460C46C2B110462DF032F920
:10D0F00020EAE076002C05DA28462CF06AFB04448E
:10D1000024EAE4741B202BF055FB074620B133467C
:10D11000224629462CF0EFF93846F8BD6FF000465C
:10D12000E8E7F8B507460C46CAB110462DF012F9EB
:10D1300020EAE07524EAE474A542B8BF23464FF024
:10D140001B00BCBF2C461D462BF034FB064620B10D
:10D150002B1B224639462CF0CEF93046F8BD6FF035
:10D160000040E5E708B508B1036823B91B20BDE816
:10D1700008402BF01FBB00212BF0F2F8BDE808405F
:10D180002EF056B870B504462BF0BFFD10B9002440
:10D19000204670BD0022294920462DF0A5FA0646FA
:10D1A0002BF0B3FD002837D00022254930462DF062
:10D1B0009BFA05462BF0C1FD08B35EB1F389A3F5D8
:10D1C00000739BB2F381F38903F4F05313B9304633
:10D1D0002BF070FF002D2ED02C681A4BE31A5C4206
:10D1E0005C41002DD4D0EB89A3F500739BB2EB8199
:10D1F000EB8903F4F053002BCAD1284618E05DB147
:10D20000EB89A3F500739BB2EB81EB8903F4F05338
:10D2100013B928462BF04EFF002EB8D0F389A3F5A2
:10D2200000739BB2F381F48914F4F054AFD130460B
:10D230002BF040FFACE72C46D3E700BF3E020600D0
:10D2400002440600D51E030008B52CF033F908BDD2
:10D2500070B5054686B01B200E462BF0ABFA04468F
:10D2600030B328462BF004FE10B3002E20DB3246EC
:10D27000294601A827F08EF9DDE901239A420AD256
:10D28000059B03B19B5C8DF8033001220DF1030176
:10D2900020462CF0D9F9049850B1C389A3F5007346
:10D2A0009BB2C381C38903F4F0530BB92BF002FF87
:10D2B000204606B070BD37B505461B202BF07AFA24
:10D2C000044628B1294601A826F0BBFD019810B9F3
:10D2D000204603B030BD2DF01CF82DF077FD012263
:10D2E0008DF803000DF1030120462CF0ADF901A8E3
:10D2F00026F092FDEAE7000070B506460D462BF0D9
:10D30000B7FD044630B932461349032027F026FC06
:10D31000204670BD1149002022F058FB32461049CA
:10D3200004462DF087F945B128462BF0A1FD68B9D8
:10D3300032460949032027F011FC00202BF0A2FA05
:10D340000849024620462DF096F9E1E72A460649AB
:10D3500020462DF06FF9F0E7FE3D0600480206007A
:10D36000293E0600303E06003A3E060038B500224F
:10D37000084905462DF0B8F9044640B9064922F09F
:10D3800025FB04490446024628462DF053F9204661
:10D3900038BD00BF67B40600F13D0600F8B507468A
:10D3A0000E462BF0B2FC00283CD000221E49384625
:10D3B0002DF09AF904462BF05BFD70B320462CF05B
:10D3C00008FA002E01DD864206D3174938462DF0B3
:10D3D0007DFD25462846F8BD3246002120462CF02A
:10D3E000CDF86FF000423146054620462CF0C6F8D5
:10D3F0000D49024638462DF03EF9002CEAD0E3896B
:10D40000A3F500739BB2E381E38903F4F053002B8F
:10D41000E0D120462BF04EFEDCE71B202BF0CAF9B2
:10D420000546EAE70546D5E7A73F060038B50C46AE
:10D43000054651F8043B9847002DA2BFA36901336C
:10D44000A36100280BDB04F11C05C1B2284626F0BD
:10D4500060FF284626F0BEFD63690133636138BD75
:10D460002DE9F04F89B000AF0D469246804621F07D
:10D4700093FA4FF0010BF91D0446284687F807B0D0
:10D48000F4F714FA0023064607F108015046BB6082
:10D490002CF0FCF90546F0B9504628F04DFF8146C6
:10D4A000B86026F0D1F909F58073834207D9454960
:10D4B000584627F053FB2437BD46BDE8F08F09F1ED
:10D4C000070323F00703ADEB030D6D464A462946DB
:10D4D000504628F021FFBB68002BECD0142C1DD146
:10D4E000394A1278002AE6D0F9793848BD6100221D
:10D4F00091427A61FA61BB754FF0402114BF134627
:10D50000202307F114027E75F7F7DAFD02460028A2
:10D51000D1D02F49042027F021FBCCE7002CCAD121
:10D520002C49224640462DF0DFF88146014607F19E
:10D530000C001EF0C1FE90B32246274940462DF054
:10D54000D3F82DF058FD3B7CB874FF2B27D07A7CA4
:10D55000FF2A24D07A753B75B875FA681F4B93FB88
:10D56000F2F307F11400012BD8BF2346D7F808B017
:10D5700097F807A0BB611EF065FE710001F4FF7112
:10D5800007F114001EF016FEA34514DCBAF1000FDB
:10D5900003D007F114001EF021FEBB7DBB74B87CE4
:10D5A0002BF068F90C49024640462DF043F84946F5
:10D5B0002CF0A2FD7FE7295D07F114001EF0FAFDB3
:10D5C0000134E1E74D010600F8D10020B8CA00207F
:10D5D0003D3B0600513B06005A3B060090D003003D
:10D5E0002DE9F04F93B000AF0E461546814621F06D
:10D5F000D3F94FF0010A044607F11701304687F8C6
:10D6000017A0F4F753F9002D804606DC4FF0000810
:10D6100040464C37BD46BDE8F08F26F015F905F5BC
:10D620008073834204D95F49504627F097FAEDE7AB
:10D63000EB1D23F00703ADEB030D142C6E463BD11D
:10D64000594B1B78CBB1002307F120024FF040214A
:10D650005648C7F82230C7F826307B8587F820A0C7
:10D6600087F8218087F822507E62F7F729FD02466D
:10D6700018B14F49042027F071FA2946012029F0FA
:10D680009BF980460028C1D00146002207F1200006
:10D6900028F02EFC354416F8011B07F1200026F077
:10D6A00038FE07F1200026F095FCB542F3D107F1D2
:10D6B000200026F027FBABE7002CA7D13D492246EE
:10D6C00048462DF011F88246014607F118001EF079
:10D6D000F3FD002859D02246374948462DF004F87A
:10D6E0002DF089FC3B7FB877FF2B4ED07A7FFF2A45
:10D6F0004BD0F97D87F8212087F82030BA6987F868
:10D7000022002E4B93FBF2F307F12000012BD8BF30
:10D710002346F9607B621EF095FD4FEA480101F453
:10D72000FF7141F0010107F120001EF043FD05F1FA
:10D73000FF38A8EB04035942594108224FF0000B6F
:10D7400007F12000C7E901121EF0DCFCBA68796815
:10D750004FEA4B0B013A40EA0B0BF1D107F12000E5
:10D760001EF0FEFC012197F8210014F0C3F906F821
:10D7700004B00134A542DCD1FB681BB107F12000E5
:10D780001EF02CFD97F82230BB77B87F2BF072F893
:10D790000949024648462CF04DFF51462CF0ACFC9E
:10D7A0006BE700BFA93A0600F8D10020B8CA0020F4
:10D7B000DE3A0600513B06005A3B060090D00300BB
:10D7C0002DE9F04F89B08946009021F0E5F84946EF
:10D7D000044602A81EF070FD40B3142C40F00281F4
:10D7E0009DF80C40204621F0D1F99DF80D5018B15C
:10D7F000284621F0CBF9E0B9224629468A4827F08D
:10D800007BF9B9F1000F00F00A81884A0098494677
:10D810002CF096FF50B1C389A3F500739BB2C3816E
:10D82000C38903F4F0530BB92BF044FC09B0BDE8F5
:10D83000F08F7F49029E7F4B04EB440405EB4505C6
:10D840000C440D449E4294F801806F7858DD7A4B69
:10D850009E42D4BF4FF080664FF0CD66774A784C39
:10D8600013785BB323681BB1764B1021C3F880108B
:10D870004FF040234FF0FF31C3F80813D3F80012E4
:10D880000021C3F80012C3F80015012184F822100A
:10D8900094F8271079B9D3F808154FF0A04001F596
:10D8A000E07140F2023540F82150D3F80C3503F511
:10D8B000E07340F82350002384F8223094F822309B
:10D8C00001251570FBB108225F49042027F046F9B5
:10D8D0009DF80C40204621F059F920B14FF42071F9
:10D8E000204614F08FFA9DF80D40204621F04EF9A5
:10D8F000002886D04FF49451204614F083FA80E734
:10D900004FF0CC76AAE79DF81E2084F827209DF8DA
:10D910001D20A360C4E9003384F8253084F8243046
:10D9200072B34FEA8800B90000F1A04001F1A041B4
:10D9300040F20C624FF0A04BC0F8002705FA08FA3D
:10D94000C1F80027BD4040F20D620193CBF808A555
:10D95000CBF80855C0F80027C1F800270420F5F7D8
:10D9600065F8019BDBF810150D422BD043B14FF049
:10D97000A04A0420CAF80C55F5F758F8CAF808551B
:10D980004FF0A04308F5E07140F20C6243F821200B
:10D9900007F5E07143F821204FF040231D46C3F8FE
:10D9A0000885C3F80C75C3F8246522681AB10621EE
:10D9B0000420F7F7DFFD0523C5F80035022384F8BE
:10D9C000223085E701930420CBF80CA5F5F72EF85B
:10D9D000CBF808A50420F5F729F8019B0133092BA2
:10D9E000C0D1C4E7002C7FF40CAF9DF80C00FF28D9
:10D9F00007D0012114F07EF803219DF80C0014F0EB
:10DA000023FB9DF80D00FF283FF4FBAE012114F02D
:10DA100071F803219DF80D0014F016FBF1E603499F
:10DA200000982DF053FA01E7F13A0600513B060049
:10DA30008002060097AB020087F50400F8D10020B1
:10DA4000B8CA002000E100E0203B0600F0B58DB030
:10DA50000D4616461C4620F09FFF13289DF848707F
:10DA600005D02E49012027F079F80DB0F0BD16B988
:10DA70000CB90F2403262A4B1B78F6B2E4B25BB92B
:10DA80002849ADF810306FF0FF02CDE9011201A86E
:10DA9000254A039214F0D4F9FF2F03D00021384611
:10DAA00021F072FE28462BF058F970B128462CF070
:10DAB00051FC22463146C0B2F3F702FCFF2FD4D00E
:10DAC0000121384621F060FECFE728462BF0FBF914
:10DAD000E8B1802383F311880122294601A828F0A8
:10DAE0004AFA01A826F05DF9054601A825B926F0F5
:10DAF00019F985F31188E1E726F04BFB2246314600
:10DB0000C0B2F3F7DDFB01A826F07EFAE9E72A466A
:10DB10000649012027F022F8D0E700BF4D3F06005C
:10DB2000EAD10020A086010000010800753F060030
:10DB3000F0B58DB00D4616461C4620F02DFF13287B
:10DB40009DF8487005D02F49012027F007F80DB047
:10DB5000F0BD16B90CB9032401262B4B1B7806F037
:10DB60000F0604F00F045BB92849ADF810306FF0D0
:10DB7000FF02CDE9011201A8254A039214F060F9D1
:10DB8000FF2F03D00021384621F0FEFD28462BF060
:10DB9000E4F870B128462CF0DDFB22463146C0B2D5
:10DBA000F3F74EFBFF2FD2D00121384621F0ECFDD8
:10DBB000CDE728462BF087F9E8B1802383F311885D
:10DBC0000122294601A828F0D6F901A826F0E9F893
:10DBD000054601A825B926F0A5F885F31188E1E7E7
:10DBE00026F0D7FA22463146C0B2F3F729FB01A846
:10DBF00026F00AFAE9E72A460649012026F0AEFF98
:10DC0000D0E700BF253F0600EAD10020A086010032
:10DC100000010800753F060013B50C4620F0BCFE5D
:10DC20008DF807000938062805D80DF107020349C9
:10DC3000204628F011FA02B010BD00BF31E002000A
:10DC400070B586B00E4602AA01A91CF0D3FC60B1E3
:10DC50006EB9FF2502AA0199304628F0FDF9FF2D83
:10DC600003D00121284621F08FFD06B070BD316838
:10DC70000029EEDD013930462AF072FB04462BF014
:10DC8000D5F930B3204620F012FF0546304629F082
:10DC900097F950B1C389A3F500739BB2C381C389BF
:10DCA00003F4F0530BB92BF005FA5CB1E389A3F54B
:10DCB00000739BB2E381E38903F4F05313B9204668
:10DCC0002BF0F8F9FF2DC5D00021284621F05CFD8E
:10DCD000C0E7002CBDD0FF25E8E700002DE9F041AA
:10DCE00098B00E46174607A908AA1CF083FC002826
:10DCF00000F0A780FF2F03D00021384621F044FD1B
:10DD000030462BF02AF880463046B8F1000F1AD082
:10DD10002CF020FB08A920EAE070079B9847002818
:10DD200004DA08A94FF0FF30079B98472AF0AAFDB4
:10DD30000446FF2F03D00121384621F025FD20465F
:10DD400018B0BDE8F0812BF093F80546002850D0BC
:10DD50001B202AF02FFD31460446424602A826F039
:10DD600019FC4646DDE902239A4218D3059800289B
:10DD700032D14645DDDD25F043FD0028D9D108A983
:10DD8000079B4FF0FF30984701228DF807000DF1F7
:10DD90000701204608F101082BF056FCE9E725F0C1
:10DDA0002FFD0028E2D1069808B1029BC05C079BBA
:10DDB00008A99847002806F1010609DB8DF807003D
:10DDC00001220DF10701204608F101082BF03CFC6F
:10DDD00002A826F0B9F8C5E7C389A3F500739BB282
:10DDE000C381C38903F4F053002BC2D12BF062F935
:10DDF000BFE7304628F0A0FA0146012028F0DCFDFC
:10DE00000446002895D001462A460EA8CDE90C55B7
:10DE100028F06EF807AA0C49304628F01DF9DDE914
:10DE20000C239A4203DB0EA825F06CFF81E725F056
:10DE3000E7FC0028F7D107A94FF0FF30FFF7F6FA0B
:10DE4000EDE704467BE700BF2DD402007FB50C460A
:10DE5000054620F0A1FD2146064668461CF026FB3B
:10DE6000B0B1132E16D1684613F0EAFF54B3184A26
:10DE7000214628462CF064FC50B1C389A3F50073F9
:10DE80009BB2C381C38903F4F0530BB92BF012F991
:10DE900004B070BD002EFBD19DF80500FF2802D014
:10DEA000012114F0D1F89DF80600FF2802D00421CA
:10DEB00014F0CAF89DF80700FF28D7D0012114F00C
:10DEC000C3F8D3E7024928462DF000F8E0E700BF89
:10DED000513B0600F2F77DBD2DF0C6BEF0B589B00E
:10DEE0002AF021FD044638B310224FF4DA25002130
:10DEF0000DEB02000095F1F715FB04A928462DF063
:10DF00003BFDC8B101AD06AE0027059B01330CD126
:10DF100096E8030085E8030028468DF80C702BF086
:10DF200085FF014620462AF027F8002204A968460A
:10DF30002DF074FD0028E8D1204609B0F0BDF7B5FA
:10DF4000074608460C4616461D462AF0DEFE00B37C
:10DF500000222046114609F061FF002504462E46A6
:10DF600038462DF0BDFE009533462246F2F7E8FD17
:10DF700005465CB1E389A3F500739BB2E381E389B5
:10DF800003F4F05313B920462BF094F8284603B05D
:10DF9000F0BD002CE4D0E28902F5007292B2E28179
:10DFA000DEE738B52DF09CFE2DF09EFD044688B1CD
:10DFB00000212BF0A5FCE389A3F500739BB2E3815C
:10DFC000E38903F4F053054613B920462BF072F8A9
:10DFD000284638BD0546FBE708B52DF081FEBDE8B3
:10DFE00008402DF081BD38B52DF07AFE2DF07CFD76
:10DFF000044680B106F0B2FAE389A3F500739BB240
:10E00000E381E38903F4F053054613B920462BF06E
:10E0100051F8284638BD0546FBE708B52DF060FEEF
:10E02000BDE808402DF06DBD4FF4DA202DF090BD15
:10E030000B78C1B218461EF0E5BD00002DE9F04393
:10E0400089B01F4680460C46914620F0A5FCA0F101
:10E050000903DBB2062B06463AD80F280FD1374BFF
:10E060001B7863B94FF0FF324FF41651CDE904121B
:10E0700004A8334A06928DF81C30F7F7A1FA314D07
:10E080008DF80060B9F1000F03D020462DF00EF896
:10E0900004466A462946204627F0DEFFB9F1000F04
:10E0A0000CD05CB1E389A3F500739BB2E381E389F3
:10E0B00003F4F05313B920462AF0FCFF2FB1694650
:10E0C0000D20A84769460A20A84709B0BDE8F0839B
:10E0D0000028FAD102461C4940462CF005FB324686
:10E0E00005461A4940462CF0FFFA0DF11008064685
:10E0F0000246294640461DF0FDFE5EB1F389A3F5B8
:10E1000000739BB2F381F38903F4F05313B93046E3
:10E110002AF0D0FF5DB1EB89A3F500739BB2EB81D0
:10E12000EB8903F4F05313B928462AF0C3FF98E8AB
:10E130000F006D4607C52B70054DA3E7F9D10020F0
:10E1400008000100F1CF0400B4360600513B060080
:10E15000B9C3040000231A46FFF770BF01231A4613
:10E16000FFF76CBF00230122FFF768BFF0B585B051
:10E17000044620F011FC002205463C4920462CF0C4
:10E18000B3FA064628B93A49012026F0E7FC05B063
:10E19000F0BD0022374920462CF0A6FA324601464F
:10E1A000074668461DF0A6FE394630462BF0A4FF10
:10E1B000304920462CF08AFE2C4920462CF086FE61
:10E1C000A5F10903DBB2062B44D900222A492046D7
:10E1D0002CF08AFA08B32CF0F9FDC4B200212046D5
:10E1E00013F06CFB00201DF019FE0546A8B1214676
:10E1F00029F0BCFF044618B1014628462CF0FAFD70
:10E2000028462AF0F1FF20B91C4B1D4958682CF014
:10E210005DFE294620462BF06FFF9DF80600FF2883
:10E2200002D0002113F010FF9DF80700FF2802D054
:10E23000002113F009FF9DF80400FF2802D00021FF
:10E2400013F002FF9DF80500FF28A0D0002113F075
:10E25000FBFE9CE7A5F10E03DBB2012BDDD8FF220C
:10E26000002128461EF0ACFBD7E700BF513B06005B
:10E27000F03E0600B4360600173F06008C2D002045
:10E280001C3F0600F0B585B005460F46144620F049
:10E2900083FB0646D4B922465B4928462CF024FA73
:10E2A00004462246394668461DF024FEA0B95CB1FA
:10E2B000E389A3F500739BB2E381E38903F4F05390
:10E2C00013B920462AF0F6FE05B0F0BDE38903F548
:10E2D00000739BB2E381E4E700982AF0D3FA4B493C
:10E2E000024628462CF0C7F97CB12246464928460A
:10E2F0002CF0C1F9A6F10903DBB2062B0AD80F2EC8
:10E30000E2D16846F7F75CF9DEE73F4928462CF092
:10E31000DDFDEFE7002ED7D19DF80500FF2807D0DF
:10E32000012113F091FE01219DF8050021F02CFA46
:10E330009DF80400FF280BD0052113F085FE602016
:10E340002AF028FB044660B93149012026F006FC7A
:10E350009DF80630FF2BB7D02E49012026F0FEFB9A
:10E36000B2E702462C4928462CF085F920462AF0CF
:10E3700016FD002680F84060044613F0D5FB009B94
:10E380009DF80A2084F85860C4E914369DF80830D6
:10E3900013449DF80920B24218BF0133C4E91201A9
:10E3A00084F8593001219DF8040013F087FA0446DF
:10E3B00010B32AF067FA1949024628462CF05BF997
:10E3C00001201DF02BFD06460028C1D02A4621461B
:10E3D00029F048FFF389A3F500739BB2F381F38919
:10E3E00003F4F05313B930462AF064FE013C0C4BA1
:10E3F0000C4A43F82420ABE79DF804200A49012089
:10E4000026F0ACFBA4E700BF513B0600B436060083
:10E410006B3E0600C83E0600913E0600173F060010
:10E42000A4D6002039BE0400993E060010B50C4663
:10E4300020F0B2FAA0F10903DBB2062B04D8214682
:10E44000BDE810401FF012BE02490120BDE8104097
:10E4500026F084BB403E06002DE9F3471F4601230A
:10E4600013600C690646894615460CB10B68E45CDE
:10E4700030782E2800F0E3805B282CD101237B72BA
:10E4800096F801A0BAF15E0F02D12B6801332B6020
:10E490004FF000080CE03B4601AA4946FFF7DCFFBD
:10E4A0002B68019A48EA000813445FFA88F82B6049
:10E4B0002B68F45CF018002C00F0C3805D2CEAD1CE
:10E4C00001332B6000237B72BAF15E0F14BF444608
:10E4D00088F001040BE05C2866D102232B60707881
:10E4E000642808D1303C092C8CBF0024012420462C
:10E4F00002B0BDE8F087442805D1303C092C94BF18
:10E5000000240124F3E7662864D06E2864D07228C2
:10E5100064D0732805D1204602B0BDE8F04725F04D
:10E5200057BB532806D1204625F052FB80F001004E
:10E53000C4B2DCE7742853D0762853D077280DD1A5
:10E54000A4F13003092B7AD9204625F035FB0028A9
:10E5500075D15F2C14BF00240124C8E757280CD1C3
:10E56000A4F13003092B66D9204625F025FB0028AD
:10E5700061D15F3C18BF0124B9E7A0F13003DBB2E1
:10E58000092B31D978280FD1B3786BB1F3785BB10F
:10E5900004232B60B07825F0AEFA8046F07825F0A1
:10E5A000AAFA40EA0810C0B27B7AFBB12B68F35C90
:10E5B0002D2B1BD178812868013028603B4601AAA9
:10E5C00049463044FFF748FF2B68019A134404463C
:10E5D0002B608CE70C20E7E70A20E5E70D20E3E756
:10E5E0000920E1E70B20DFE71846DDE73A7A62B160
:10E5F000A4F14103192B98BF2034A0F1410398BF27
:10E60000E4B2192B9CBF2030C0B2B7F90A30B3F581
:10E61000807F12D0DBB22AB1A3F14102192A9CBF3C
:10E620002033DBB24FF480729C427A8103D3844260
:10E6300001D8984263E7002459E784428AE701241D
:10E6400055E70249012026F089FA50E752410600B9
:10E6500082B02DE9F047B2B00C463AA9064681E8EF
:10E660000C0025F0CDF830B10025284632B0BDE8C9
:10E67000F04702B0704733780BB17C2B5AD1582247
:10E680003AA91CA831F086FCDDE93A67DDF8F48090
:10E690002AF049F9A26823681A440546D21B394674
:10E6A00030462AF06BFF002104460246284629F036
:10E6B000D9FD5CB1E389A3F500739BB2E381E389E3
:10E6C00003F4F05313B920462AF0F4FC0DF1800A4C
:10E6D0004FF00009C1450DDB38462AF0D3F89149C7
:10E6E000024628462BF0C7FF32468F4928462BF0BA
:10E6F000A1FFBAE75AF8041BDAF820203046521A74
:10E700002AF03CFF09F10109044602464946284621
:10E7100029F0A8FD002CDDD0E389A3F500739BB29E
:10E72000E381E38903F4F053002BD3D120462AF090
:10E73000C1FCCFE75E2B09D12368A268D34293D1F5
:10E7400027F026FA00288FD0013607E0242B1DD1B0
:10E75000D4E900329A4206F101060CD850223CA9B5
:10E76000684631F017FC3AAB0CCB21463046FFF738
:10E770006FFF054679E74C223DA9684631F00AFC57
:10E780003AAB0ECB304600F0FAFAF2E7282B0FD165
:10E790003D9B2168A2683AA80A44191D082B40F83D
:10E7A000212000EB83014A63CADC01333D93C7E7B4
:10E7B000292B0AD13D9B002BC2DD3AAA02EB830331
:10E7C0002168A2680A441A63BAE73AAB1BAA214639
:10E7D0003046FFF741FE1B9FF35DA3F12A02012A99
:10E7E000804606EB070500F284800137374450B9B4
:10E7F0002B2B08D14C223DA9684631F0CBFB3AAB1C
:10E800000ECB3846BFE7214614A814AD25F016FEFE
:10E810000FCD0DF1700CACE80F0050222B68CCF836
:10E8200000303CA9684631F0B5FB3AAB0CCB1CA9D3
:10E830003846FFF70DFF05461F9850B1C389A3F571
:10E8400000739BB2C381C38903F4F0530BB92AF060
:10E8500031FCD4E900239A42BFF407AFB8F1000FAE
:10E860003FF403AF204625F06FFB3AAB1BAA2146CD
:10E870003046FFF7F1FD2146804614A825F0DEFD65
:10E880000DF1500EBEE80F000DF1700CACE80F005A
:10E890005022DEF80030CCF800303CA9684631F058
:10E8A00079FB3AAB0CCB1CA93846FFF7D1FE814669
:10E8B0001F9850B1C389A3F500739BB2C381C3896C
:10E8C00003F4F0530BB92AF0F5FBB9F1000F0ED0A9
:10E8D0005DB1EB89A3F500739BB2EB81EB8903F487
:10E8E000F05313B928462AF0E5FB4D46B1E7A94697
:10E8F000FBE7D4E900239A420BD250B1204625F021
:10E9000023FB27F045F900283FF4AEAE1B9B1E44C5
:10E9100024E74C223DA9684631F03CFB3AAB0ECBD4
:10E92000284630E7744106007A4106002DE9F04799
:10E93000BAB08046084614AF2CF0B8FB00228349D9
:10E94000054640462BF0D0FE2CF040FA00228049CC
:10E95000824640462BF0C8FE06462AF089FA044655
:10E9600040B9314628462BF0C7FB20469837BD46B4
:10E97000BDE8F08730462AF02CFF00F1080323F0B1
:10E980000703ADEB030D0DF15009421C494630461B
:10E990002CF062FC5EB1F389A3F500739BB2F381A6
:10E9A000F38903F4F05313B930462AF083FB69214D
:10E9B0004046FEF7DDFA4FF48072002387F84800E6
:10E9C000A7F84A202946524607F1180087F849302F
:10E9D000FB643D6425F0DEFD07F11801384625F0A3
:10E9E0002DFDBC46BCE80F0007F12C040FC45022DB
:10E9F000DCF80030236007F148016846C7F844A0FE
:10EA000031F0C8FA07F140030CCB07F12C0148465E
:10EA1000FFF71EFE0446B86B564650B1C389A3F5F6
:10EA200000739BB2C381C38903F4F0530BB92AF07E
:10EA300041FB07F1180025F087FA07F1400A1CB9DD
:10EA4000D7E906239A4229D3786A50B1C389A3F53E
:10EA500000739BB2C381C38903F4F0530BB92AF04E
:10EA600029FB5DB1EB89A3F500739BB2EB81EB89C8
:10EA700003F4F05313B928462AF01CFB002C3DD1B7
:10EA8000022029F097FE00250446284629F0FAFEC8
:10EA90002E49024640462BF0EEFD66E707F11801CD
:10EAA000384625F0CBFCBC46BCE80F0007F12C042F
:10EAB0000FC40136DCF800302360502207F1480112
:10EAC00068467E6431F066FA9AE80C0007F12C0182
:10EAD0004846FFF7BDFD0446B86B50B1C389A3F5A6
:10EAE00000739BB2C381C38903F4F0530BB92AF0BE
:10EAF000E1FA07F1180025F027FAA0E76721404660
:10EB0000FEF736FA00B30021204629F029FC002246
:10EB10001049064620462BF0E7FD2CF057F9054634
:10EB200030462AF056FE0544002EAED0F389A3F5F8
:10EB300000739BB2F381F38903F4F053002BA4D14B
:10EB400030462AF0B7FAA0E705469EE7303E0600B9
:10EB5000293E0600744106002DE9F84F05460E4691
:10EB60002AF086F920B94FF000084046BDE8F88F3A
:10EB700029F0D9FE80460028F5D01EB9294628F094
:10EB8000A3FAF2E73046F2F77FF9002800F081801F
:10EB9000002029F077FE6A49024630462BF06BFDD3
:10EBA00029463046FFF7C2FE0027044684B12046BE
:10EBB0002AF068F8814618B3E389A3F500739BB285
:10EBC000E381E38903F4F05313B920462AF072FA83
:10EBD000002029F057FE5A49024630462BF04BFDE3
:10EBE00028462AF0F6FDB842BFD339466FF00042FE
:10EBF00028462AF0C3FC0146404629F0BDF9B4E797
:10EC00004946204629F0ACFB4A464E4982462046FA
:10EC10002BF06AFD2CF0DAF8814650462AF0D9FD37
:10EC20008346BAF1000F0ED0BAF80E20A2F500729A
:10EC300092B2AAF80E20BAF80E2002F4F05212B9DD
:10EC400050462AF037FAA9EB0702394628462AF03F
:10EC500095FC0146404629F08FF9E389A3F500733E
:10EC60009BB2E381E38903F4F05309EB0B0713B97B
:10EC700020462AF01FFA384629F004FE30490246A1
:10EC800030462BF0F8FC29463046FFF74FFE04468D
:10EC90008CE730462CF00AFA064698B12AF099FD26
:10ECA000814628462AF095FD002700F1010BABEBC9
:10ECB000090A3C46544531DCB9F1000F1CD1C4B9F6
:10ECC0000134F7E78146ECE75C461FE00146404629
:10ECD00028F0FAF9FB89A3F500739BB2FB81FB894D
:10ECE00003F4F05313B938462AF0E4F904EB0907AA
:10ECF000E6E754450AD111E05445E5D00123224608
:10ED000031462846F1F798FD0028D9D1E21B394653
:10ED100028462AF033FC07460028D7D1002E3FF4BE
:10ED200024AFF389A3F500739BB2F381F38903F455
:10ED3000F053002B7FF419AF30462AF0BBF914E7EB
:10ED4000303E06007441060038B5FFF7EFFD05467A
:10ED500020B129F097FF80F00100C0B200F001045B
:10ED60005DB1EB89A3F500739BB2EB81EB8903F4F2
:10ED7000F05313B928462AF09DF9204638BD84B0D7
:10ED8000F0B59BB021AE054686E80E0026F000FFE8
:10ED900068B9044620461BB0BDE8F04004B0704797
:10EDA0005C2C03D16C78002CF4D03D4601352C78D6
:10EDB000002CEFD07C2C05F10107F1D1DDE9211207
:10EDC00015A825F0E7FB502223A9684631F0E2F8A8
:10EDD00096E80C0015A93846FFF73AFC0446189847
:10EDE0000028D7D0C389A3F500739BB2C381C38920
:10EDF00003F4F053002BCDD12AF05CF9CAE70000F0
:10EE0000F7B5064608460D46144629F096FF30B978
:10EE10002A463349032025F0A1FE03B0F0BD6CB3B0
:10EE20000022304930462BF0B9FB0090C0B12BF0E6
:10EE300074FA012300906A46002029461EF02AFF3A
:10EE400000980028E9D0C389A3F500739BB2C38161
:10EE5000C38903F4F053002BDFD12AF02BF9DCE750
:10EE6000214F0022394630462BF03EFC044638B98B
:10EE70002A46394630462BF0DDFBCEE71B4FF0E744
:10EE800029F03BFF78B12946204628F01DF9E38997
:10EE9000A3F500739BB2E381E38903F4F053002BE5
:10EEA000BBD12046D9E702216846CDE9004529F0CB
:10EEB0003DFD39460546024630462BF0BBFB002D92
:10EEC000E5D0EB89A3F500739BB2EB81EB8903F4EA
:10EED000F053002BDBD128462AF0ECF8D7E700BF2F
:10EEE0006236060086360600583606005D36060095
:10EEF00010B500220446FFF783FF2046BDE810400E
:10EF0000FEF734BA38B5154601220446FFF778FFFC
:10EF100025B1002229462046FFF772FF2046BDE8B2
:10EF20003840FEF723BA00002DE9F04F85B00546C2
:10EF300029F0C9FF044640B92A464849032025F074
:10EF40000DFE204605B0BDE8F08F4549002020F0B9
:10EF50003DFD04460028F4D048F20801414829F05C
:10EF6000D8FC06460028ECD022463F49DFF8F8B02E
:10EF70002BF060FB29F0D7FC2946824603A824F039
:10EF800060FF4FF0000847460398D8B9A7EB080088
:10EF900029F078FC3549024620462BF06CFB52469E
:10EFA000334920462BF067FBF389A3F500739BB22E
:10EFB000F381F38903F4F053002BC2D130462AF0D9
:10EFC00079F8BEE72BF0A5F90546FEF7DBF8002837
:10EFD0003BD048F26001274829F09BFC8146384627
:10EFE00029F050FC00210246019048462BF022FEF9
:10EFF000019B5BB1DA89A2F5007292B2DA81DA89FB
:10F0000002F4F05212B918462AF054F82246594632
:10F0100048462BF00FFB494632462846FFF772FF61
:10F0200049462BF069F85DB1EB89A3F500739BB2FB
:10F03000EB81EB8903F4F05313B928462AF03AF830
:10F0400003A8013724F0E8FE9EE72A4639465046D9
:10F0500029F008F908F10108E5E700BFC13D060005
:10F06000F13D060085F102006C180600E63D060041
:10F07000EC3D0600C5F0020037B5054601910F488A
:10F0800048F2080129F045FC0446A8B12A460C497B
:10F090002BF0D0FA012301AA214628461EF0FAFDE2
:10F0A000E389A3F500739BB2E381E38903F4F05392
:10F0B00013B9204629F0FEFF03B030BD3FF4020033
:10F0C0006C1806002DE9F0410F46904618490022C1
:10F0D00006462BF009FB2BF079FE00220546154968
:10F0E00030462BF001FB0446F8B142463946013D5B
:10F0F00029F0B8F8284629F0C5FB0D4902463046EC
:10F100002BF0B9FA1DB921463046FFF7B5FFE38968
:10F11000A3F500739BB2E381E38903F4F05323B9B1
:10F120002046BDE8F04129F0C5BFBDE8F08100BF31
:10F13000E63D0600EC3D060037B5054601910F4857
:10F1400048F2080129F0E5FB0446A8B12A460C491B
:10F150002BF070FA012301AA214628461EF09AFDE1
:10F16000E389A3F500739BB2E381E38903F4F053D1
:10F1700013B9204629F09EFF03B030BD39F40200D8
:10F180006C18060038B500220D460D4904462BF0D8
:10F19000ABFAA0B1C389A3F500739BB2C381C38945
:10F1A00003F4F0530BB929F085FF204604492BF0F6
:10F1B0008DFE29462046BDE83840FFF7BDBF38BD6B
:10F1C000EC3D06002DE9FF4106461046019114462C
:10F1D00029F093FD0746002852D0214603A824F0C9
:10F1E00030FE0024039810BB454930462BF06EFEDC
:10F1F000444930462BF06AFE0022434930462BF04A
:10F2000073FA4149054630462BF060FE24F01AF9A6
:10F21000804600283ED001462846FFF78DFF2A464B
:10F22000214640462AF03CFF04B0BDE8F0812BF0B7
:10F2300070F801AB01223146054620F0F5FAEFB92E
:10F2400050B1C289A2F5007292B2C281C38903F49F
:10F25000F0530BB929F02EFF5DB1EB89A3F50073D4
:10F260009BB2EB81EB8903F4F05313B9284629F0E4
:10F2700021FF03A824F0D0FD0027B3E70446EBE705
:10F28000002CB1D0204601AB0122314620F0CCFA4F
:10F290000446A9E74DB32046FDF774FF50B348F28A
:10F2A00008011A4829F035FB48F2080106461848BB
:10F2B00029F02FFB0746A6B198B12A4615493046DA
:10F2C0002BF0B8F92A46134938462BF0B3F901223E
:10F2D00031462046FFF794FD424639462046FFF767
:10F2E0008FFD394630462AF007FF294620462AF08E
:10F2F00003FF99E721462846FFF7BEFEF5E700BF6A
:10F30000583606005D36060067B4060079F0020044
:10F3100039F102006C180600414B2DE9F047B2F1BB
:10F3200000080E464FF000023E493F4F054608BF19
:10F330001F462BF0D9F9044668B1C389A3F50073C1
:10F340009BB2C381C38903F4F053002B66D1BDE89F
:10F35000F04729F0AFBE012029F08CFA314902466E
:10F3600028462BF088F92246394628462BF0BCF96E
:10F37000044600284ED102462C49DFF8B0902846BA
:10F380002BF0B2F90446CCB9B8F1000F3BD03246AD
:10F39000274928462BF04EF9002C3FD02246314613
:10F3A0002846FFF70FFFE389A3F500739BB2E381C3
:10F3B000E38903F4F0538BBB2046C8E700223946AB
:10F3C00020462BF091F98246024648B1314620464C
:10F3D000FFF7F8FE21465046BDE8F0472AF08CBE04
:10F3E000494620462BF080F9E389A3F500739BB2D0
:10F3F000E381E38903F4F053824613B9204629F0F0
:10F4000059FE5446BFE732460A490120BDE8F0479D
:10F4100025F0A4BBB8F1000FC0D0B8E7BDE8F08775
:10F420005D3606008F3606005836060067B40600C3
:10F4300086360600943606000022FFF76DBF0122D3
:10F44000FFF76ABF2DE9F74F12F06EFB89460746BA
:10F4500027F094FB834612F067FB80468A46FDF74F
:10F4600085FA0446002800F0A580554B5549586898
:10F4700000222BF039F90546002800F09F8028F083
:10F4800076FFEB89A3F500739BB2EB81EB8903F464
:10F49000F053064613B9284629F00CFE4A490025C8
:10F4A00001235A1E12018818B0F80EC01CF03F0F3D
:10F4B0000DD0CDE9003229F069FC0135009B4249AD
:10F4C00028B1019A8A580F321209134415440133A6
:10F4D00040F6C4129342E4D9B018AB1B401B009312
:10F4E00029F0D0F93949024620462BF0C4F8009B98
:10F4F000184629F0C7F93649024620462BF0BBF8DA
:10F5000040F6C41029F0BEF93249024620462BF0DD
:10F51000B2F8304629F0B6F92A49024620462BF0C7
:10F52000AAF8584629F0AEF92B49024620462BF09E
:10F53000A2F8B8EB07006AEB09012FF0E9FF0022FF
:10F54000264B30F013F8264B002230F00FF841EC38
:10F55000100B29F085F92349024620462BF08BF841
:10F56000214829F08FF92149024620462BF083F8E3
:10F57000002029F087F91E49024620462BF07BF82F
:10F580001C4829F07FF91C49024620462BF073F8ED
:10F590004FF4DA2029F076F91849024620462BF07C
:10F5A0006AF84FF4002029F06DF91549024620460B
:10F5B0002BF061F8204603B0BDE8F08F06466DE7FA
:10F5C0008C2D0020533D0600AC2D00205B3D060035
:10F5D000603D0600663D06006C3D060000408F4021
:10F5E0000000B03E6F3D0600E0E30020763D0600DF
:10F5F000863D060034C40600923D0600A33D060089
:10F60000B43D060010B5FDF7B1F9044629482AF0CB
:10F610000DFC2949024620462BF02DF827482AF0F8
:10F6200005FC2749024620462BF025F825482AF0FC
:10F63000FDFB2549024620462BF01DF84FF4002023
:10F6400029F020F92149024620462BF014F84FF406
:10F65000803029F017F91E49024620462BF00BF89E
:10F6600006F050F81B49024620462BF004F81A4BCE
:10F670001B78093BDBB20B2B96BF184A184852F88F
:10F6800023002AF0D3FB1749024620462AF0F3FF55
:10F6900015482AF0CBFB1549024620462AF0EBFF1D
:10F6A000134829F0EFF81349024620462AF0E3FFF9
:10F6B000204610BDA53C0600AD3C0600B53C06004A
:10F6C000BD3C0600C83C0600CF3C0600D53C060009
:10F6D000A15B0600DB3C0600E72C00202836060074
:10F6E00026B60600E23C0600EA3C0600453D060060
:10F6F000E82C00204D3D060038B50849054600209D
:10F7000020F064F9044638B1284629F022F904496A
:10F71000024620462AF0AFFF204638BD623B060075
:10F72000433806002DE9F74F0D4603210446CDE985
:10F73000002312F089FC4FF0000B4FF0010A4FF04C
:10F740008008D94615F1FF3502D203B0BDE8F08F2D
:10F75000009B0AEA0306019B0BEA030756EA07032C
:10F7600016D088F311880021204612F0C3F90A2030
:10F770000AF096FF0121204612F0BCF989F31188A6
:10F7800037200AF08DFF1AEB0A0A4BEB0B0BD9E777
:10F7900088F311880021204612F0ACF941200AF0CC
:10F7A0007FFF0121204612F0A5F989F31188052079
:10F7B000E7E710B40C7802460023204608215DF8E4
:10F7C000044BFFF7AFBF2DE9F8430D460321074671
:10F7D00012F03AFC002401264FF08008A14615F1F2
:10F7E000FF3502D22046BDE8F88388F31188002156
:10F7F000384612F07FF903200AF052FF0121384603
:10F8000012F078F90A200AF04BFF384612F05EF940
:10F8100000B1344389F3118835200AF041FF7600A6
:10F82000DDE710B50321044612F00EFC002120464E
:10F8300012F060F94FF4FA700AF032FF012120460D
:10F8400012F058F950200AF02BFF204612F03EF932
:10F8500004464FF4D2700AF023FF84F00100C0B2D6
:10F8600010BD000008B5002203492AF03DFFBDE8A5
:10F8700008401FF077B900BF433806002DE9F04F6C
:10F880008BB00C46FFF7EEFF06461FF07FF928B954
:10F890004FF0000840460BB0BDE8F08F29F043F868
:10F8A00080460028F4D0631EFF2B28BFF024224698
:10F8B000E317CDE900234FF000093046FFF7B1FF11
:10F8C0000028E7D0DDE9002308213046FFF72AFFB2
:10F8D00001240025AA46274601213046FFF773FF81
:10F8E00001215FFA80FB3046FFF76DFFBBF1010F8E
:10F8F000C0B22BD101283AD1402FCBDD9DF80C307E
:10F90000002BC7D005AC0DF10C090025A34619F852
:10F91000017B380923F0A2FF207007F00F0023F0CD
:10F920009DFF0135082D607004F10204EFD1002322
:10F9300058468DF824302AF079FA0146404628F0DE
:10F940001BFBD146BAF1000FA4D0B6E70AAB2B449B
:10F95000834513F81C3C2DD14F4524DA1C4214BFBB
:10F960004FF0010B4FF0000BBBF1000F21D00AABA1
:10F970002B444FF0010B13F81C3C23430AAA2A44E2
:10F98000012102F81C3C30465A4600236400FFF770
:10F99000C9FE14F0FF0404BF01350124072D07F14F
:10F9A000010799DDA8E70CBF4FF0010B4FF0000BEA
:10F9B000DAE7BA4623EA0403E0E770B58AB00C46FA
:10F9C000FFF750FF06461FF0E1F868B3204629F024
:10F9D000C4F918B320462AF0BDFC014605460120B3
:10F9E00026F0EAFF044650B101460022684626F0A0
:10F9F0007FFA15F1FF3505D2684624F083F92046D9
:10FA00000AB070BD08213046FFF7DDFEC1B268467E
:10FA100024F07FFC684624F0DDFAEAE7082130464E
:10FA2000FFF7D1FE28F02EFF0446E8E737B50D4674
:10FA30001446FFF717FF8DF807001FF0A7F880B1F5
:10FA40000DF107020C49284626F006FB9DF8070039
:10FA50004CB1012112F04EF801219DF8070012F07F
:10FA6000F3FA03B030BD042112F0EEFA01219DF843
:10FA7000070012F03FF8F4E7B3F7020010B5FFF704
:10FA8000F1FE04461FF082F838B12046CC22002354
:10FA90000821BDE81040FFF745BE10BD2DE9F04735
:10FAA00086B00C46FFF7DEFE07461FF06FF840B148
:10FAB000204629F0DDF938B922463049032025F0E7
:10FAC0004DF806B0BDE8F087204629F082FE1028E8
:10FAD000F2D13846FFF7A5FE2146002201A824F006
:10FAE00059FD0024A146A046A246059B0BB1019AF0
:10FAF0009B5C8DF8003001A824F026FA059B0BB121
:10FB0000019A9B5C8DF8013001A824F01DFA0023B6
:10FB10001A46102168468DF802A024F064F8A4F17A
:10FB20002002C4F12003A14000FA02F220FA03F3FC
:10FB30001143A0401943083440EA090641EA080588
:10FB4000402CB146A846D0D1049850B1C389A3F542
:10FB500000739BB2C381C38903F4F0530BB929F03E
:10FB6000A9FA3846552200230821FFF7DBFD32466B
:10FB70002B4640213846FFF7D5FDA2E76A3B060039
:10FB800010B5FFF76FFE04461FF000F820B12046C5
:10FB9000BDE81040FFF745BE10BD00002DE9F7435A
:10FBA00005460F46904629F0C8F8044640B92A4653
:10FBB0006E49032024F0D2FF204603B0BDE8F08355
:10FBC000284629F067F8002835D0A988286828F049
:10FBD000A0FE04460028EFD02946684624F031F9FB
:10FBE000009E002E37D0F38903F500739BB2F3819A
:10FBF00030462AF08EFB8146304629F08DF920B33D
:10FC0000B9F1000F33D0012130462AF0B7FD054687
:10FC100078B1014620462AF013FCEB89A3F5007366
:10FC20009BB2EB81EB8903F4F05313B9284629F01A
:10FC300041FA01250AE0284629F076F8002814BF89
:10FC40000820072028F0B6FDC3E7054649463046A0
:10FC50002AF052FA6DB9B8F1000F0ED1009D002DB7
:10FC600057D13A46424920462AF0E4FCA4E74D46E3
:10FC7000ECE7684624F0D0F8B2E7414601A824F04A
:10FC8000E0F801980028E9D02AF043FB009D0646E1
:10FC9000A5B1EB8903F500739BB2EB81284629F0EF
:10FCA0003BF988B9EB89A3F500739BB2EB81EB8933
:10FCB00003F4F05313B9284629F0FCF93246002129
:10FCC00020462AF0B7FF13E00122002128462AF03F
:10FCD00025FF314680462AF015F9414620462AF094
:10FCE000AFFB284641462AF007FA684624F094F80C
:10FCF0005EB1F389A3F500739BB2F381F38903F43A
:10FD0000F05313B9304629F0D5F901A824F084F84E
:10FD1000B7E7EB8903F500739BB20122EB81114633
:10FD200028462AF0FBFE064678B1014620462AF016
:10FD300087FBF389A3F500739BB2F381F38903F486
:10FD4000F05313B9304629F0B5F9EB89A3F50073E8
:10FD50009BB2EB81EB8903F4F05313B9284629F0E9
:10FD6000A9F9684624F058F878E700BF9F390600E3
:10FD70006C1806002DE9F04F8FB0814602AF104697
:10FD80008A46164629F09FF8044600285ED0304681
:10FD900029F053FD4028834680460AD9024630495F
:10FDA000012024F0DBFE002420463437BD46BDE8A8
:10FDB000F08F8300DA1D22F00702ADEB020D02ADD9
:10FDC0002A462B440021934219D101223146381D85
:10FDD00026F0D1F8381D23F0E4FF98B9381D23F040
:10FDE000A1FF00231946CDE900855246484627F079
:10FDF000AFFA2946044640462AF000F9D4E742F813
:10FE0000041BE0E7381D23F05AFF044629F017F9D8
:10FE100058B120462AF09EFA061E06DBB34504DDE3
:10FE2000381D24F06AFB45F826005CB1E389A3F590
:10FE300000739BB2E381E38903F4F05313B92046C6
:10FE400029F038F9381D24F0DFF8C3E72EB1324627
:10FE50000449012024F082FEA6E7B0463546C0E7FB
:10FE60001C3906006439060001381F289DBF034B6A
:10FE700023FA00F000F00100002070478B808080A2
:10FE80002DE9F04317461D46421E47F6FE739A427F
:10FE90008FB08146884602D84A1E9A4205D96449E5
:10FEA000012024F05BFE002408E03846FFF7DCFF69
:10FEB000044638B95F49012024F050FE20460FB0B7
:10FEC000BDE8F0835C4900201FF080FD0446002857
:10FED000F4D0684619F0C8F8002628468DF804606A
:10FEE0008DF805608DF806600094ADF80790ADF8C8
:10FEF00009808DF80B7028F008FF002865D0324685
:10FF00004E4928462AF0F0FB2BF075F828B1BDF8D1
:10FF1000053043F00103ADF805300022484928467A
:10FF20002AF0E2FB2BF067F828B1BDF8053043F06A
:10FF30000403ADF805300022424928462AF0D4FBDC
:10FF40002BF059F828B1BDF8053043F00803ADF89F
:10FF5000053000223C4928462AF0C6FB2BF04BF81E
:10FF600088B19DF80B0001280BD1BDF8053043F096
:10FF70000203ADF80530BDF809305B0703D0334903
:10FF80008FE733498CE72846002232492AF0ACFB40
:10FF90000546D0B1304929F0D5F950B92F49284646
:10FFA00029F0D0F9C0B9BDF8053043F08003ADF8B1
:10FFB0000530EB89A3F500739BB2EB81EB8903F469
:10FFC000F05313B9284629F075F8684618F0E2FB9B
:10FFD000684618F05FFF71E72149284629F0B2F919
:10FFE00020B9BDF8053043F48073E0E71D49284689
:10FFF00029F0A8F920B9BDF8053043F4C073D6E75D
:020000023000CC
:100000001949284629F09EF920B9BDF8053043F476
:100010000073CCE71549284629F094F920B9BDF8BA
:10002000053043F42073C2E7114824F045FDC0E7D2
:10003000701C06007D1C06004E1C0600D63906000A
:10004000DD390600E1390600ED3906002B3A0600DD
:10005000FB390600643A0600703A0600743A06005E
:10006000783A06007C3A0600803A0600843A060098
:10007000883A06002DE9F74F21F0004589461646DB
:100080001F464FF0FF32414B2946804604462FF071
:1000900007FD002876D14FF0FF323C4B4046294601
:1000A0002FF0F4FC00286DD132463B4630463946ED
:1000B0002FF0F6FC002865D1002200234046494677
:1000C0002FF0C6FC28B309F100450022002330467A
:1000D00039462FF0BDFC10B107F100431F46002246
:1000E0000023304639462FF0A9FC78B94FF0FF3293
:1000F000264B304639462FF0B5FC38B14FF0FF3271
:10010000224B204629462FF0ADFCE8B900240025FB
:1001100022E04D46D9E700221D4B204629462FF00C
:1001200025FACDE90001B246BB4652465B46DDE901
:1001300000012FF0A1FC52465B46E0B9204629465B
:100140002FF05CF804460D4622462B4630463946D1
:100150002FF088FC0028DED10022002340464946CB
:100160002FF076FC10B105F100431D4620462946CC
:1001700003B0BDE8F08F104619462FF041F88246D3
:100180008B46D2E70024034DF0E700BFFFFFEF7F6F
:100190000000E03F0000F87F2DE9F84355EC114BDB
:1001A00011EE100A294657EC106B2FF08FFC09282E
:1001B000804619D82FF070F922462B462FF03EFCCE
:1001C00090B1B8F1000F63D030463946B8F1010F55
:1001D00003D141EC100BBDE8F88332463B462FF0CB
:1001E000C5F908F1FF38F1E700220023304639460F
:1001F0002FF02EFC0022D8B3284B20462946FFF7CB
:1002000039FF002200232FF019FCF0B300224FF039
:10021000804320462946FFF72DFF002200232FF0C0
:100220000DFCB04607F1004949EC108B68B12DF088
:10023000EBF922462B4651EC100B2FF097F9BDE855
:10024000F84341EC100B2DF05BB92DF0DDF922469F
:100250002B4651EC100B2FF089F941EC100B2DF0CF
:100260004FF953EC102B10EE100A03F10041B0E7E8
:100270000023304639462FF0E1FB30B10022002345
:10028000204629462FF0EEFB28B147EC106BCEE755
:10029000002002499DE7002000219AE70000F03F7E
:1002A00037B50D46014668461446FCF781FC98B107
:1002B000019890F82532013B022B0DD874B181686A
:1002C00029441BF07AF9014630B10548054B002C52
:1002D00008BF1846FCF752FB03B030BD2146EFE7DC
:1002E000903806009F38060070B50E4E34783CB941
:1002F00018F02AFF054628B90B49012024F02EFCEE
:10030000204670BD09490A4801221BF041FD014603
:1003100018B10848FCF732FBF2E7012333702C4692
:10032000EEE700BF6DD40020FE36060026B60600BC
:1003300070D400202F3706002DE9F04790B0044616
:100340000E46FFF7D1FF08B900242AE0214601A894
:10035000FCF72EFC0028F7D0029B93F8252202F030
:10036000FD02012AF0D100220092DD689B68ED1A9F
:10037000EAD026EAE676B54228BF3546284628F078
:1003800009FB0446C8B1029E28F009FD6B460146F0
:100390002A4630461BF0A9F9014610B12848FCF75F
:1003A000EDFA204610B0BDE8F0871AF8081003A84F
:1003B00023F04EFD08F1010823E005468146AE42D8
:1003C00026D9771B202F28BF20270DF1200A6B4646
:1003D0003A4651460298CDF800901BF086F98046C7
:1003E00040BB009B83B154B91B2028F0E3F90446BD
:1003F0000028A9D00146424603A824F0CBF84FF0CC
:100400000008009B4345D0D8009BBB421D44D6D07A
:10041000002C99D006980028C3D0C389A3F5007397
:100420009BB2C381C38903F4F053002BB9D128F0E8
:1004300041FEB6E701460248FCF7A0FAE8E700BF34
:100440007C3806002DE9F04F9BB005460C46FFF7BF
:100450004BFF002800F00B81294605A8FCF7A8FBFC
:1004600028B94FF0000B58461BB0BDE8F08F069B33
:1004700093F82532023B012BF3D8012221460FA825
:1004800025F079FD4FF0000B0FA823F08AFC08B986
:10049000054659E007AC0027A2460FA823F079FED5
:1004A00004F8010B0FA823F0AFFD0FA8013723F0CC
:1004B00078FC08B1202FF0D1069C204618F08AFE67
:1004C0000546002840F0CB80E379002B40F0C68041
:1004D000A3799E0740F1C680A368FB42814604D2FF
:1004E00004F124030393A3684FB9D4E90232934281
:1004F00088BFE360A37943F02003A3711DE0C3F339
:100500000802002A40F09780206890F8028008F1E5
:10051000FF3808EA532818F0FF02029230D123BBBB
:10052000216921B91AF028FC01460028DDD00129F3
:100530001DD14FF00203E3710225CB44B9F1000F46
:1005400000F09380002D9FD00FA823F0EBFB494BC8
:100550001B781B0702D406981BF0C2F9002D82D02D
:1005600029464548FCF70AFA7DE76169DAE7481C45
:1005700002D10125E571E0E72369616103B92161D9
:10058000A3795A060CD52068A26903994078012303
:100590001AF014FA0028ECD1A37923F04003A371D8
:1005A000236861690193184618F0AFFE0028C0D097
:1005B000029BB7F5007F00EB03082AD3019B029A48
:1005C0009B7801987E0A32449A4288BF029A40780A
:1005D00088BF9E1A3346424651461AF0EFF900286A
:1005E000C7D1A169A1EB08018E420AD94FF400726C
:1005F0000AEB4121039818F093FEA37923F04003FE
:10060000A3717602A3683344B244A360B144BF1B14
:1006100069E7A36998450CD0D4E902329A4208D917
:10062000019803994078012342461AF04DF90028B9
:100630009FD1C4F81880A068C0F30800C0F5007608
:10064000BE4228BF3E46243032465146204418F070
:1006500067FEA37943F04003A371D3E71D464FF033
:1006600000096AE78146072567E701256CE78346AD
:10067000F9E600BF6FD40020AE38060037B5044657
:10068000FFF732FE002841D021466846FCF790FA79
:1006900000283BD0019C94F82632012B36D120460D
:1006A0001BF01EF920B9204618F094FD00B9206017
:1006B000019B1749022283F82622164B0022586814
:1006C0002AF012F8054608B30122009927F0D3FC5E
:1006D000044678B1014628462AF08CFBE389A3F54D
:1006E00000739BB2E381E38903F4F05313B920460E
:1006F00028F0E0FCEB89A3F500739BB2EB81EB895A
:1007000003F4F05313B9284628F0D4FC03B030BDED
:10071000753806008C2D002037B5214B21495868CB
:10072000002229F0E1FF0446A0B1014601A823F010
:1007300088FB0198E8B920462AF0ECFBE389A3F591
:1007400000739BB2E381E38903F4F05313B92046AD
:1007500028F0B0FC144B1A782AB10022114610463A
:100760001A701BF015FBFF21002018F0FDFC03B0F0
:1007700030BD29F0CEFD0546FFF780FF5DB1EB8966
:10078000A3F500739BB2EB81EB8903F4F05313B92B
:10079000284628F08FFC01A823F03EFBC9E700BFE4
:1007A0008C2D0020753806006DD40020FFF7B4BFF3
:1007B00038B504460D4628F0A8FA30B922460C494F
:1007C0000120BDE8384024F0C9B928461EF0DEF902
:1007D00028B908490120BDE8384024F0BFB9FFF727
:1007E0009BFF29462046BDE8384018F0BDBC00BF3D
:1007F000F9370600243806002DE9F04FC1B0044651
:100800000F46FFF771FD68B3AE4BAF49586803223E
:1008100029F06AFF824628B300253C22294611A808
:100820001095EEF77FFEA94B8DF80A501B88ADF8A6
:100830000830002C00F00A8110AE21463046FCF74B
:10084000A3F9814680B9BAF80E30A3F500739BB2C4
:10085000AAF80E30BAF80E3003F4F05313B950462C
:1008600028F028FC0024E0E027B1032202A9384642
:100870002AF0F2FC954902A82FF0B4FB002800F002
:10088000EC80934902A82FF0ADFB002800F00C810A
:10089000904902A82FF0A6FB002800F009818E499C
:1008A00002A82FF09FFB002800F006810024ADE095
:1008B00028F075FA5A4607468849204629F0DBFE9B
:1008C000012387F824320023039687F8255287F8FE
:1008D00026323B6008F01E0203A907A81BF050F85F
:1008E0000646C8B904AB0D93039920AB07A80E9335
:1008F0001AF09AFB0C9D064610B9002D08BF06267B
:1009000018F01C0F00F09580BEB1042E04D107A88A
:100910001AF0EEFC0646C8B1E389A3F500739BB25A
:10092000E381E38903F4F05313B9204628F0C2FBB6
:1009300031466B48FCF722F8B8E7EB7A13F0110F59
:1009400040F0828018F0080F36D002E00C9D48F08D
:10095000080818F0EFFCC0F30723EB73030C002624
:10096000A8732B74000E079B6874EE722E776E7757
:10097000AE77EE7718780193294618F01DFC019B9D
:10098000AE760122EE762E756E7583461A7198B199
:100990001A6B0192014618461AF0E2FD019A0646CA
:1009A0000028B9D107980BF1FF33C36011461AF044
:1009B0007EF806460028AFD1079E336B18F0080F6B
:1009C00018BF48F02008C7E9073587F806804FF0C0
:1009D000000887F807803078294618F0EDFB386169
:1009E000EB69C7F81880C7E902833E60F388BB80D3
:1009F000B9F1000F03D0F96838461AF0DEFD012383
:100A000087F826322146504626F05EFBBAF80E30B3
:100A1000A3F500739BB2AAF80E30BAF80E3003F4B7
:100A2000F05313B9504628F045FB204641B0BDE8CD
:100A3000F08F002E7FF470AFEB7ADA060BD418F04B
:100A4000020FB9D0DB07B7D5072665E72549012096
:100A500024F084F8DAE704265EE74FF001088146C7
:100A60004546214900201EF0B1FF044600283FF40E
:100A70001DAF40F2272027F08DFF834600287FF42A
:100A800017AF1A4A137843F008031370E389A3F5EC
:100A900000739BB2E381E38913F4F0557FF406AF52
:100AA000204628F007FB01E74FF012080225D8E79F
:100AB00081464FF00A08F9E781464FF012080325F6
:100AC000CFE700BF8C2D00207538060023360600C6
:100AD000B9840600A85E060047380600BE36060048
:100AE0004A3806005E380600703806006ED40020D2
:100AF00038B50446174829F099F9014605462046BD
:100B0000FFF77AFE04465DB1EB89A3F500739BB253
:100B1000EB81EB8903F4F05313B9284628F0CAFAA5
:100B2000B4B16FF000412046FFF706FC05462046B1
:100B3000FFF7A4FDE389A3F500739BB2E381E3898A
:100B400003F4F05313B9204628F0B4FA284638BD10
:100B50002546FBE7233606002DE9F04FC7B00446D3
:100B600000213C2217A81691EEF7DCFC54BBFFF7DE
:100B7000BBFB002800F0C48016AB099318F0DAFB29
:100B80000122064609A90DA81AF0FAFE044698B9F2
:100B90000AAB1393099926AB0DA814931AF044FAE3
:100BA0000446002800F0D280042805D1139BD97A8E
:100BB00011F020010FD0062465482146FBF7DEFE28
:100BC000002005E0214616A8FBF7DEFF0028CED165
:100BD00047B0BDE8F08F0D981AF0CEF80546002812
:100BE00000F0AA80012D0D9800F0AC806B1C00F085
:100BF000AB8019F056FF0446002840F09E80DDF8D7
:100C000034A02946504618F080FB0AF13408074604
:100C10000AF50D73C146994574D10AF13F02434666
:100C20002021934271D110238AF83F30F3B201930F
:100C30008AF84A30C6F3072302938AF84B30C6F38A
:100C4000074303938AF84C30330E04938AF84D30EF
:100C50002E0CEBB22E2405938AF84E305FFA86FBF9
:100C6000C5F30723360A8AF84F30202241468AF816
:100C700034408AF848B08AF849600AF15400069373
:100C800018F04EFB0D9A8AF8554011780F9B0329F6
:100C900003D1916A8B4208BF00238AF86E30C3F3F8
:100CA00007211B0C8AF868301B0A8AF869308AF819
:100CB0006F1092F802A00123BA44574528D10DA81D
:100CC0001AF016FB0446002837D1129B0D9883F8C2
:100CD00014B01022DA72019A9A75029ADA75039AA0
:100CE0001A76049A5A76059A9A76069ADA765E7594
:100CF000012303711AF0A4FD044600287FF45CAFC1
:100D0000012065E709F8014B85E703F8011B88E737
:100D10000D98791C07630371079119F09FFE044633
:100D200058B90799404601230022814501D10F4659
:100D3000C3E700F8012BF8E7072429460D981AF0BD
:100D40000FFC39E70224F8E70124F6E7082433E72B
:100D5000C338060070B5C8B0044600213C2219A86B
:100D60001891EEF7DFFB34B9FFF7BEFA50B9002453
:100D7000204648B070BD214618A8FBF705FF0028A3
:100D8000F2D1F4E72022002107A8EEF7CBFB18AB45
:100D9000002203A90FA803931AF0F2FD0028E6D160
:100DA00004AB28AE039915930FA816961AF03CF9D8
:100DB00005460028DBD1149B002BD8D007A90FA82B
:100DC00018F022FAFBF7D2FD04460028D0D007988D
:100DD00027F058FD21490246204629F04CFC9DF899
:100DE0002400C0F3001027F045FD1D4902462046AF
:100DF00029F041FCBDF820305A0A02F2BC7212926E
:100E0000C3F34312013A03F01F030FA8119210938A
:100E100007F0ECF9BDF822302890DA0A2C92C3F3DF
:100E2000451203F03F032B92CDE9295309F0A6FAAE
:100E30002D90304607F058FACDE9000109492846BF
:100E40001EF0C4FD9DED000B054602F0B9FC2A46DC
:100E50000549204629F00FFC8AE700BFA9010600DA
:100E6000F7380600FB38060000390600F0B5C7B0B9
:100E7000044600213C2217A81691EEF753FBD4B983
:100E8000FFF732FA00287BD016AB0122694604A88E
:100E900000931AF075FDE8B901AB0A93009926ABEF
:100EA00004A80B931AF0C0F8A0B90A9BDB7A9A0643
:100EB00009D506200EE0214616A8FBF765FE00289E
:100EC000DED147B0F0BD09990029F2D0CC7AE30712
:100ED00006D5072001463248FBF750FD0020F0E719
